:020000040800F2
:10000000F8FF0120E11509087D1609088D2805086B
:100010007D1609087D1609087D16090800000000F4
:100020000000000000000000000000007D1609082C
:100030007D160908000000007D16090869480408BB
:100040007D1609087D1609087D1609087D16090820
:100050007D1609087D160908E51704080D1804081F
:10006000351804085D1804088518040849030000C1
:100070005D03000071030000850300009903000088
:10008000AD030000C10300007D1609087D160908B4
:100090007D1609087D1609087D160908AD180408A3
:1000A0007D160908212C04087D160908112C040866
:1000B000312C0408412C0408512C0408591404085C
:1000C0004D1404088D140408811404087D160908D1
:1000D0007D160908C1300000893200006D3400002F
:1000E000ED1804087D160908000000000D2D040815
:1000F000E52C04081D2D0408D52C0408D5030000A8
:100100007D1609087D160908612C04087D1609086A
:10011000553600003D380000712C0408C957080806
:10012000E9030000FD0300001104000025040000A5
:10013000390400007D1609087D1609087D16090896
:1001400000000000000000000000000000000000AF
:100150004D0400006104000075040000253A000011
:10016000C1140408B51404087D1609087D16090891
:100170007D1609087D1609087D1609080000000093
:100180007D1609087D1609080D3C0000F53D0000AC
:100190007D1609087D1609087D1609087D160908CF
:1001A0007D1609087D1609087D1609087D160908BF
:1001B0007D1609087D1609087D160908F51404083E
:1001C000E91404087D1609087D1609087D1609083A
:1001D0007D160908094E08087D1609087D160908CC
:1001E0007D1609087D1609087D1609087D1609087F
:1001F0007D1609087D1609087D1609087D1609086F
:100200007D1609087D1609087D1609087D1609085E
:100210002D2D04083D2D04084D2D04087D160908D8
:100220007D1609087D1609087D16090800000000E2
:100230007D1609087D160908000000007D160908D2
:100240007D1609087D1609087D1609087D1609081E
:100250007D1609087D1609087D1609087D1609080E
:100260007D1609087D1609087D1609087D160908FE
:100270007D1609087D160908DD3F0000000000001A
:100280007D160908000000007D1609080000000026
:08029000000000007D160908C2
:020000040804EE
:10000000114A037A0168D35C10B4CC58CA1824F0A2
:100010000104CC501368DB07FCD4037D1F2B09D9E6
:10002000203B20225DF8044B02FA03F343F018034F
:10003000CB60704720225DF8044B02FA03F343F0D3
:1000400018038B60704700BF20B109084368426DF8
:1000500030B49A61EFF31182502383F31288416820
:10006000D2B2856C0B68046D23EA050323430B6051
:1000700082F31188436981681A68096822F00102D5
:10008000D0E908541A60826A1D605C615A60D0E948
:100090000B429C60DA600023B0F86C2030BCCA626E
:1000A00003777047002A4FEA014C034630B508BF7A
:1000B000E64600F1C00514BF8E468C460024196840
:1000C0000C3353F8042C43F8084C41EA0C0142EA83
:1000D0000E02AB4243F80C1C43F8042CEFD1D0F8CD
:1000E000C03043EA0E03C0E93144C0F8C03030BD2F
:1000F00010B40C4C6368002B11DD002004F1080CD7
:100100000146DCF8AC3003F1C00259600C33934275
:10011000FBD1013063680CF5867C8342F1DC5DF82D
:10012000044B704704000020F0B5404C04EB401332
:1001300093F8543403B9F0BD3D4B42011D7893F858
:1001400001C065450CD00CEB4C0E03EBCE0E9EF8B7
:1001500004604FEA4C0E771E012F5AD9032E52D05D
:100160002244A2F83814EFF31181902383F312880C
:1001700092F83A34C9B2B2F8380443EA4003002096
:100180009BB282F83A0481F311881909207881EA38
:1001900013215940D8B1C9431B01D2F8505401244E
:1001A000D2F83C049BB201F00F01D5F8AC2084409A
:1001B0000B4302F1C000590013F4004F8BB202D17F
:1001C0005168214351600C329042F4D1F0BDD2F815
:1001D0003C041B01D2F8502401F00F0110309BB2F7
:1001E0000124D2F8AC200B43844002F1C000590036
:1001F00013F4004F8BB202D15168214351600C328D
:100200009042F4D1F0BD0CF1010606F00306AE42B7
:10021000A6D0E64403EBCE030344597C00299FD0CB
:10022000A318012083F83A049AE700BF04000020D5
:10023000801A0024704700BF024B03EB401393F871
:100240005504704704000020D0E90920131A5842D1
:100250005841704790F8573830B53BB990F8551869
:10026000012490F85638DAB2914200D830BD04FA31
:1002700003F2B0F85E5801332A43A0F85E28F2E793
:100280000379024613F0010006D0D2E90731D268A3
:100290005B1A013A03EA0200704710B5037904467D
:1002A00013F001030ED0FFF7EBFF034650B1226AB3
:1002B0006369E1689B5C0132B2FBF1F0DBB201FBE8
:1002C00010222262184610BD03799B070AD5436AA3
:1002D0008269D154436A02690133B3FBF2F102FB34
:1002E00011334362704770470171704703790146CB
:1002F00013F0020007D00B69D1E90921013B521A22
:100300001A40D2B2981A704710B584464FEA810E4F
:10031000102312F4004F4FEA420214BF0E240724A8
:10032000013B92B2CCF80040F444F2D100EB8112D0
:100330008C010351122042F8213010BD10B58446C3
:100340004FEA810E0424130B013C4FEA021203EB27
:10035000430392B203F11803CCF80030F444F2D115
:1003600000EB01130A018450062043F8214010BD20
:10037000704700BF704700BF00EB4000024B03EB2B
:10038000C00393F84905704704000020064B93F81A
:10039000F825824206D900EB400003EBC003D3F8F6
:1003A0004C05704700207047040000201D4B93F857
:1003B000FC25AAB3D3F8381509B100200860012A3A
:1003C0002ED0D3F8501509B100200860022A27D09A
:1003D000D3F8681509B100200860032A20D0D3F8AB
:1003E000801509B100200860042A19D0D3F89815A7
:1003F00009B100200860052A12D0D3F8B01509B160
:1004000000200860062A0BD0D3F8C81509B10020D7
:100410000860072A04D0D3F8E0350BB100221A6037
:10042000704700BF040000201D4B93F8FC25AAB3C1
:10043000D3F8381509B100200860012A2ED0D3F86E
:10044000501509B100200860022A27D0D3F868159A
:1004500009B100200860032A20D0D3F8801509B123
:1004600000200860042A19D0D3F8981509B100209B
:100470000860052A12D0D3F8B01509B10020086031
:10048000062A0BD0D3F8C81509B100200860072A46
:1004900004D0D3F8E0350BB100221A60704700BFDA
:1004A00004000020C34B1B78002B40F04D81C24B51
:1004B00093F8FC25002A00F0478193F8481530B5E1
:1004C00000294ED1D3F838150020012A086047D9F9
:1004D00093F86015002966D1D3F850150020022A40
:1004E00008603DD993F87815002940F0C980D3F809
:1004F00068150020032A086032D993F89015002966
:1005000040F0E080D3F880150020042A086027D945
:1005100093F8A815002940F0F680D3F8981500202C
:10052000052A08601CD993F8C015002940F00D81F8
:10053000D3F8B0150020062A086011D993F8D81511
:10054000002959D1D3F8C8150020072A086007D917
:1005500093F8F025002A72D1D3F8E03500221A6012
:1005600030BDD3F83C25910AA1F58011522940F203
:100570000D814FF0FE0CEFF31181502080F31288B3
:100580008E4C4FF02C0E556AC9B250690EFB0C4CC4
:10059000013540F00100CCF88C50506181F3118896
:1005A00093F8FC258EE7D3F85425910AA1F5801124
:1005B000522940F2EF804FF0FE0CEFF311815020F2
:1005C00080F312884FF02C0E556A7C4CC9B25069EA
:1005D00001350EFB0C4440F00100C4F88C50506112
:1005E00081F3118893F8FC250020D3F85015022AD6
:1005F00008603FF677AFB3E7D3F8CC25910AA1F5B1
:100600008011522900F2E2806D4810F801C0EFF32A
:100610001181502080F312884FF02C0E556A674CE0
:10062000C9B2506901350EFB0C4440F00100C4F81A
:100630008C50506181F3118893F8FC2582E7D3F840
:10064000E425910AA1F58011522900F2C2805C488C
:1006500010F801C0EFF31181502080F312884FF0A1
:100660002C0E556A554CC9B2506901350EFB0C442D
:1006700040F00100C4F88C50506181F311886BE7A1
:10068000D3F86C25910AA1F58011522940F2868099
:100690004FF0FE0EEFF31181502080F312884FF0DF
:1006A0002C0C556A454CC9B2506901350CFB0E44FF
:1006B00040F00100C4F88C50506181F3118893F828
:1006C000FC2514E7D3F88425910AA1F5801152295D
:1006D00068D94FF0FE0CEFF31181502080F312889F
:1006E0004FF02C0E556A354CC9B2506901350EFBDE
:1006F0000C4440F00100C4F88C50506181F3118823
:1007000093F8FC25FEE6D3F89C25910AA1F580110B
:1007100052294BD94FF0FE0CEFF31181502080F39A
:1007200012884FF02C0E556A244CC9B2506901351D
:100730000EFB0C4440F00100C4F88C50506181F372
:10074000118893F8FC25E8E67047D3F8B425910AA0
:10075000A1F58011522935D94FF0FE0CEFF311812C
:10076000502080F312884FF02C0E556A134CC9B2FA
:10077000506901350EFB0C4440F00100C4F88C5068
:10078000506181F3118893F8FC25D1E60C4810F8EC
:1007900001C0F0E60A4810F801C00EE7084810F85A
:1007A00001E077E7064810F801C094E7044810F824
:1007B00001C0B1E70000002404000020801A0024DA
:1007C00060330908044810F801C0C7E74FF0FE0C79
:1007D0001DE74FF0FE0C3DE76033090800EE100AFC
:1007E000B8EE400A704700BFBCEEC00A10EE103AE7
:1007F00098B2704707280AD84FF4B472054B02FB31
:100800000033B3F80006B0FA80F0400970470020CA
:10081000704700BF04000020072807D8044B4FF49E
:10082000B471012201FB003383F80226704700BF38
:1008300004000020072808D8044B03EB401393F86A
:10084000542412B1012283F83A2470470400002096
:10085000072808D8054B03EB4013B3F83804B0FA67
:1008600080F0400970470020704700BF040000205E
:10087000054B93F8F825824204D903EB4013D3F8D3
:100880004404704700207047040000200346012202
:1008900000205A77704700BF826908B50346006B95
:1008A000D96A02449A6101B18847002008BD00BF9F
:1008B000436A02461B681B6A5B685B7813F00100A1
:1008C00008BF5077704700BFC2628161704700BFA8
:1008D000704700BF043070470C4B93F8FC22D3F8EC
:1008E000F81202440144D2B2C3F8F81283F8FC2291
:1008F00093F8FC22120605D593F8FC2282F08002C0
:1009000083F8FC22024B01225A707047801A00249F
:10091000000000242DE9F84F164FD7F80053ED0AD8
:1009200023D00026DFF850A007F54179B0467419AE
:10093000D7F804134FF01003524648BF0134D1F8E2
:1009400028B04846C7F830836410E102D8470F2822
:100950000BDD094B03F1100153F8042B013207D1D1
:100960008B42F9D12546B542E1DCE802BDE8F88FBB
:10097000661CF8E7801A002440D40024194BD3F8F1
:100980003813D3F83C238A1A322A05DCD3F85023D3
:100990008A1A002A11DC7047D3F8401349B193F842
:1009A0004C23888802F001020968120100FA02F261
:1009B0008A610022C3F850237047D3F840236AB1FC
:1009C00010683231928810B44469C3F8501322423F
:1009D0005DF8044B18BF1204826170473231C3F8CE
:1009E00050137047801A0024074AD2F840334BB1A5
:1009F00092F84C239988186802F001031B0101FA50
:100A000003F3836100207047801A0024044B4FF4E5
:100A1000007C0020D3F86033A2F800C00B60704760
:100A2000801A002400207047012070470120704781
:100A30000020704710B5044651F0E6FB0146204601
:100A400089B2BDE81040FFF76FBB00BF38B50B4D52
:100A500000EB400005F5A763C40003EBC003254489
:100A600093ED027AD3ED037AE7EE007AB0EE670AEF
:100A700051F0CAFBD5F83835186038BD04000020A5
:100A800002692DE9F843C36812EA030828D0054635
:100A90000E464FF00047B8FA88F327FA03F21B3BE3
:100AA000D24308EA02082A61042B16D8DFE803F0D3
:100AB0003B30251A0300B36A002B3FD003F1FF3906
:100AC00000231FFA89F9B362746A34B1236820469F
:100AD000494698476468002CF8D1B8F1000FDAD184
:100AE000BDE8F88370680028F7D0696B036889B2A5
:100AF0009847B8F1000FCED1F2E7B0680028ECD0EB
:100B0000A96B036889B29847B8F1000FC3D1E7E732
:100B1000F0680028E1D0E96B036889B29847B8F122
:100B2000000FB8D1DCE730690028D6D0296C036803
:100B300089B29847B8F1000FADD1D1E7EB6A1FFA3F
:100B400083F9C1E78069B43041F0F4B9F8B5A0F594
:100B500007642379DB0725D5657994F8543805F0C7
:100B600001073D46FBB1D4F848341A68D36A5B08E4
:100B7000536294F8583823B1B4F862380133A4F8BA
:100B8000623885F00101606C48F0ECFB012384F8C9
:100B90005738002384F8553884F85638A4F85E385E
:100BA00084F85438F8BD94F85768012E03D194F8AE
:100BB000553884F856382046FFF74CFB4EB90123D0
:100BC00085EA030184F85738606CBDE8F84048F0C6
:100BD000C9BB0023394684F85738F5E738B542F0E9
:100BE0008DFE0D490D4CD1F8FC20A4FB00400C4DAE
:100BF00042F080720B4B800CC1F8FC204FF0604239
:100C00000949C5F8E003C2F8B01F00225A601A680B
:100C100042F001021A6038BD00ED00E083DE1B43A4
:100C2000801A0024001000E055CEACC570B5054612
:100C30000A26084C013E00D170BD94F900001AF05C
:100C40006BFE031E04DB6178EA185172A278EA5445
:100C50000434EFE7B333090838B590F82830044678
:100C6000012B06D0407F08B9012038BD00236377EF
:100C700038BD406A03681A7B9AB9637F002BF3D0B2
:100C80000A4D022305F1200205F140013CF004FC6D
:100C900095F82130D84303F0010300F00100637799
:100CA000E6E71B6A002BE8D0002038BD40D40024C2
:100CB00038B5044694F82830012B07D0637F0BB178
:100CC00000236377012038BD1B6A23B1606A036883
:100CD0001A7B002AF8D1637F002BF3D0074D022343
:100CE00005F1200205F140013CF0D6FB95F82130DA
:100CF00003F00102DB076277E4D5DBE740D4002490
:100D0000F0B5002395B0224E0446069302200B93C3
:100D100006F18002109313931193009206F1A00242
:100D2000277F1C4D0192626A04950D460290CDE921
:100D30000E3301238DF80C3007938DF820308DF899
:100D400034308DF8483006F1C0030593124B0993F7
:100D500006F160030A933B1D10680C934EF040FAB5
:100D60009FB12A0E06F1620386F861202A0A9D705F
:100D7000280C69465A701870606A3CF0D3FB636AAD
:100D800018684EF02DFA15B0F0BD06F16103EDE7DD
:100D900040D40024B10804088D08040810B594B0AC
:100DA000044650220649684651F006FF6946606ACB
:100DB0003CF0B8FB636A18684EF012FA14B010BD2C
:100DC000D83309082DE9F8431F46436A044688468C
:100DD000186891464EF004FA237FA069002B3BD09F
:100DE000254E020E052386F8E120E236234D012F21
:100DF000B0706B634FEA10434FEA1020337070708D
:100E00004FF00000D8F800302B64D9F80030AB6404
:100E10002363A86523D0022F1CD1D9F804202865AC
:100E20001344D8F8041085F84C00EA65012269657E
:100E30002363134B85F860206B66124B627FA3F12E
:100E40001401606A002A08BF19463CF06BFBE36A94
:100E500063B1206BBDE8F88304230B4EC6E7084B53
:100E600085F84C706865E8652B65E6E7636A186885
:100E70004EF0B6F9EDE700BF40D400240000002496
:100E8000990804081800002421D5002400B583B077
:100E90008161019201A9049A00930123C2626A460A
:100EA000FFF790FF03B05DF804FB00BF2DE9F843A6
:100EB000DDF820800F4616460021202204461D46FC
:100EC00051F0D8FEB8F1000F0CD0D8F80030B8F8C7
:100ED0000A20E3811B0C2382D8F804306282E3826B
:100EE0001B0C238338464FF093FEF30619D4431EA0
:100EF000B8B107EB000C01E0013B12D31CF801ED87
:100F0000BEF12E0FF8D1C01A03F10109421EB944F7
:100F1000032AA8BF0322082BA8BF082390461A461D
:100F200006E008280246B9464FF00008A8BF08228C
:100F30004FF02033394620462360636051F03CFE79
:100F4000164B04F10800424649462381837051F054
:100F500033FE611EE21D11F801CFACF16103ACF16B
:100F6000200C192B98BF81F800C09142F3D104F1F5
:100F70000A0011F8013FA3F16102203B192A98BF32
:100F80000B708142F5D1182365832D0CE672237313
:100F9000099BA582E361BDE8F88300BF2020200003
:100FA0002DE9F04FDFF8509485B0D9F83803C9F82F
:100FB0003C03002B5ED00C46154601F5FE7603EB94
:100FC000020B1DE0002D62D0D9F86C33AB4200F06B
:100FD000C580D9F86833AB4200F0F780D9E9DC313D
:100FE000AB424BD88D42C0F07281691A204647F05F
:100FF000DBFB013504F5007406F500765D4539D05C
:10100000D9F87823AA42DDD8AA1AD9F88873D30868
:10101000396B02F0070802338B4202D3BA6B93425A
:101020000BD939461846039347F08EFB039B0746BE
:10103000002800F06C81C9F888033A79002A40F052
:101040001D81D7F828A0BAF1000F00F059813A6B42
:10105000013520464FF400719B1AFA6804F50074BC
:1010600006F5007608EBC3083B4602EB4822D04762
:101070005D45C5D1002005B0BDE8F08F8D42B4D2EA
:101080004FF400720021204651F0F4FDB1E74FF417
:1010900000722946204651F0EDFD8023CA4A84F8AB
:1010A000BE310C2384F8C231D9F86813D9F8603303
:1010B0009142C4F8C611C4F8CA3100F30D81C34A85
:1010C000013BC34F82FB0102C81787FB01C70A44DB
:1010D000C0EB6212C0EB2730BE4F87FB02C7C2EBEA
:1010E000821C84F8C1018010A1EB0C01174420F090
:1010F0003F0001310843D117C1EBE71184F8C0016B
:101100000A4484F8BF21B04A934200F3F180AF4A09
:10111000AF4882FB0312D91780FB03701A44C1EB5E
:101120006212C1EB2031AB4880FB0270C2EB821728
:1011300084F8C5118910DB1B104421F03F010133F5
:101140001943D317C3EBE01384F8C4111A4484F88D
:10115000C3214AF65523A4F8FE314AE74FF0FF3386
:1011600000274FF4F072201D84F8EC31394684F8E2
:10117000ED3184F8EE3184F8EF315223237063703F
:101180006123A37084F8E7314123E37084F8E631EA
:10119000722384F8E43184F8E531D9F88033C4F857
:1011A000E83151F067FD5523C4F8F07184F8FE3141
:1011B0006FF05503C4F8F471C4F8F87184F8FC7149
:1011C00084F8FD7184F8FF3113E74FF400720021B9
:1011D000204651F04FFD804B022203CB45F6EB0336
:1011E0002274227323809023A273A370F82384F8BF
:1011F0002C200822C4F803006273C4F8071063753A
:10120000D9F86813D9F860335B1A2362D9E9DC1383
:101210005B1A4AF6552163620023E372E373637736
:10122000A377E37784F82D3084F82E3084F82F30BC
:1012300084F83130694BA3613E232377012384F87E
:101240003030802384F84030654BC4F84230654B21
:1012500084F84620A4F8FE11634A03CBC4F84B106F
:101260001988C4F847009B78A4F84F1084F85130CF
:1012700003CAC4F85200C4F85610BAE64FF400721C
:101280000021204651F0F6FC3B6CB8F1000F45D12F
:1012900004F1200A002B00F081803B6B112253499E
:1012A0002046CDE90088FFF701FE3B6C1A6C002A4E
:1012B00000F081801B6B504611224D49CDE900881A
:1012C000FFF7F4FD04F1400A4FF4E07871E0E91A09
:1012D000204647F069FA8CE6FF22013B84F8C121E1
:1012E0004FF6FF72A4F8BF21374A93427FF70FAF42
:1012F000FF2384F8C5314FF6FF73A4F8C33128E704
:1013000051464FF40072204651F0B4FC71E6231FA1
:10131000384A43F8042F9E42FBD16AE6002B7F6CCB
:1013200014BF02230123C3EB0813002F3FF461AE67
:10133000013BBF6C002B01DD002FF9D1A2464FF419
:101340000078002F3FF455AE0AEB080303959A4648
:101350000BE00025A8F12008CDE900E5FFF7A6FD88
:10136000BF6CCFB1B8F11F0F16D93D7907F11C0E34
:10137000112239683B6BAAEB0800002DE9D17A797C
:10138000A8F120083D6942F02102CDE900E5FFF710
:101390008DFDBF6C002FE5D1039D2AE6CDE90088C5
:1013A00043464FF4F0780822D9F864132046FFF73B
:1013B0007DFD7F6CC5E75046434611220C49CDE9BF
:1013C0000088FFF773FD7DE7FF03FB0083200882A1
:1013D000975545418180808058B009083F00FF0043
:1013E00029940E0D64B0090870B0090850B00908BE
:1013F00054B00908DEADBEEF801A002430B40D4CA5
:10140000BFF34F8F0C4BC3F85C42BFF34F8FBFF35A
:101410006F8F0A4B0A4D03F13000DA792AB15979FE
:1014200034F8112092B225F811200C338342F4D104
:1014300030BC704780D7002400ED00E0641E00241B
:10144000E0D6002400207047704700BF014841F0FB
:101450005FBF00BFD01E0024084810B4D0F850343D
:10146000D0F8844499691A682CB1234600F58A6043
:101470005DF8044B18475DF8044B7047801A002450
:10148000014841F045BF00BF341F0024084810B494
:10149000D0F8B434D0F8E84499691A682CB12346DE
:1014A00000F2B4405DF8044B18475DF8044B7047F8
:1014B000801A0024014841F02BBF00BF981F002470
:1014C000084810B4D0F81835D0F84C4599691A6816
:1014D0002CB1234600F5A3605DF8044B18475DF876
:1014E000044B7047801A0024014841F011BF00BF2F
:1014F000FC1F0024084810B4D0F87C35D0F8B04563
:1015000099691A682CB1234600F27C505DF8044BAF
:1015100018475DF8044B7047801A00242DE9F0410C
:101520000468D4E90435A8611A7D1F681F2A49D9C7
:10153000203A20212E6801FA02F242F01802FA60E5
:101540002A7D1F2A48D9203A202101FA02F242F0CE
:101550001802F2606A68002158680160384611601C
:10156000116841F01001116093F80880A2694146AA
:101570004CF00EFA2D7AE269304629464CF008FA12
:10158000226A63689468184A12F80800515D5A6824
:101590006FF30F0222435A603A5842F001023A5068
:1015A000725842F0010272509A6842F440429A60C6
:1015B0001A6842F001021A601A6842F400721A6056
:1015C000BDE8F08120212E6801FA02F242F01802F3
:1015D000BA602A7D1F2AB6D8202101FA02F242F011
:1015E0001802B260B6E700BF20B10908D3B20F2BD2
:1015F00021D8124B00B503F17E0E02E00333734590
:1016000016D093F800C08445F8D193F801C08C45FA
:10161000F4D102EB42020A48997800EB82037C3055
:10162000C3F8841000EB820083F87C105DF804FBA3
:1016300000205DF804FB0020704700BF2834090833
:101640000000002410B40C4C002304F5B96C01E038
:10165000152B0CD003EB430201331CF8021081421E
:10166000F6D1144494F9CA055DF8044B70474FF065
:10167000FF305DF8044B7047801A002430B5124DDE
:10168000002305F5A47C02E001331A2B1AD05CF884
:1016900033408442F8D10CEBC30EDC009EF804E02A
:1016A0008E45F1D102EB4202084B254403EB820147
:1016B0007C3395F84D4103EB8200C1F8844081F8FA
:1016C0007C4030BD002030BD60330908000000249C
:1016D000F0B1002310B504460E4894F804E000F57C
:1016E000B96C01E0152B11D003EB430201331CF858
:1016F00002107145F6D183186179206893F9CA25E3
:10170000D3B20F2B02D8BDE81040B7E7002010BDC0
:1017100000207047801A002401380E4B0E4A00EB5F
:10172000C000D2F8D81003EB800310B4D3F83C31DA
:1017300083B00A4CA34214BF022301231943C2F809
:10174000D810D2F8D82013400193019B03B05DF864
:10175000044B70470000002400440258000002407F
:101760000138F8B500EBC000124C1D46124B04EBDB
:10177000800417460E46D4F83C01984214BFA120BD
:10178000A02049F065F8B4F95201B909C4F84C61D8
:10179000C4F8545148F0CAFCB4F95231002B07DBAD
:1017A00003F01F0001225B090449824041F8232015
:1017B000F8BD00BF000000240000024000E100E08E
:1017C000800AA0F58010522806D8044B1B5C0D2B14
:1017D00002D8034AD056704700207047603309088A
:1017E00010B109084FF0B042D2F88030D2F888101A
:1017F0000B4003F00103C2F8883023B1024BD3F849
:101800000806036818477047801A00244FF0B0425A
:10181000D2F88030D2F888100B4003F00203C2F8EF
:10182000883023B1024BD3F80C0603681847704781
:10183000801A00244FF0B042D2F88030D2F88810DD
:101840000B4003F00403C2F8883023B1024BD3F8F5
:101850001006036818477047801A00244FF0B04202
:10186000D2F88030D2F888100B4003F00803C2F899
:10187000883023B1024BD3F8140603681847704729
:10188000801A00244FF0B042D2F88030D2F888108D
:101890000B4003F01003C2F8883023B1024BD3F899
:1018A0001806036818477047801A0024F8B54FF0EF
:1018B000B043D3F88050D3F88820154005F47875EC
:1018C000C3F888507DB1084F0126B5FA85F4C4F1FC
:1018D0001F0407EB840306FA04F4D3F80806036830
:1018E0009847A543F1D1F8BD801A0024F8B54FF010
:1018F000B043D3F88050D3F88820154005F47C45D8
:10190000C3F888507DB1084F0126B5FA85F4C4F1BB
:101910001F0407EB840306FA04F4D3F808060368EF
:101920009847A543F1D1F8BD801A002430B103686F
:1019300082881B691A4214BF01200020704700BF33
:1019400010B1036882889A61704700BF18B183881C
:1019500002681B049361704770B50D4682B004465F
:10196000164640B101680C4B0C4A0B449B0A02EB33
:101970004303B3F8180248F06BFFC5F38101C5F3C8
:10198000411305F01302CDE90016A18820684CF040
:1019900061FF02B070BD00BF0000FEA76033090800
:1019A00000B1D9E770472DE9F84FC44F64230446CE
:1019B00003FB0073D3F83864002E00F06981D3F87C
:1019C0004084B8F1000F04D098F90630002B40F0A5
:1019D0005F81642303FB0473D3F8445425B195F964
:1019E0000630002B40F05481631CDBB2B8F1000FCD
:1019F00004D0152288F8073088F8062015B1162281
:101A0000EB71AA714FF0640A308D48F021FF29462E
:101A10000AFB04FA40464EF0FBFA404607EB0A097F
:101A2000DFF8BC8299F84A3499F84824002B0CBF9F
:101A30004FF01E0B4FF03E0B5946FFF7B1FF284603
:101A40009F4D594699F849245544FFF7A9FF4C2268
:101A50000021284651F00EF9D9F83834994A5B68CC
:101A60009342C9F85034DFF87C9240F0138141F082
:101A700067FFD9F82030C3F30213434493F82C32A4
:101A800003F01F039FED907A9FED905AB0EE084A45
:101A9000D8406423F7EE003A4FF0000C07EE900AAE
:101AA00003FB047340F21458F8EE677AB3F84CA4C1
:101AB000C7EE275A07EE90AA9FED857AF8EEE77AEF
:101AC000C7EE274ADFED837AB0EE007AE5EE877A3B
:101AD000A5EE875A25EE844A37EE856A74EEE72A2A
:101AE000BAF5C87F0CF1010ED5BF4FF4967278227B
:101AF0006423322307EE90EAD8BF4FF416791344DB
:101B0000A2F13202F8EEE76AC8BF4FF4827907EE1D
:101B1000903AD4BF41464FF4FA7166EEA56AB8EE2A
:101B2000E77AC7EE267A07EE102A01EB0902B8EE33
:101B3000C77A37EE447A77EEE37AFCEEE77A17EE6F
:101B4000903AC7EE267AFCEEE77A17EE900A07EE97
:101B5000909AB8EEE73A07EE902AF8EEE77A23EE8D
:101B6000243A83EE277A37EE453A32EEC77AC3EE4F
:101B7000267A77EEE37AFCEEE77A17EE901AC7EE54
:101B8000267A77EEE37AFCEEE77A17EE902A02F1F6
:101B9000020909EB010BB0EE467A07EE90BAF8EEB7
:101BA000677AA6EEA77AF4EEC74AF1EE10FA7DDC6A
:101BB00043EA00095FFA89F9B9F10F0F78D841EAD1
:101BC00002091FFA89F9B9F1FF0F71D81B0500044A
:101BD00003F07F6392B200F47F0003433E4843EA80
:101BE0000C7300EA01210B4313436422284602FBD5
:101BF00004740027C4F854340123C4F85874C4F89A
:101C00005C34C4F86074C4F86474C4F86C74C4F8C8
:101C100070744CF0D1FD94F89134202BD9B21AD1C4
:101C200094F89034012B16D0242384F89134D4F8FE
:101C300050341A6822F001021A601A6822F48052A5
:101C40001A601A681A601A6842F001021A6084F871
:101C5000911484F89074002196F82B0048F066FAED
:101C600096F82B3001241D4D5A0903F01F03002163
:101C700004FA03F345F8223096F82A0048F056FAA1
:101C800096F82A305A0903F01F039C4045F8224079
:101C9000BDE8F88F41F054FED9F81C30C3F30213AD
:101CA000984498F82C32EBE6F44619E7013170E7D6
:101CB000BEF10F0FF8D1002397E700BF801A002470
:101CC000D01E0024001C0058286B6E4E00001643E6
:101CD000002474490000704200FFFF0000E100E0B2
:101CE000603309080044025808B1002234E6704706
:101CF00070B50E4C94F8F865AEB104F58764002514
:101D000003E001352034B5420DD0237F002BF8D0FD
:101D1000E06800220028F4D00135217DFFF71CFE89
:101D20002034B542F1D1012070BD00BF0400002075
:101D300070B590F8EE311C09013C082C0FD81A4EF2
:101D4000054603F00F0306EB4402B2F83C0240FAEA
:101D500003F2D20703D595F8F121012A01D0012021
:101D600070BD9A402644013A104051F033F996F87C
:101D700050320E4A034402EBC30452F83320A388C6
:101D800010691840ECD0002395F8EF21022120467D
:101D900085F8F131FFF7E0FDD5F85021136843F0E5
:101DA00008031360DBE700BF60330908C820002484
:101DB00038B5BFF34F8F6A4A6A49A2F58653C1F816
:101DC000683220339342FAD1BFF34F8FBFF36F8F46
:101DD000654C94F8CD23B4F8DC33022A11D094F882
:101DE000CD23012A00F08D80D4F890530C2B0CD811
:101DF000DFE803F0110B0B0B300B0B0B4D0B0B0B38
:101E00006A00002384F8DE3338BD00236B620123AF
:101E100084F8CD3338BDD4F8B403544B544AC3646A
:101E200090F83430C263012B00F09780012290F8C3
:101E30003530934280F8342000F0858000234FF441
:101E4000006280F8343042656B62EB6843F40073E3
:101E5000EB60DCE7D4F8B803444B454AC36490F820
:101E60003430C263012B61D0012290F835309342A7
:101E700080F8342053D000234FF4006280F83430CF
:101E800042656B62EB6843F48063EB60BFE7D4F8B4
:101E9000BC03364B364AC36490F83430C263012B1E
:101EA0004ED0012290F83530934280F8342040D053
:101EB00000234FF4006280F8343042656B62EB68B7
:101EC00043F40063EB60A2E7D4F8C003274B284A31
:101ED000C36490F83430C263012B1DD0012290F806
:101EE0003530934280F834200FD000234FF4006245
:101EF00080F8343042656B62EB6843F48053EB60EA
:101F000085E7022284F8CD236EE740F22A4305F1EB
:101F10004002184940F0FAFC00236B62ECE740F203
:101F20002A4305F13802134940F0F0FC00236B62AC
:101F3000A8E740F22A4305F13C020E4940F0E6FCD6
:101F400000236B62BBE740F22A4305F134020949E2
:101F500040F0DCFC00236B6277E700236B6274E7E0
:101F60002032012400ED00E0801A002499F60708D1
:101F7000F1F6070860210124014B53F82000704757
:101F800050400058014B43F8201070475040005813
:101F900019481A4B01681A4A41F4807130B482B072
:101FA0000160D3F8F410FF24CA2041F48031C3F853
:101FB000F410D3F8F41001F4803101915321019D04
:101FC000546250625162D3F8D030DB010CD40C4B18
:101FD00000220C495A659A65DA651A665A669A664D
:101FE000196502B030BC7047126D064B9A42EED1B3
:101FF00002B030BC704700BF00480258004402588D
:1020000000400058316665422DE9F84FD0F85C7108
:102010000446534B00F59676FDB227F0FF0982681F
:1020200000F1E00A103D4846D2F80080A3FB0535D8
:102030002D0929464BF008FDD4F81C210023B2F5E8
:10204000807F84F820317FD00DD8102A00F0848062
:102050005DD8012A46D0042A16BF6FF400616FF0E4
:1020600008013C230EE0B2F5805F71D0B2F5803FED
:102070003BD0B2F5806F15BF6FF400616FF00801BF
:102080003C230423324608F11806404656F803C0A4
:1020900001EA0C01F150D4F81CB159464BF082F919
:1020A000BBF5807F2ED024D8BBF1100F3FD037D89E
:1020B000BBF1010F02D0BBF1040F34D14FF0080C7B
:1020C000336852462946484643EA0C0333604023AE
:1020D000C4F8E8304BF05CFC3B6843F010033B6015
:1020E000BDE8F88F6FF00801CCE76FF008013C23E2
:1020F000C8E7BBF5805F22D0BBF5803F1AD0BBF5A7
:10210000806F10D108F11C064FF0080CD8E7402A68
:1021100015BF6FF400616FF008013C230023B1E7A5
:10212000BBF1400FCAD03C364FF4006CC8E74FF407
:10213000006CC5E708F154064FF0080CC0E708F141
:102140001C064FF4006CBBE76FF00801042399E70D
:102150006FF40061042395E76FF4006192E700BF1C
:10216000ABAAAAAAD0F8E8312DE9F04F93F83230A3
:1021700085B0DFF878B304464FEA531A03F01F0323
:1021800006795BF82A200BEB8A0916F0020622FA80
:1021900003F202F00102029204D090F8EE61003ED8
:1021A00018BF012601279F40C9F88070BFF34F8FE9
:1021B000BFF36F8FD4F8DC311A6822F4F8721A601A
:1021C0009A6822F001029A60C9F88071BFF34F8FBC
:1021D000BFF36F8F2423D4F85051A168C4F8D031D5
:1021E00000232A6822F001022A6004F5A8722B60FD
:1021F0006B60AB60C4F8D83184F8CC31C4F8D0310E
:10220000C4F87031C4F8D4310192C4F85411B34900
:10221000C4E9593363798D424FEA832202F4805234
:10222000C4F858214FEA033202F40052C4F85C218A
:102230004FEA032202F48062C4F8602100F0BC81FE
:10224000227903F00101D00700F1588116B108206E
:10225000C4F86401002940F0628194F8F0214AB189
:10226000D4F8782142F00802C4F878214FF40042F3
:10227000C4F8882113F0080FD4F8D0314FF02403AC
:102280000198C4F8D0312B6823F001032B6000F0D3
:10229000838141F0E9FE012817D0D4F87831002B72
:1022A00040F08E816B6823F490436B60AB6823F041
:1022B0002203AB60AB6843F00803AB602B68019866
:1022C00043F001032B604BF081FC2379DB0775D5CC
:1022D000D4F82C81B8F1000F00F04B8100234FF4AB
:1022E000807CC4F83C802366E366C4E91133C4E90A
:1022F0001433C4E91933D4F83431C4F8B8304FF486
:102300008063E3644FF48033C4E916C304F13C03F3
:10231000184603934CF034FE039840F057F9039BA2
:10232000C4F8C831019B6367D4F8D431202B41D164
:10233000E368626998B2EAB3B0FA80F14909C8B3B8
:1023400094F8CCC1BCF1010F34D04FF0220CC4F88A
:10235000D811A4F8AC010120C4F8D4C1DFF890C1B1
:10236000C4F8A821C4F878C0DFF888C1C4F88C107C
:10237000C4F87CC0DFF880C184F8CC01C4F888C000
:1023800094F870C084450CD084F8700094F8710003
:10239000012800F01D814FF4006384F87010C4F828
:1023A00090301023C4F8D831002384F8CC31202396
:1023B000C4F8D031D8F80430C4F84431002E00F00D
:1023C0008780D4F83061002E00F0BF80002304F134
:1023D000B405C4F8B460C4F8C0302846C4F8D0309E
:1023E000C4E93233C4E93633C4E93833D4F8383178
:1023F000C4F8B8304023C4F8BC304FF48063C4F84C
:10240000C4304FF48033C4F8D4304CF0B9FD2846C2
:1024100040F0DCF8002840F09080019B304AC4F87E
:10242000EC30304BC4F8C451964218BF9E4202F1C2
:1024300018020CBF01230023964208BF43F001039A
:102440001832964208BF43F001031832964208BF83
:1024500043F001031832964208BF43F001031832DB
:10246000964208BF43F001031832964208BF43F07A
:10247000010302F55672964208BF43F00103183279
:10248000964208BF43F001031832964208BF43F05A
:1024900001031832964208BF43F0010318329642F6
:1024A00008BF43F001031832964208BF43F001030E
:1024B0001832964208BF43F001033BB90A4BF31AA6
:1024C000B3FA83F35B09002B00F09A80002373605A
:1024D000029B002B46D105B0BDE8F08F000C0058E0
:1024E0002800024010000240B804024000E100E071
:1024F00079F70708ADF70708B1F707080420C4F813
:102500006401DEB900293FF4A8AED4F8781141F097
:102510000201C4F878114FF48031C4F88011920799
:102520007FF59BAED4F8782142F00102C4F87821FF
:102530004FF40032C4F87C218FE6FEE70C20C4F88B
:10254000640100293FF489AEDFE7D4F8DC311A6872
:1025500042F080021A601A6842F040021A60029B40
:10256000002BB8D0C9F880714BF82A7005B0BDE8CF
:10257000F08FD4F8DC311A6842F480721A609A68DD
:1025800042F001029A601A6842F020021A601A684A
:1025900042F010021A6011E741F066FD01283FF495
:1025A00094AED4F878317BB96B6823F490436B60B8
:1025B000AB6823F02A0380E60422C4F874213FE6C6
:1025C000019841F04FFF6DE6019841F04BFFEBE7BA
:1025D0009BB2039805F1240140F098F900287FF49C
:1025E000E0AE84F8CC012B6843F480732B60AB68B9
:1025F00043F00103AB60AB6843F04003AB60D9E646
:10260000736065E738B50409013C082C1AD80F4DF2
:1026100000F00F0305EB4402B2F83C0240FA03F26B
:1026200012F0010210D00122254402FA03F3013B0B
:10263000184050F0CFFC95F85032054A034402EBA5
:10264000C30038BD002038BD104638BD60330908CE
:10265000C82000242DE9F047984D05EB0013D3F86E
:10266000C84A002C00F08F80B3F8D27A06464FEAB1
:102670000019384648F0ECF801227B0907F01F07E3
:10268000023BBA40082B0FD8DFE813F0BF00C700A9
:10269000CF00D700DF000900E700EF00B70088494E
:1026A000CB6F23EA0203CB6705EB0903013693F8EE
:1026B000CC0AF6B2FFF7A6FF074610B11223C67187
:1026C000837105EB090393F8CD0AFFF79BFF824660
:1026D00010B11323C671837105EB090393F8CE0A79
:1026E000FFF790FF804610B11423C67183714D44EB
:1026F00050462E2195F8D02AFFF752F995F8D12AA5
:1027000040460E21FFF74CF995F8CF2A2E21384686
:10271000FFF746F923686B4A23F0010394422360D4
:1027200033D0694B9C423ED1654BD3F8902042F4A4
:102730008042C3F89020D3F8902022F48042C3F85E
:102740009020E36843F00043E360A36823F4F07350
:10275000A3602368DA0716D4A1685C4A5C4B0A4080
:102760001343A360E368DB0042D5E268594B134092
:1027700043F0E863E360236823F400632360236D80
:1027800023F001032365BDE8F0874D4BD3F8982073
:1027900042F48052C3F89820D3F8982022F4805253
:1027A000C3F89820CDE74C4B9C4213D04B4B9C4236
:1027B00063D04B4B9C426ED1414BD3F8982042F4EE
:1027C0008012C3F89820D3F8982022F48012C3F81E
:1027D0009820B6E73A4BD3F8902042F40042C3F871
:1027E0009020D3F8902022F40042C3F89020A8E76C
:1027F000236843F480532360B7E73149D1F89C3014
:1028000023EA0203C1F89C304EE72D49D1F89830F5
:1028100023EA0203C1F8983046E72949D1F89030FD
:1028200023EA0203C1F890303EE72549D1F89430FD
:1028300023EA0203C1F8943036E72149D1F8803009
:1028400023EA0203C1F880302EE71D49D1F8843015
:1028500023EA0203C1F8843026E71949D1F88C3005
:1028600023EA0203C1F88C301EE71549D1F88830FD
:1028700023EA0203C1F8883016E7114BD3F89820F9
:1028800042F40052C3F89820D3F8982022F4005262
:10289000C3F8982055E7134B9C427FF452AF03F5E1
:1028A0000C33D3F89C2042F02002C3F89C20D3F8CC
:1028B0009C2022F02002C3F89C2042E7801A0024CA
:1028C000004402580030014000380040E0FFBF8F54
:1028D00007000020FFFF39D8003C004000340140D1
:1028E000005001400014005808B51D20FFF78AFE73
:1028F00010B190F9063053B11E20FFF783FE10B1DE
:1029000090F9063003B108BD5523C38008BD552397
:10291000C380F1E7F8B50E4C94F8F875A7B104F54B
:10292000C064C7F109070925013D0FD0A6683079B9
:10293000FFF768FE94F8DC10F27908B1FFF70CF8A5
:10294000AF4204F5B474EFD10120F8BDAB68FFDEEF
:1029500004000020F8B50446EFF31185502383F3FB
:10296000128803799B0702D590F8EE3133B9012321
:1029700084F8E031EDB285F31188F8BDD0F830313C
:102980001B6803F00103002BF4D1D0F8D021D0F85C
:10299000D4110A4302F02102212AEBD0D0E9091216
:1029A0009142E4D090B24BD8194623691B1A9BB2CE
:1029B000A162002184F8E011D4F8D0112029D9D1E6
:1029C000A1698918D6D0B3FA83F25209002BD1D06D
:1029D00094F8CC010128CDD02120A4F8A6314FF0E5
:1029E000010CC4F8D821C4F8D001D4F8C401D4F83B
:1029F0005061C4F8A011A4F8A43184F8CCC140B34C
:102A0000194F90F834E0C763184FE6450265076434
:102A1000174FC7640AD090F8357080F834C0674506
:102A200011D04FF4006380F8342043651021002258
:102A30002023C4F8D81184F8CC21C4F8D03199E708
:102A4000081A83B2B4E706F128023FF05FFF0028BE
:102A5000ECD100234022326284F8CC31B36843F0D9
:102A60008003B36086E700BF51F7070875F70708D2
:102A7000B1F70708BFF34F8F0549064BCA6802F448
:102A8000E0621343CB60BFF34F8F00BFFDE700BF91
:102A900000ED00E00400FA0519484FF6FF0C194A52
:102AA00084B0C168184B01EA0C010A43C260D3F834
:102AB000D020D3F8DC2042F00052C3F8DC20D3F859
:102AC000DC2002F000520192019AD3F8DC2042F09F
:102AD0008042C3F8DC20D3F8DC2002F0804202926E
:102AE000029AD3F8DC2042F00042C3F8DC20D3F88D
:102AF000DC3003F000430393039B04B0FEF76EB891
:102B000000ED00E00005FA050044025808B51D4834
:102B10000023C0F88430BFF34F8F436923F4803320
:102B20004361BFF34F8FD0F8803043F6E074C3F3B6
:102B30004E3CC3F3C90E4FEA4C1C0CEA0401734629
:102B400041EA8372013BC0F874225A1CF8D1ACF1FF
:102B5000200C1CF1200FF0D1BFF34F8FBFF36F8F0C
:102B6000BFF34F8FBFF36F8F4369002223F400330D
:102B70004361C0F85022BFF34F8FBFF36F8F72B61F
:102B8000FFF778FF00ED00E003689B0AA3F58013D0
:102B9000522B00D970470E4AD35C0D2BFAD84FF058
:102BA0004C0C10B40B4C42790CFB03400223D0F8C0
:102BB000280BDA409340C26829B922EA03035DF882
:102BC000044BC360704713435DF8044BC360704708
:102BD00060330908801A002403689B0AA3F5801358
:102BE000522B10D8084AD25C0D2A0CD84079022307
:102BF00006494FF04C0CD8400CFB02128340D2F82F
:102C0000282BDB431361704760330908801A0024C6
:102C100001490248FDF734BFE41A002400000140D6
:102C200001490248FDF72CBFE41A002400000140CE
:102C300002494FF08040FDF723BF00BF101B002466
:102C400001490248FDF71CBF3C1B00240004004062
:102C500001490248FDF714BF681B0024000800402A
:102C600001490248FDF70CBF941B0024000C0040F2
:102C7000F8B5164D164E2A69EB681A404FF0004021
:102C8000B2FA82F3EAB120FA03F3012A6FEA0303EE
:102C900002EA03012B610A46F2D1D6F868718FB1BE
:102CA000013F0023BFB2C6F86831D6F8644134B1A1
:102CB00023682046394698476468002CF8D10022E2
:102CC000DCE7F8BDEF6ABFB2EFE700BF00100040DD
:102CD000801A002401490248FDF7D2BE181C0024C6
:102CE0000004014010B5064C064804F5CC71FDF710
:102CF000C7FE04F5F8710448BDE81040FDF7C0BEFA
:102D0000801A002400040140001C004001490248D0
:102D1000FDF7B6BE441C00240018004001490248DB
:102D2000FDF7AEBE9C1C0024002000400149024873
:102D3000FDF7A6BEC81C002400400140014902481E
:102D4000FDF79EBEF41C00240044014001490248E6
:102D5000FDF796BE201D0024004801402DE9F041FA
:102D60004FF425728EB0002173484FF083FF734BF0
:102D7000734D4FF00008D3F8F02040F27D27A5F501
:102D80001F7605F6F41442F00102C3F8F020D3F8E0
:102D9000F02002F001020092009AD3F8E82042F0FD
:102DA0000102C3F8E820D3F8E82002F00102019202
:102DB000019AD3F8E82042F00202C3F8E820D3F8E1
:102DC000E82002F002020292029AD3F8E82042F0D0
:102DD0000402C3F8E820D3F8E82002F004020392CA
:102DE000039AD3F8E82042F00802C3F8E820D3F8A9
:102DF000E82002F008020492049AD3F8E82042F096
:102E00001002C3F8E820D3F8E82002F0100205927F
:102E1000059AD3F8E82042F02002C3F8E820D3F85E
:102E2000E82002F020020692069AD3F8F02042F041
:102E30000202C3F8F020D3F8F02002F00202079259
:102E4000079AD3F8E82042F04002C3F8E820D3F80C
:102E5000E82002F040020892089AD3F8E82042F0F5
:102E60008002C3F8E820D3F8E82002F0800209923B
:102E7000099AD3F8E82042F48072C3F8E820D3F826
:102E8000E82002F480720A920A9AD3F8F02042F401
:102E90008032C3F8F020D3F8F02002F480320B9295
:102EA0000B9AD3F8F02042F40032C3F8F020D3F8A4
:102EB000F02002F400320C920C9AD3F8F02042F485
:102EC0008022C3F8F020D3F8F03003F480230D9370
:102ED0000D9B55F82810002354F83320914226D03A
:102EE00001330E2BF8D1002008F1070847F0B0FCA1
:102EF000B845EED14FF0000840F27D2755F8281074
:102F0000002354F8332091420CD001330E2BF8D11A
:102F1000002008F1070847F09BFCB845EED10EB041
:102F2000BDE8F08106EBC303B3F8740CF1E706EBE0
:102F3000C303B3F8740CD7E7E41A00240044025822
:102F4000DC350908800AA0F5801052280DD8074BFF
:102F50001A5C0D2A09D8064B4C2101FB0233D3F829
:102F6000282B136843F0010313607047603309088E
:102F7000801A00241F4B984210B50ED003F58063D1
:102F800098420AD01C4A03F58043984218BF9042E9
:102F900003D003F5806398421BD140F0D1FC174B5E
:102FA0001749DC69DA69C4F3022CC2F3022201EB8F
:102FB0000C0393F82C3203F01F03D8400F4B114938
:102FC0001B69C3F3C03342EAC303CB5C03FB00F0CD
:102FD00010BD40F0B5FC094B0949DC69DA69C4F35E
:102FE0000214C2F302120B1993F82C3203F01F03E0
:102FF000D840E3E70000014000400140004402588F
:1030000060330908FCB009082DE9F04F002391B0A6
:10301000AD4C0093AD4BAE4FA3F54E66AB4D4FF0AC
:103020000009AC4BD5F800A093F8AE2F4FEA9A23D5
:10303000A3F58013522B00F2CE80F35C0D2B00F22F
:10304000CA80012A17F903B000F01081022A02D1C8
:10305000BBF1080F3BD14FF00008414658460EF037
:103060001BFE0EF0A1FE90F900C0BCF1000F18BFCE
:10307000BCF1540F14BF4FF0010C4FF0000C40F0A6
:10308000E98008F104081FFA88F8B8F1100FE4D1BC
:10309000009B002B00F0AA808B4A0AE0F35C0D2B0A
:1030A0000ED8FB565B450ED002F58672944200F0B6
:1030B000998091680B689B0AA3F58013522BEDD978
:1030C00000235B45F0D14B7969799942ECD109F144
:1030D00001091C35B9F1080FA3D1009B04F58674D2
:1030E0000133042B009399D17B4A4FF0010B92F8E6
:1030F000F83502F5876901330393039B5B4567D07D
:10310000744B99F81020D9F80C6093F8C23F0092E4
:10311000002E5DD0704AD6F800A055686F48B2887E
:10312000002D504401924FEA902040F3AE80664A51
:10313000002405E0013402F58672AC4200F0A28062
:1031400011688142F6D1604B4FF48672019D02FBFB
:103150000434009B0322C9F80C6089F81030019BED
:10316000C9F81840B3FA83F7C7F11F035800C9F82C
:103170000430B27186F807B002FA00F6A16C0122A1
:10318000D4F854C0314302FA00F002FA03F3A16408
:10319000216D0143D4F8AC0021654F490E7899B2F6
:1031A000002E00F04E8143EA0C036365CAF8185004
:1031B000FCF778FF0BF1010B2046FCF747FF09F104
:1031C000200940F20113BBF1090F29F8043C94D106
:1031D00011B0BDE8F08F013A012A7FF678AF4FF0C9
:1031E000000B38E7BCF1000F7FF471AFA868002234
:1031F0003B4904E001320C31102A00F088834B680F
:103200009842F7D152B269795046FEF737FA354AFB
:103210004068002351680133884208D0102B02F126
:1032200024023FF454AF516801338842F6D1DBB237
:103230002D4A013B03EBC30302EB830393F958319F
:10324000002B7FF444AFC9EBC909204B03EB890382
:10325000A36042E7009B002B7FF41EAF09F1010938
:103260001C35B9F1080F7FF4DCAE36E7BBF1010F76
:103270003FF4F1AE09F101091C35B9F1080F7FF4F3
:10328000D0AE2AE7042C00F049824FF48671124A2E
:1032900001FB052211690491002900F0048390606C
:1032A00001304FF054019C46C4B20D4882F8101111
:1032B00082F811416A1C08494A60049A11689768AB
:1032C00002915179002216E00C00002040400908CC
:1032D00010B10908801A0024040000200000FEA795
:1032E0007C0000243C0100240000002401320C304A
:1032F000102A00F00C8343689F42F7D152B2029823
:10330000CDF814C0FEF7BAF9944B4FF48672DFF88B
:103310007C8202FB05310022059B0132D0E901705D
:10332000C1E9077041464868874208D0102A01F178
:1033300024013FF44DAF486801328742F6D1D2B242
:103340008749013A02EBC20201EB820292F958115D
:1033500000297FF43DAF4FF4867182F859410693FE
:10336000542401FB05F37F4882F858419A107E49A6
:10337000059300FB02F201F560747848C2EBC20CC1
:1033800002EBC202184401EB4C1104EB4212C0F8EC
:103390000CA0C0F8B410C0F8FC203322C0F8B8204C
:1033A0008C22C0F80021714A0298D418FFF7E2FD80
:1033B000069B062B00F0B981072B6D496D4B6E4AB9
:1033C00018BF1A466D4B18BF0B464FF48671DDF8D7
:1033D00008A0B0FBF3F3B0FBF2F2013B5F48013A07
:1033E00001FB05019BB2A1F8BC20A1F87430236653
:1033F000059B03F1580100F10803504619440023CE
:10340000A4F858306366E3654AF04AF9DAF8003008
:1034100043F08003CAF80030049B5B791A46069398
:103420000C2A1CD8DFE812F003021B001B001B0053
:10343000DD011B001B001B00BB011B001B001B0050
:103440009601C7F12F072D0402FA07F3324643EA2B
:103450000C036365CAF81850FCF724FEAAE63F4A3D
:103460004FF4867302984FF0000A03FB05230222F3
:10347000CDF828A059690368079123F00103CDF81E
:1034800034A0CDF83CA00360602308934FF4807310
:103490000E93012309930A23CDE90B3208AA49F0C0
:1034A00081FF0799B1F5807F00F0288240F24081CA
:1034B000B1F5805F00F00E82B1F5803F00F004822C
:1034C000B1F5806F15BF4FF4006308234FF03C0A3D
:1034D0004FF0040A029A183252F80A100B4342F8CD
:1034E0000A30049B1879002840F0CB81029A1368B7
:1034F00043F0010313600023D8F8042001339742FE
:1035000000F0BC81102B08F12408F5D14FF0FF33F7
:103510000027134A03EBC30302EB8303D3F83C01F8
:10352000174B984214BFA120A02047F091F9069AAA
:103530000C2A00F2A081134B03EB4203B3F8C0CD79
:103540004FF48673054A104803FB0523DDF808E0B5
:1035500000F23471A3F818C0002320E0040000201A
:10356000000000246B4CA407601901240C0000200B
:10357000D0DD0600449508001055220040771B005E
:103580000000024060330908FC1000203C010024C8
:10359000964500F09D810133042B00F0BB8151F86A
:1035A0003320002AF4D1D0F854270132C0F8542730
:1035B00000EBC300029ADB00C0F8342719443846F8
:1035C000234690228F884CEA070C0027A1F804C0FC
:1035D000C349FEF7C5F84FF48673C24A40214FF441
:1035E000403CC14803FB052A4FF48052DAF81C50D6
:1035F0002B6843F010032B602B6843F014032B60FF
:10360000C4E91F77C4E92777C4E92977DAF82030BD
:10361000A167E9B2C4F89430069310394FF480637F
:10362000C4F898C0A0FB01014FF4804CC4F884306A
:10363000DAF8B8000909059BC4F8900025F0FF00EE
:10364000DAF80C80C4F8882008F11802049102907E
:1036500008F11008226703F17002A44B1A44DAF84B
:10366000B430C4F88CC063674AF092F9D5F800C052
:10367000059BC4F820C0D5F814C003F1B8029B4BD9
:10368000C4F824C0D5F804C01A44069BC4F828C066
:10369000D5F808C00499C4F82CC0D5F80CC0C4F8FB
:1036A000DC304FF48063C4F8C870C4F8CC304FF4F9
:1036B0000033C4F830C0C4F8E0300298C4E9307771
:1036C000C4E93977C4E93B774FF40067DAF8003191
:1036D000C4F8B880C4F8D0704FF48047C4F8D8302C
:1036E000DAF8FC30C4F8D470C4F8BC304AF050F9B1
:1036F0002B68D6F800A063636B69A3636B68E36310
:10370000AB682364EB6863642B6843F010032B60A1
:103710002B6843F014032B60B5881AE50323744A21
:1037200082F8C33F11B0BDE8F08F724A724B4CE68D
:10373000102900F0E98000F2BD80012900F0E2804C
:10374000042915BF4FF4006308234FF03C0A4FF0E3
:10375000000ABFE602984FF4867262494FF0020AEF
:10376000036802FB05124FF4805123F001035161FD
:1037700008AA036000230A930D930F936023089314
:103780004FF480730E93012309930A23CDE90B3A7A
:1037900049F008FE4FF0040A4FF400639AE60298DD
:1037A0004FF486724F494FF0020C03684FF0040A41
:1037B00002FB05124FF4807123F001035161602276
:1037C000036000230E910A930D930F930123CDE91B
:1037D00008230A2308AACDE90B3C49F0E3FD08239E
:1037E00078E602984FF486723E494FF0000A03686B
:1037F0004FF0020E02FB0512102123F00103CDF859
:1038000028A0516108AA03606023CDF834A0089372
:103810004FF48073CDF83CA00E93012309930A2343
:10382000CDE90B3E49F0BEFD4FF4006352E602982D
:103830004FF486722B494FF0000A03684FF0020ED6
:1038400002FB0512012123F00103CDF828A05161EC
:1038500008AA03606023099108934FF48073CDF8A0
:1038600034A00E930A23CDF83CA0CDE90B3E49F0DD
:1038700099FD08232EE64FF0000C61E6DFB27B1EB7
:1038800047E6FEF7BFFE824638B1049B0221DA7993
:10389000FEF762F85423AAF80630029A536C43F4F8
:1038A0000043536422E60223114A82F8C33F11B059
:1038B000BDE8F08F402915BF4FF4006308234FF097
:1038C0003C0A4FF0000A05E608234FF03C0A01E6E7
:1038D000DB0073E64FF400634FF0040AFAE500BF23
:1038E0000100000004000020ABAAAAAA0C000020DE
:1038F000801A0024882A1100A0BB0D0008234FF075
:10390000040AE7E50823E5E54FF40063E2E5002358
:103910005B68FFDE00239B88FFDE00BF2DE9F04FD0
:10392000B14C8DB094F8C47F1FB900200DB0BDE834
:10393000F08F00222F2138460EF08CFA0646002820
:10394000F3D090F80580D0F80090A4F8DC83FDF760
:10395000BFFE0028E9D0D0E901530093002DE4D048
:10396000DFF8C0A20022514601E0102ADDD04868ED
:10397000013224318542F8D1D2B29C4B013A02EB9C
:10398000C20203EB820292F958B1BBF1000FCCD115
:103990002F214846C4F89093A2F85811FFF7EAFA8D
:1039A000934A904280F0FE805A464FF0010B484601
:1039B0000192FFF7DFFA019A8E49C4F89423B0FB15
:1039C000FBF2120A8C48A1FB02210022C4F8A023BA
:1039D000C4F898230A090909A0FB0202C4F89C1341
:1039E0005208A4F8C82F5200A4F8C62F94F8CD238B
:1039F00002F0FF01002A00F0E580022248467F49DC
:103A000084F8CD2340F072FA0122384684F8D82396
:103A100084F8CE2384F8CF2384F8D02384F8D123EC
:103A200084F8D22384F8D32384F8D42384F8D523CC
:103A300084F8D62384F8D72384F8CD23FEF7E2FD5B
:103A4000C4F8CC0F28B12F21C1804E21F279FDF7A7
:103A500083FF6B4A0021009BB8F10C0FC4F8DC1FF8
:103A6000C4F8D43FC4F8EC1FC4F8F41FC4F8FC1F1A
:103A7000D2F8D800C4F8D05F40F00100614BC2F822
:103A8000D800D2F8D80000F0010002900298D2F8D5
:103A9000D80040F00200C2F8D800D2F8D82019604F
:103AA00002F002020392039A4FF04002C4F8D82FAA
:103AB0004FF48062C4F8E02F4FF48052C4F8E42F32
:103AC0004FF48042C4F8E82F4FF40032C4F8F02FCE
:103AD0004FF00302C4F8F82F77D84B4A02EB4802A4
:103AE000B2F8DC7DB946083748485146002204EB5D
:103AF000870ECEF89003A0F54460986048680132C4
:103B00002431854264D0102AF8D14FF0FF32374B70
:103B100002EBC20203EB8202D2F83C013C4A904223
:103B200014BFA120A02046F093FE0022DAF8041072
:103B300001320AF1240A8D424DD0102AF6D100201C
:103B400004EB87044B4660223249FDF709FED4F8A6
:103B500090033EF03BFD00287FF4E7AEB4790027E8
:103B600060260A906300424604A92B4803F0020332
:103B70000693E300CDE9046703F00803002600275D
:103B80000793CDE9086745F0EBFE00287FF4CDAE42
:103B9000A3074146204820D540F01CFAB0FA80F037
:103BA0004009C3E64846FFF7E5F91C4A1C490244B0
:103BB000A1FB0212920D02F1FF3B1FFA8BF202F100
:103BC000010BF4E684F8CC1317E789460F468AE721
:103BD000D2B2013A9BE7D0B2B2E740F0FBF8B0FABC
:103BE00080F04009A2E600BF801A002400000024F3
:103BF000006CDC02598B4F01ABAAAAAA141E002448
:103C000000440258802A002460330908502A002406
:103C100000000240D5020000101E002400366E0194
:103C2000819F5E163C010024830AA3F58013522B6A
:103C300000D970472DE9F04115460F4AD65C0D2E8C
:103C400017D80E4C4FF04C08013908FB064789B2D3
:103C5000C7F8341BFFF78EF907F62C31B0FBF5F2ED
:103C6000013AD7F8280BC7F82C2BBDE8F04140F0FB
:103C70003DB9BDE8F08100BF60330908801A002417
:103C8000830AA3F58013522B6ED82DE9F04390469A
:103C9000714A85B0D65C0D2E63D84C256F4F044613
:103CA00006FB05F507EB0509D9F8283B834258D0F8
:103CB0000139C9F8280B083589B2C9F8341BFFF758
:103CC00059F907F628310023B0FBF8F00D4401380C
:103CD000C9F8303BC9F82C0BC5E9023399F8653BAC
:103CE00003F0FF02002B40D04C25022305FB0611F8
:103CF00005FB06750431D5F8288B85F8653B4046F1
:103D000040F0F4F8012385F8703B85F8663B85F8B0
:103D1000673B85F8683B85F8693B85F86A3B85F821
:103D20006B3B85F86C3B85F86D3B85F86E3B85F801
:103D30006F3B85F8653B4A4B9C4219D0B4F1804FEC
:103D400016D0A3F57C439C4212D003F580639C42BD
:103D50000ED003F580639C4260D003F578439C420B
:103D60005CD005B0BDE8F083704789F8642BBBE7F1
:103D70004C2303FB067393F8642B012AF1D0022233
:103D800083F8652B374AD8F808100A40C8F808208D
:103D9000012283F8652B002283F8642B00224C2338
:103DA0002F4903FB067303928845CDE901224FF0AA
:103DB000020283F8652BD8F80420D8F8083028D000
:103DC00001F58061884524D022F07002C8F80420F3
:103DD000254A90450DD0B8F1804F0AD0234902F50D
:103DE0000062904518BF884503D002F540629045B7
:103DF00003D123F08003C8F808304C2301210022AE
:103E000003FB067383F8651B83F8642B05B0BDE8DC
:103E1000F08317491140C8F80410EAE74C2303FB6C
:103E2000067393F8642B012A9BD0022283F8652B3A
:103E30000C4AD8F808100A40C8F80820012283F874
:103E4000652B002283F8642B0A4B9C42A6D003F515
:103E500078439C42A2D084E760330908801A00248A
:103E6000000001408800CEFF000400400008004030
:103E70008FFF0FFF000C004037B590F867380446FD
:103E8000032B2FD10023204D8DF807309DF80730EC
:103E900094F868289A4201D803B030BD9DF80730E5
:103EA00005EBC30313F8AC3C8BB181F0010383B184
:103EB0009DF8073005EBC30353F8B00CFDF740FD48
:103EC0009DF807300133DBB28DF80730DEE70B4693
:103ED000EDE79DF8073005EBC30353F8B00CFDF791
:103EE00035FDEDE7D0E910039B7903F0010399421A
:103EF00004D003B0BDE83040FDF722BD03B0BDE8FB
:103F00003040FDF723BD00BF782B002438B50446B0
:103F100000790D4650B1FEF775FB08B10323C3804D
:103F2000E2792946BDE83840FDF73ABD38BD10B505
:103F300004462221FFF7EAFF2046FEF74DFE204609
:103F40000121BDE81040FEF71FBE10B50446012157
:103F5000FFF7DCFF00212046BDE81040FEF714BE4D
:103F600038B510F8133CA0F66C041BBB94F8583815
:103F70008BBBD4E909239A421CD05A1CA169A262C6
:103F8000CB5C21695B008A4228BF002243F40073A6
:103F9000A262A4F85C380A2384F85A38012384F812
:103FA000583894F86738012B01D0042B02D1606C8B
:103FB000FFF7CBFF94F85438002B6DD194F85538A7
:103FC0000133DBB2092B84F8553825D12046BDE8F2
:103FD0003840FCF73FB994F95A586DB1B4F85C1801
:103FE000013D20464B0801F00101A4F85C38FFF7C1
:103FF00043FF84F85A58DDE7D4E9092384F8585878
:104000009A42D7D194F86738012B01D0042BD1D133
:10401000606CFFF78CFFCDE70A2B3DD194F8573841
:104020002BB9B4F85E3843F00103A4F85E38237965
:10403000D9070AD5B4F85E08820501D4C30718D49D
:10404000B4F864380133A4F864380122002384F8FA
:10405000542894F8572884F85538012A1CD16179DE
:10406000606C84F8573801F00101BDE8384045F034
:1040700079B9E36AC0F3470013B1216B9847E4E7CD
:10408000E3696269D054E369E2680133B3FBF2F19A
:1040900002FB1133E361D8E738BD00BF2DE9F043DF
:1040A000BFB0BFF35F8FA24A0020516A03460446A7
:1040B00021F4803151620146C2F89400C2F8983070
:1040C0000133C2F89C10112BC2F8A010F6D10523C1
:1040D000C2F89430536A43F480335362BFF34F8F76
:1040E000BFF36F8F9348944A9449121A4EF064FDBF
:1040F0009348944A9449121A4EF05EFD934BDA6D40
:10410000042A00F0FB8005D8012A00F07283022AFD
:1041100000F08583864A00238D4C0120D2F8881058
:104120008C4E41F470018C4DC2F8881020602361E0
:10413000216841F0800121602168014321602168EC
:1041400041F480312160216841F480512160A361F4
:10415000E3612362A362E36223636363A363E363B4
:1041600023646364216821F4802121607B492366F4
:10417000C1F808014FF000614FF6FF00784B9160E5
:10418000D16801400B43D3603FF0B8FBA3690246FE
:104190000F20C3F30323A169334493F82C3203F0B7
:1041A0001F0322FA03F3C5F8A4333DF08DFE6D4AD8
:1041B000D36813F0040FD36840F0A2806A4B00214B
:1041C000684A0591D96A21F00101D962DB6A03F0DE
:1041D00001030593936943F440439361936903F4A6
:1041E00040430593059B93699B04FCD54C22002119
:1041F0000EA85E4C4EF03EFD5D4A42F2030312688B
:10420000B3EB124F4FF000030893A4F1140308BF5F
:104210001C46E268002A4DD0534B5249D86A20F020
:104220000100D862DB6A03F0010308938B6923F471
:10423000404313438B618B6903F440430893089B0D
:10424000484A93699F04FCD5414B4FF44037494895
:104250000321D3F8E02042F08002C3F8E0200122DD
:10426000D3F8E03003F080030793079B87610D9B31
:104270000091019300234AF0EDFA022322690EA86F
:10428000CDE91733A3781E9201221993A3881A93BC
:10429000A3791B93E3791C93237A1D9300231F9327
:1042A0004FF48033CDE90E233FF070F803283BD064
:1042B00098B1FEE72B4A2C4B916941F44041916142
:1042C000926902F440420892DA6A42F00102DA622C
:1042D000DB6A03F001030893B1E7274B1A6812F079
:1042E0000E0F4DD11A6822F00F0242F002021A603E
:1042F0001B6803F00F03022B42D0FEE7DC6509E7E1
:1043000023F007031D4C43F00203D36054F8701CE4
:1043100006E054F8703C5B1AB3F57A7F3FF64EAF77
:1043200053689804F5D549E772B6FEF7A3FB00BFC2
:1043300000ED00E000000000A84200004C400A0828
:104340000000002004000020C6A70A080040005812
:104350000044025860330908000000240080005126
:104360000003FA0500480258000400589003002496
:104370000010005C001C025800200052782B002422
:104380006E4A936903F070033F2B05D8936923F0BD
:10439000700343F040039361684AD36903F07003EC
:1043A0003F2B05D8D36923F0700343F04003D3615A
:1043B000624AD36903F4E063B3F5806F05D2D36931
:1043C00023F4E06343F48063D3615C4A136A03F02F
:1043D00070033F2B05D8136A23F0700343F04003AA
:1043E0001362564B9A69100705D49A6922F00F029E
:1043F00042F008029A61514A936923F47063936111
:10440000136899017FF579AF136941F288304C4CFC
:1044100023F0070343F00303136154F8701C05E015
:1044200054F8703C5B1A834200F29B81136903F0DD
:104430003803182BF4D1936903F00F03082B05D927
:10444000936923F00F0343F0080393613D4A136817
:1044500003F00F03022B0BD9136823F00F0343F073
:1044600002031360136803F00F03022B7FF445AFC0
:10447000324A936903F07003402B05D9936923F006
:10448000700343F0400393612C4AD36903F0700337
:10449000402B05D9D36923F0700343F04003D36167
:1044A000264AD36903F4E063B3F5806F05D9D36975
:1044B00023F4E06343F48063D361204A136A03F07A
:1044C0007003402B00F245811C4F3FF017FA034662
:1044D000D5F8A803BA69B969C2F30322164496F85D
:1044E0002C2202F01F02D340C5F8A4333DF0ECFCAF
:1044F000002840F07D811023159017900EA80E9390
:104500003EF044FF002840F023813B680E4A43F010
:1045100080033B60D7F8F43043F00203C7F8F4306F
:10452000D7F8F43003F002030493049B136A43F0BA
:1045300001031362054B54F8701C0CE00044025850
:10454000782B0024002000520004005800E20400F0
:10455000013B3FF4E9AE54F8702C9142F8D054F886
:10456000702C54F8703C9B1A0A2BFAD9AF4C4FF4BC
:1045700080224FF440130EA80E924FF000082F93A4
:1045800049F050FBD4F8EC3041F20302A84903266D
:1045900043F002030EA8C4F8EC30D4F8EC3003F07A
:1045A00002030393039BD4F8943043F00203C4F84E
:1045B0009430D4F8943023F00203C4F894300B689C
:1045C0009C49B2EB134F9C4B9C4A28BF0A465A6049
:1045D0001A6822F47C5242F400521A601A6842F0BF
:1045E00060021A600E96CDE92B8849F01BFB4FF450
:1045F000E0430EA8CDF8E4800E93CDE9258849F07C
:1046000011FB18230EA8CDF8B8800E93CDF8CC80FE
:1046100049F008FB4FF400230EA80E934FF400332B
:10462000369349F0FFFAD4F8E0304FF480718448B3
:1046300043F00103C4F8E030D4F8E03003F00103A4
:1046400009934346099A0222CDE900684AF002F92B
:1046500023694FF400717B4823F0FE7343F08873A5
:104660002361D4F8E03043F00403C4F8E03043465B
:10467000D4F8E02002F004020692069A0222CDE964
:1046800000684AF0E7F8236923F07E4343F0FC43D7
:1046900023613FF033F96C4B6C4A4146C5F8A403E3
:1046A0001846D21A4EF0E6FA69486A4A6A49121A5E
:1046B0004EF082FABFF35F8F684D4646684C012783
:1046C0006B6A23F480336B62C5F8948023E0002981
:1046D00046D0D4F80090637A103414F8060C1B0608
:1046E00043EA007343EA410314F8051C43EA81439B
:1046F00014F8041C43EA414314F8031CC5F89860FD
:10470000013643EA0143C5F89C90032E43F00103B0
:10471000C5F8A03026D06368217A002BD7D0D4F812
:1047200000900029D7D129F01F01A3EB0108B8F1AF
:10473000200F38BF4FF0200840464EF07BFA431E52
:10474000014607FA03F0804508BF1946C9B2C2E71F
:10475000FEE7136A23F0700343F040031362B3E6ED
:10476000FEE7CAE50523C5F894306B6A43F480334D
:104770006B62BFF34F8FBFF36F8FBFF34F8FBFF3EA
:104780006F8F0022C5F85022BFF34F8FBFF36F8F9A
:104790006B6943F400336B61BFF34F8FBFF36F8FCF
:1047A000C5F88420BFF34F8FD5F8805043F6E076EC
:1047B0002A49C5F34E34C5F3C905640104EA06006D
:1047C0002B4640EA8372013BC1F86022F9D2203CBB
:1047D00014F1200FF2D1BFF34F8F4B6943F48033B4
:1047E0004B61BFF34F8FBFF36F8F3FB0BDE8F083D6
:1047F00083E50E4A02201B49D865D2F8F430034302
:10480000C2F8F430D2F8F43003400E930E9AD1F887
:10481000003883F30888D1F804389847FEE704216C
:104820000320FDF7AFFB72B6FEF724F900440258EF
:104830000010005C7FBB2200008400407FBB223060
:104840000000025800080258E0D6002480D7002457
:1048500040D40024E0D60024CAA70A0800ED00E0F6
:10486000AC0300240090F01F30B4EFF3118210234A
:1048700083F312880C4C4FF0E0200C4B0025D4F849
:104880003813D2B20131C4F83813816943F86C1C73
:1048900043F8685C016982F3118853F8702C013287
:1048A00030BC43F8702C7047801A0024782B002409
:1048B000254B5B68C3F3080330B4FBB9EFF31183F6
:1048C000E3B9224C4FF0E02C214BD3F83823DCF82D
:1048D0001800D3F838138A42F7D154F86C1C884278
:1048E000F3D8D3F8E0434FF47A7101FB04F3181ABC
:1048F000B0FBF4F030BC01FB02007047EFF3118213
:10490000102383F312884FF0E023104C9D6919693E
:10491000C90303D5012144F8681C9D690C49D2B232
:10492000D1F8380354F8683C82F311884FF47A7256
:10493000D1F8E013034402FB01F0401BB0FBF1F09F
:1049400030BC02FB0300704700ED00E0782B002430
:10495000801A00242DE9F8431B4EFFF7A9FF756864
:10496000002D1BDD07464FF000084FF48679002329
:104970001C4609FB0362013392F80521AB4244EA6D
:104980000204F6D1FFF794FFC01BB0F5FA6FCCBF5D
:10499000002304F0010333B19846E8E7FFF788FFEE
:1049A0000020BDE8F88344EA080010F0FF00F8D0CA
:1049B000064B13F8642C542AF3D133F85C2C0132E3
:1049C00023F85C2CBDE8F88304000020782B002439
:1049D000BE4803780BB9012070474368BC4A002BDE
:1049E0002DE9F04FD2F8386387B018DD00F10805E3
:1049F0000024B849D5F8F430BFF34F8F03F5907217
:104A0000C1F85C3220339342FAD1BFF34F8FBFF32A
:104A10006F8F0134436805F586759C42EADB90F898
:104A2000F8154FF00009AC4A0491A2FB0612AB4BFB
:104A3000AB4D5209DFF8C0B2A3FB0213DB0803EB56
:104A40008303A2EB4303DAB205EB830A05F538735F
:104A500005920093049B994500F01681DBF818300D
:104A6000DBF80470D3E93D46FFF722FFDFF88CC284
:104A70009C4901221CF8648C71180190B8F1540F04
:104A80001CF8500C02FA07F204EB410104EB40035E
:104A900001D12CF85A0C994240F26B811F881742C1
:104AA00000F060815F88174200F071819F88174293
:104AB00000F06F81DF8808331742ECD11C1B99424C
:104AC0004FEA640440F25581301B452828BF452039
:104AD00003EB4000834280F0508100261F46B6461B
:104AE0003146CDE90298B3F8008008EA020888450B
:104AF0001CD1B3F8028008EA0208414540F01B814E
:104B0000B3F8048008EA0208414540F01681B3F882
:104B10000690083309EA0209494508D1984209D9A3
:104B2000B3F8008008EA02088845E2D002339842D0
:104B300000F2E680BEF1110FDDE9029840F21D811E
:104B4000DEF1150200F1198167495CF84C0CD1F8CF
:104B5000DC339C4238BFC1F8DC43019C231A002B94
:104B600014DB624B03449C4201D9234605334CF8C5
:104B70004C3CD1F8DC33052B40F20D81053BDBB218
:104B80000CF8503C4FF0FF33C1F8DC333AB106FA71
:104B900002F2CEF1140E012606FA0EF61643544B1D
:104BA000C6F3C43203EB8202D2F8F80D06F01F02FE
:104BB00003EB8202D2F8F81DC6F34412C6F3842632
:104BC00003EB820241EA0031D2F8F82D03EB8603B1
:104BD00041EA0211D3F8F83D41EA0321454B81EA4D
:104BE0001122D3F8403A82EA1212013302F00F0286
:104BF0000F2A40F0A480B1F5803F80F0A080B8F18A
:104C0000540F4FEA111147D03A4AB1F5606FC2F81C
:104C1000403A4DD0009B998195F8583005988342D1
:104C200010D0DAF808202B689B1A2B606B68DAF832
:104C300030209B1A6B600023CAF80830CAF8303065
:104C400085F858002B6801332B60DAF808300133FF
:104C5000CAF808304FF6FF73994207D16B680133E9
:104C60006B60DAF830300133CAF83030009B09F15C
:104C700001095C350AF15C0A1433B9F1080F0BF134
:104C8000200B00937FF4E6AE01231A4A012082F83C
:104C90003C3B07B0BDE8F08F3CF8602CB1F5606F8D
:104CA00002F101022CF8602C124AC2F8403AB1D14C
:104CB000074A537803EB430302EBC3034B445B7C8B
:104CC0000D2BA7D18023009A9377A5E7040000203D
:104CD000801A002400ED00E01F85EB51CDCCCCCC38
:104CE00054180020C7FFFF7F0000002420A1070008
:104CF00060330908FC1000203C040020782B0024BD
:104D0000A3EB0708254F33F8021C4FEA680811404F
:104D100008F1010887FB0897A7EBE8774FF0010837
:104D2000012FB8BF0127BE40BE44013F08FA07F774
:104D30003E431F46D7E60433F9E60633F7E6B8F1FB
:104D4000540F04D13CF8602C01322CF8602C144A2A
:104D50004FF6FF71C2F8403AD2F83C3A0133C2F83C
:104D60003C3A59E702331C1B99424FEA64043FF670
:104D7000ABAE10B101380CF8500CB8F1540F7FF401
:104D800075AF3CF85E3C01332CF85E3C6EE70433B3
:104D900094E6063392E60023F2E600BF56555555D9
:104DA000FC100020264B70B51A785B789A4242D1ED
:104DB000244E7368002B22DD06F108000025224CEA
:104DC000D0F8AC30BFF34F8F03F1E002C4F8683283
:104DD00020339342FAD1BFF34F8FBFF36F8F3378F5
:104DE00013B1037F012B20D042690135716800F5B2
:104DF00086701368A94243F001031360E0DCFFF7FB
:104E000057FD124BD3F85447002C0DDD03F23473D9
:104E100003EBC4041968083333F8042CC8689C42B7
:104E200042EA0002CA60F5D170BD002380F8FC3070
:104E3000FBF70CF9D8E74BF049F90028B8D170BD61
:104E4000801A00240400002000ED00E0FC10002087
:104E50002DE9F04F484D85B02B781BB9012005B0E6
:104E6000BDE8F08F454BD3F83843FFF721FD95F8A7
:104E7000F8350193002B00F0C881414B05F5C06562
:104E8000404E0027A3FB042300955B09A6FB0326E5
:104E90003D4AF60802F5EB6806EB8606A3EB4606EC
:104EA000D2F8483BC11A1346F2B203F6382A08EB8F
:104EB000860689460392B9F1000F05DB009BD3F803
:104EC00024314B4500F388814FF4B4732A4A03FB25
:104ED000072393F82037002B00F0C080009D2B485B
:104EE000D5F85C11AB681A68CBB221F0FF01103B1A
:104EF000A0FB030326481B09C35C0B44A9895C681B
:104F0000D368A4B223EA0103C4F11604D360072CCA
:104F100040F2A4801C4A0121D5F86451D2F8403AED
:104F20008B46AE4602970133C2F8403A0022286809
:104F3000944614E0BCF1140F2CDC13F1080748BFB1
:104F400003F117073B110CEB271C5F1E013102FA1E
:104F500003F30BFA07F78C4247EA03021AD303461E
:104F60008C425EF8040FA0EB0303E3D8CCF11503E9
:104F70004FF0150CE9E700BF04000020801A002460
:104F80001F85EB51CDCCCCCCFC100020ABAAAAAA3B
:104F900020B10908BCF1150F029F40F013819F4812
:104FA000C2F38423C2F3441100EB830300EB8101BD
:104FB000D3F8783ED1F8781E1B0243EA011302F0C1
:104FC0001F01C2F3C43200EB810100EB8202D1F871
:104FD000781ED2F8782E0B4343EA023383EA132279
:104FE00082EA121202F00F020F2A40F0EB80C3F3A4
:104FF0000F134FF6FF72934200F0E480B3F5606F39
:1050000000F0EE80AAF80C3098F8582003988242FD
:1050100010D0B168D8F80020521AC8F80020D8F88B
:105020000420316B521AC8F804200022B2603263A7
:1050300088F85800D8F800200132C8F80020B2687B
:105040000132B2604FF6FF72934207D1D8F80430B4
:105050000133C8F80430336B01333363009C0137EC
:1050600008F15C085C3620460AF1140AFCF7CCFF14
:1050700004F5B4730093019BBB427FF41CAF6849F5
:105080000122002381F83C2BC1F8483B6549D1F847
:10509000083691F8D8261B6812F0020FD1F81C17B9
:1050A0001A6A0CBF0A4342EA81021A62019B012B71
:1050B0003FF4D4AE5B49D1F8703791F840281B68B3
:1050C00012F0020FD1F884181A6A0CBF0A4342EAA0
:1050D00081021A62019B022B3FF4C0AE5149D1F804
:1050E000D83891F8A8291B6812F0020FD1F8EC19F2
:1050F0001A6A0CBF0A4342EA81021A62019B032B1F
:105100003FF4ACAE4749D1F8403A91F8102B1B68F8
:1051100012F0020FD1F8541B1A6A0CBF0A4342EA7C
:1051200081021A62019B042B3FF498AE3D49D1F8ED
:10513000A83B91F8782C1B6812F0020FD1F8BC1C28
:105140001A6A0CBF0A4342EA81021A62019B052BCC
:105150003FF484AE3349D1F8103D91F8E02D1B683F
:1051600012F0020FD1F8241E1A6A0CBF0A4342EA59
:1051700081021A62019B062B3FF470AE2949D1F8D7
:10518000783E91F8482F1B6812F0020FD1F88C1F5F
:105190001A6A0CBF0A4342EA81021A62019B082B79
:1051A0007FF45CAE204A52F8203C92F8B0001B68B5
:1051B000D2F8F41080071A6A4CBF42EA81020A430F
:1051C0001A624BE6164AD2F83C3A0133C2F83C3A2E
:1051D000AFB14FF6FF7317E7002005B0BDE8F08FC1
:1051E00012494A7802EB420201EBC2023A44527C75
:1051F0000D2A7FF407AF80228AF81E2004E7294693
:1052000058220B484DF0D8FCE3E719460122044B25
:10521000C3F8481B83F83C2B20E600BF6033090825
:10522000FC1000200400002004100020801A00243C
:10523000E01B002038B50546FFF73AFB0446FFF7B0
:1052400037FB001BA842FAD338BD00BF2DE9F04759
:10525000294D00F1FF38294C1027294EFFF728FB74
:105260004FF001094FF0E02C4FF47A7E7368C3F3DE
:10527000080303BBEFF31183EBB9D4F83833DCF840
:105280001810D4F838239342F7D155F86C2C91427A
:10529000F3D8D4F8E0A30EFB0AF2521AB2FBFAF2EA
:1052A0000EFB03231B1AB3F57A7FDFD3B8F1010895
:1052B000D4D2BDE8F087EFF3118387F31288DCF8CE
:1052C0001810DCF81020D20303D545F8689CDCF8F0
:1052D0001810D4F83823DBB255F868AC83F3118882
:1052E0005244D4F8E0A30EFB0AF35B1AB3FBFAF3C3
:1052F0000EFB0233D6E700BF782B0024801A00246F
:1053000000ED00E001302DE9F04F5FFA80FA83B044
:10531000544E4D1E544C4FF01008544FD3464FF48A
:10532000FA7943F061FD0195FFF7C2FA4FF0E021F1
:105330004FF47A7C4FF0010E7B68C3F30803002B17
:1053400072D1EFF31183002B6ED1D4F838338A6910
:10535000D4F83853AB42F8D156F86C5CAA42F4D872
:10536000D4F8E0A30CFB0AF5AA1AB2FBFAF20CFB84
:1053700003231B1AB3F57A7FDED3B9F10109D3D128
:10538000019D4FF47A79584643F084FE0195FFF76A
:105390008FFA4FF0E0214FF47A7C4FF0010E7B68DA
:1053A000C3F308031BBBEFF3118303BBD4F83833FB
:1053B0008A69D4F83853AB42F8D156F86C5CAA42EB
:1053C000F4D8D4F8E0A30CFB0AF5AA1AB2FBFAF25F
:1053D0000CFB03231B1AB3F57A7FE0D3B9F1010963
:1053E000D5D1019D013D9AD203B0BDE8F08FEFF316
:1053F000118388F312888D690A69D20302D546F8B1
:1054000068EC8D69D4F83823DBB256F868AC83F3C6
:1054100011885244D4F8E0A30CFB0AF35B1BB3FBE6
:10542000FAF30CFB0233D5E7EFF3118388F312880C
:105430008D690A69D20302D546F868EC8D69D4F803
:105440003823DBB256F868AC83F311885244D4F8A1
:10545000E0A30CFB0AF35B1BB3FBFAF30CFB023378
:1054600087E700BF782B0024801A002400ED00E0BD
:105470002DE98848431C0A265A4DDFF870815FFAEF
:1054800083FB594C4FF4FA79B24643F0ADFCFFF779
:105490000FFA01264FF0E0214FF47A726368C3F3EC
:1054A0000803002B7BD1EFF31183002B77D1D8F8C1
:1054B00038C3D1F818E0D8F838339C45F7D155F8FF
:1054C0006C3C9E45F3D8D8F8E033D8F8E07302FB83
:1054D00003F3A3EB0E03B3FBF7F302FB0C331B1A2E
:1054E000B3F57A7FDAD3B9F10109D0D14FF47A79E3
:1054F000584643F0CFFDFFF7DBF901264FF0E021DE
:105500004FF47A726368C3F3080333BBEFF311837C
:105510001BBBD8F838C3D1F818E0D8F838339C450D
:10552000F7D155F86C3C9E45F3D8D8F8E033D8F85D
:10553000E07302FB03F3A3EB0E03B3FBF7F302FBF1
:105540000C331B1AB3F57A7FDCD3B9F10109D2D140
:105550005646013E96D143F0D7FFEFF3118C10234E
:1055600083F312888B691F460B69DB0303D545F86B
:10557000686C8B691F46D8F838E35FFA8CFC55F8E5
:10558000683C8CF311887344D8F8E0E302FB0EFC0E
:10559000ACEB070CBCFBFEFC02FB03C3D1E7EFF353
:1055A000118C102383F312888B691F460B69DB0370
:1055B00003D545F8686C8B691F46D8F838E35FFA65
:1055C0008CFC55F8683C8CF311887344D8F8E0E300
:1055D00002FB0EFCACEB070CBCFBFEFC02FB03C3A6
:1055E0007DE700BF782B002400ED00E0801A002446
:1055F0002DE9F043144C83B0DFF85090DFF8508071
:1056000004F5906602E00834B44219D094F90650CB
:10561000002DF8D12768083407EB08039B0A09EB33
:105620004303B3F8180245F013F934F8041C0123BE
:105630002A463846CDE9005549F00CF9B442E5D187
:1056400003B0BDE8F08300BFC82000246033090820
:105650000000FEA70246074B02209A4208D80133F9
:105660005B0840009A4280B202D2FF28F8D9704706
:10567000704700BF7FF0FA0211F001010ED170B542
:1056800090F8285082B00446012D08D0C368B3F1C9
:10569000807F01D90123037702B070BD70470B4BA7
:1056A000466A53F8480CFFF7D5FFE368B080B3F1C2
:1056B000807FF1D94FF0B70C0A4630462B4601A93E
:1056C00025778DF804C037F0E7FEE5E7782B002456
:1056D0002DE9F0411F46436A94B014460646186807
:1056E0000D4649F07DFD0B940022274C069204F5EF
:1056F00090738DF820201392009304F5A0730C97FB
:1057000001930223CDE9092202930123CDE90E2260
:10571000CDE910221D4A8DF80C308DF834308DF80B
:105720004830049204F58072337F05921A1D079267
:105730002BB32B0E04F5817404F8013C2B0CA570DF
:10574000DFF84C802D0A2370657058F8480CFFF77D
:1057500081FF746A737FA080A3B16946204637F049
:10576000E1FE746A206849F03BFD58F8440CFFF7ED
:1057700071FF03463846A38014B0BDE8F08104F2FF
:105780000114DBE705A9E9E740D40024B1080408C7
:10579000782B00242DE9F04F002385B0DFF800A31B
:1057A0004FF001090193B94B0AF1F00BB84FA3F187
:1057B0007C080BE0019B09F101090AF1280A0BF1B1
:1057C000050B0133062B019300F0F1809AF80030AD
:1057D000022BEFD19BF90320511C00F0EB80D2B2D9
:1057E000944602EB4204A94B9DF8041003EB840499
:1057F0000F2A5ED8A74802E00330B84259D0037898
:10580000002BF9D145788D42F6D18578D8F84061E2
:105810006068A560B042257000F04481D8F86461EA
:10582000B04200F05E81D8F88861B04200F0628139
:10583000D8F8AC61B04200F06281D8F8D061B042D3
:1058400000F06C81D8F8F461B04200F08081D8F8A3
:105850001862B04200F07681D8F83C62B04200F0A5
:105860008081D8F86062B04200F07681D8F8843246
:10587000984200F08C81D8F8A832984200F08181DB
:10588000D8F8CC32984200F0A581D8F8F03298428E
:1058900000F09A81D8F81433984200F0A781D8F824
:1058A0003833984200F0A881D8F85C33984200F071
:1058B000978101320C34D2B2624599D90023039307
:1058C0009BF90420531C79D0D2B2964602EB4204D5
:1058D0006E4B9DF8041003EB84040F2A5DD86D48CD
:1058E00002E00330B84258D00378012BF9D1457853
:1058F0008D42F6D18578D8F840616068A560B042E5
:1059000025705FD0D8F86461B04200F0EF80D8F81D
:105910008861B04200F0F880D8F8AC61B04200F085
:10592000F880D8F8D061B04200F0FD80D8F8F4617A
:10593000B04200F00281D8F81862B04200F0F8805E
:10594000D8F83C62B04200F01781D8F86062B042EB
:1059500000F00C81D8F88462B04200F02481D8F8BD
:10596000A832984200F01981D8F8CC32984200F061
:105970002581D8F8F032984200F01A81D8F8143313
:10598000984200F04B81D8F83833984200F04081BB
:10599000D8F85C33984200F0358101320C34D2B231
:1059A00096459AD200220023CAE9042302E705B0F3
:1059B000BDE8F08F4FF00F0C002212E74FF00F0EF2
:1059C000002283E700231E46029306EBC600013641
:1059D00008EB800090F958C1BCF1000FDDD16246A0
:1059E00080F84431AC462C4B1546029AC0F848C1A9
:1059F000134480F85991CAF81430132380F85831B1
:105A00003046FBF789FE039B002BCBD0DAF814401D
:105A10002046FAF7F5FADAF81000FAF7F1FADAF8B0
:105A20001830C168DAF80420596240215D6099603D
:105A300002F120019D631960C3E90355C3E90555CF
:105A4000C3E90755C3E90A55C3E90C55A4B1DAF80F
:105A50001C303032E1681D625962C3E900254FF401
:105A60008032C3E90255C3E90455C3E90655C3E9C9
:105A70000B55C3E90D559A620023304607491A4673
:105A8000FBF76EFE01238AF80C3093E67C000024BD
:105A9000A6340908283409083C0100244506000002
:105AA000382B00241846029300EBC00E013008EB9F
:105AB0008E0E9EF95861002E7FF4FBAE029A8EF88E
:105AC0004431594BCEF8485113448EF85991CAF8D5
:105AD000103014238EF85831FBF71EFE0123039378
:105AE000EEE62420012302901846DDE724201E461E
:105AF00002906AE74820022302901846D4E76C20FF
:105B0000032302901846CFE7022348201E46029046
:105B10005BE703236C201E46029056E79020042387
:105B200002901846C0E7042390201E4602904CE7DE
:105B30000623D8201E46029047E70523B4201E46C0
:105B4000029042E7D820062302901846ACE7B42022
:105B5000052302901846A7E74FF4907002900820A2
:105B6000A2E7FC200723029018469DE74FF49073AC
:105B700008260293002328E70723FC201E460290F4
:105B800023E74FF4B470022302900A208CE74FF40D
:105B9000A27309200293012386E74FF4B470022315
:105BA0000A26029011E74FF4A270092602900CE732
:105BB0004FF4D8730C260293042306E74FF4C67300
:105BC0000B260293032300E74FF4D8730C200293B3
:105BD000042369E74FF4C6730B200293032363E7A2
:105BE0004FF407730F20029307235DE74FF4EA7326
:105BF0000D200293052357E74FF4FC730E20029308
:105C0000062351E74FF407730F2602930723DCE6C0
:105C10004FF4FC730E2602930623D6E64FF4EA7384
:105C20000D2602930523D0E63C0100242DE9F04F18
:105C30004C484FF0010A4C494FF002094B4B4FF0D2
:105C4000040808271026202540244FF0800EDFF896
:105C500020C130F8022F12F0010F03D01960083371
:105C600023F804AC12F0020F03D01960083323F8B4
:105C7000049C12F0040F03D01960083323F8048C3D
:105C800012F0080F03D01960083323F8047C12F0D7
:105C9000100F03D01960083323F8046C12F0200FA2
:105CA00003D01960083323F8045C12F0400F03D0CE
:105CB0001960083323F8044C12F0800F03D01960E8
:105CC000083323F804EC12F4807F05D04FF4807B76
:105CD0001960083323F804BC12F4007F05D04FF498
:105CE000007B1960083323F804BC12F4806F05D0E0
:105CF0004FF4806B1960083323F804BC12F4006F72
:105D000005D04FF4006B1960083323F804BC12F47B
:105D1000805F05D04FF4805B1960083323F804BC22
:105D200012F4005F05D04FF4005B1960083323F8CC
:105D300004BC12F4804F05D04FF4804B1960083337
:105D400023F804BCD20B05D04FF40042196008338D
:105D500023F8042C01F5806161457FF47AAFBDE83A
:105D6000F08F00BF9A35090800000258C8200024AF
:105D7000002402582DE9F0470546086888B00C4613
:105D80004FEA902CBDF84080ACF5801C9DF844A0F3
:105D9000BCF1520F58D819462E4B13F80C600D2E3B
:105DA00052D806EBC6032C4F06EB430307EB8307E1
:105DB000FDF766FF94F80590A379BAF1000F01D0C2
:105DC00083F001035A004FF48071DB00384602F083
:105DD0000202CDF8088003F0080303924A460493B8
:105DE000602301934FF40073CDE90613002301A94A
:105DF000059343F0B5FDA379384649469F0726D45D
:105E00003DF0E8FF4C22154B02FB063393F8652B5F
:105E1000012A10D10221D3F8282B83F8651B104BDF
:105E200091680B40062B06D0B3F5803F03D0136872
:105E300043F0010313602168637901F13402696062
:105E40000021D0182860D15008B0BDE8F0873EF09E
:105E5000C1F8D7E760330908A8250024801A002478
:105E60000700010010B4284C94F8303763B3226D5A
:105E7000904234D0012B27D0D4F82C21824236D046
:105E8000022B21D0D4F80822904232D0032B1BD011
:105E9000D4F8E42290422ED0042B15D0D4F8C0239D
:105EA00090422AD0052B0FD0D4F89C24904226D0C3
:105EB000062B09D0D4F87825904222D0072B03D0A6
:105EC000D4F85426824210D0DC22591C02FB034233
:105ED00084F83017106518465DF8044B70470023AE
:105EE000DBB25DF8044B184670470723F8E701233F
:105EF000F6E70223F4E70323F2E70423F0E70523A0
:105F0000EEE70623ECE700BFFC1000200548D0F8C0
:105F1000043323B1DB6A13B100F54170184702481E
:105F2000704700BF801A00245842090838B51D4C3C
:105F3000D4F8D0301B8843B91B4D002384F8DF30E0
:105F400085F8FC32C5F8F83238BDD4F8D420002AE0
:105F5000F2DDD4F8D810012A488806D00123124D6A
:105F6000A4F8DC0084F8DE30E7E78A880132121AF0
:105F70009A42F3D10C4D0022D5F8043305F5417057
:105F8000C5F830231B699847D5F804339B68002B6C
:105F9000D3D005F5417098470028CED143F0BCFA24
:105FA000CBE700BF782B0024801A00240748D0F8E4
:105FB00000331BB1064B93F8DE300BB10020704765
:105FC000D0F8043300F541705B681847801A00244C
:105FD000782B0024184A10B4184C92F8FC32446014
:105FE0002344174C036092F8FC0294F8DF3083429C
:105FF00018D892F8FC02834207D300235DF8044BC3
:106000001A461846C1E90032704792F8FC021A1E7F
:106010005DF8044BC0F180030CBF01200220C1E9F0
:106020000032704792F8FC42002201201B1B5DF8F1
:10603000044BC1E900327047801A002400D70024C5
:10604000782B0024104B114A93F8FC1292F8DF00D1
:1060500093F8FC22904293F8FC220FD8904204D38C
:10606000D3F8F83200201844704793F8FC22D3F894
:10607000F832C2F18002104418447047801AD3F8F5
:10608000F8321844704700BF801A0024782B00248F
:1060900038B5194D194CD5F8D020937B012B08D079
:1060A000D4F8F83203F2FF736FF30A03C4F8F8323E
:1060B00038BDD4F804335B6A63B104F54170984786
:1060C000D4F804339B681BB104F54170984778B14C
:1060D000D5F8D020D4F8F8325288013B514213440D
:1060E0000B4003F2FF736FF30A03C4F8F83238BDB4
:1060F00043F012FAECE700BF782B0024801A00244A
:10610000F0B51C4C85B01C4B94F8FC221B4D03933E
:10611000134495F8DF1094F8FC220293914294F80E
:10612000FC3216D899420CD294F8FC620F46C6F1A4
:106130008006D9B9334601223F2BCDE900670DD83F
:1061400060B994F8FC02401AB0FA80F0400905B03A
:10615000F0BDCB1A002701221E46EDE76946002359
:1061600002A84AF04FFC95F8DF10EAE77318022204
:10617000E2E700BF801A002400D70024782B002417
:106180002DE9F047174684B000293ED0441E294D22
:10619000DFF8AC904FF0000A04EB0108264E0DE04A
:1061A00096F8FC320846994296F8FC321DD2C3F1AB
:1061B000800318443F281BD8A04526D095F8DF005F
:1061C00014F8013F411C4844C9B280F820300B0646
:1061D00085F8DF10E4D5002096F8FC3285F8DFA0C2
:1061E0000146994296F8FC32E1D3C01A3F28E3D920
:1061F00096F8FC329942DFD0104B5B78002BDBD055
:106200000020FFF77DFFA045D8D1694602A8FFF71F
:10621000E1FEDDE9003213443F2B00D910B904B090
:10622000BDE8F08702463B4602A84AF0EBFB04B00B
:10623000BDE8F087782B0024801A00240000002499
:10624000E0D6002430B585B0694602A8FFF7C2FE4B
:1062500058B9094C04F54175D4F8043328465B68F5
:1062600098470028F8D005B030BD0246012302A8A7
:106270004AF0C8FBEDE700BF801A002438B50023C0
:10628000124C134DC5F8003342F004FBC4F8D8009B
:10629000FFF73CFED4F8D830C4F8D000A3B19A88F8
:1062A0005B88D21A436802FB0333C5F80033FAF760
:1062B00031FB94F8DF20044695F8FC329A4201D075
:1062C000FFF7C0FFC5F8F84238BD00BF782B0024A7
:1062D000801A00242DE9F041104E1546821804461C
:1062E000D6F800330F469A420D4A88BF1D1A92F81D
:1062F000DF2096F8FC329A4201D0FFF7A3FF00207E
:1063000021462B463A46C6F83003D6F80403846A81
:106310000448A446BDE8F041604700BF801A00244D
:10632000782B0024841D00248C46134601466246C7
:106330001846CFE72DE9F043484F93B0484DFFF79B
:10634000F5FD97F8FC3295F8DF209A4201D0FFF76F
:1063500079FF0024D7F80063C7F8F842002E6DD00B
:10636000DFF800810AE097F8FC3295F8DF209A42C6
:1063700001D0FFF767FF2034A6421BD922464146D1
:10638000684601F003FC68464AF042FC01220146DF
:106390006846FFF7F5FEA3B2002BE4D1D7F84033EF
:1063A000002BE0D09A881B6859690A4218BF120472
:1063B0009A61D8E7FFF76CFE97F8FC3295F8DF207A
:1063C0009A4201D0FFF73EFF0023DFF898909846ED
:1063D0001C46C7F8F8322246494609A801F0D6FB08
:1063E0002122002168464CF045FC202269462046C7
:1063F000FFF770FF2022054609A968464CF02AFDE8
:10640000A3B2203450B9202D08D15BB1A642E2D806
:10641000B8FA88F0400913B0BDE8F08308F101082C
:10642000002BF3D1D7F84033002BEFD01A689B88AC
:1064300051690B4218BF1B049361E7E7FFF728FE81
:1064400097F8FC3295F8DF209A4201D0FFF7FAFE68
:1064500000230120C7F8F832DDE700BF801A0024CE
:10646000782B00247CB0090808B53FF0FFFA1B2008
:10647000FCF7C8F808B12923C3801C20FCF7C2F838
:1064800008B12923C38048F031FB0B4845F0BCFB21
:106490000A4B93F8E520012A01D0012008BD084AE3
:1064A000D3F8C403C3F8C02348F060F90023054AB9
:1064B000184682F8233008BDE0030024782B00241E
:1064C0001804002400ED00E00A4B93F838241AB9B0
:1064D000094A92F8C80370470849CA6D032AF7D1E0
:1064E0000020054A4FF0010C83F8380482F8C8C335
:1064F000C865EEE700000024782B00240040005817
:1065000008B503220E4BDA6572B60E4BD3E9F412CE
:1065100051EA020306D100231A4609490A664B666E
:10652000FCF7F4FA084B4EF6602CD3F838330CFB2A
:1065300000F05B1842F10002C31842EBE072ECE796
:1065400000400058782B0024801A002400210320EA
:1065500008B5FBF717FD72B6FCF78CFA154C08B5B9
:10656000D4F8D83394F8DE03ABB91420FEF76EFEEE
:1065700000BFD4F8D8335BB1196894F8DE239B8848
:1065800009690B4012B91BB1FFF7E0FF002BFBD0EC
:10659000FAF7F4F9ECE719689A880B69134020B10F
:1065A000002BE2D10B691340FAE7002BDDD00B6919
:1065B0001340FAE7782B00242DE9F04F00218BB02F
:1065C00041F69462B8484CF055FB0420FBF7D4FC2C
:1065D00001460520FBF7D0FC51EA000340F057814B
:1065E000B24B03934C220021AF4801244CF042FBF4
:1065F00000214C22AC484CF03DFB039BAA4AD3F847
:106600006C34AB4D164614711560D361136253623E
:1066100045F0F2F9FFF732FE002108460AF090FA41
:10662000FAF778F9B0F1000840F39B810024A14DFE
:10663000DFF8A4E206F14C092746A24605F5787B6F
:106640009D4E0294CDF804E004E00AF5006AD045BE
:1066500040F3AE80019AD2F83833C2F83C33FAF7EF
:106660008DF9202259465046FFF734FE12229349F5
:1066700058464CF0EFFB0028E7D1BA4525D00299E7
:106680008F4B01EB410203EB82034A1C8D491846F4
:106690000293AAEB07030592049301F077FA029B99
:1066A0004946059A41F84C3B049BC9F80C7002928C
:1066B000C9E90433D9F81C30C9E908330123C9F802
:1066C0000830814BC9F828308946039B574612226F
:1066D000D3F86C34C9F81C30A918335D013291F835
:1066E000E01399420BD00024202AF5D120375946D7
:1066F000B845384653DBFFF7EDFD0022ECE70134E7
:10670000152CF1D1D019714F20223946FFF7E2FD47
:10671000384600230A2209A9099701F06BFB0746B6
:10672000099800230A2209A90130099001F062FBAF
:106730000790002309980A2209A90130099001F065
:1067400059FB0690002309980A2209A901300990F3
:1067500001F050FB059009A9099800230A22013095
:10676000099001F047FB0023049009980A2219467A
:10677000013001F03FFB97B10599DDE9063243EAAC
:106780004212049B5B0143EAC123A7F2BC7143EAB6
:10679000600342EA412243EA0243C9F81C30029BEB
:1067A000642B43D057460AF5006AD0453FF752AFF5
:1067B000029B642B1ED0BA451CD00C22404C5E1CA0
:1067C000404902FB0344AAEB07053246204601F08C
:1067D000DDF9D9F81C20C9F80040C9F80C70029600
:1067E000C9E908220122C9F80820374AC9E9045535
:1067F000C9F82820029B002B03F1010117DC4FEAA6
:106800004803B3F1805FC0F2AD80274B9C6834B978
:106810001A461B791BB11368002B40F0D980002168
:1068200008460BB0BDE8F04F0AF08AB965214C2646
:106830001D48DFF8A8A04FF0010906FB01F432461D
:106840000021234F051928464CF014FA3246002146
:1068500028464CF00FFA1C4E134804F1100204F1C4
:106860001803029940F804A0C5F8089002312F627D
:10687000AE6240F8028002440430C2F80480039AF9
:10688000D2F86C24C25003445A606A62B7E74FF4EE
:106890007A7200234AF01AFE0E4B40F2B27240F2B6
:1068A0006D14B0FBF3F31DE000350024000000245C
:1068B0000CB10908782B0024C0B009089CB0090865
:1068C000782F0024B0B0090829630408582F002449
:1068D0000068214C80510100801A0024D8B00908BA
:1068E0005B1A013212F0030514BF21464FF4B77151
:1068F0008B42F5DA8549002D64D003910399D1F8D4
:106900003C148B42C0F29C80814D01245B1A55F8E7
:10691000041F01349942F9DD0133A2F2BC72039DD8
:1069200043EA44133C2443EA42237A4AB0FBF2F19F
:1069300002FB11024FF46160B2FBF0F100FB112287
:106940001C20C5F84004B2FBF4F004FB10225210E6
:1069500042EA401242EAC12242EA0343C5F86C34DB
:1069600040E621464C266C4BDFF8B891012706FB28
:1069700001F4324600214FF0020A1D1928464CF05E
:1069800079F93246002128464CF074F9624B039A9B
:1069900004F1180143F80490C8F10063D2F86C04C4
:1069A00004F11002BB405C4C5C4E85F805A0AF6062
:1069B0002E62A35022445360231D5850194448604E
:1069C000686222E70C4603911D21C4F8401495E744
:1069D000514800220023214626468464C463C0E94E
:1069E00010230246D56C02F14C035DB398684D1E2E
:1069F0009E64A842C2E92366DE630DD04D1CA84206
:106A000010D113F8481C00293FF409AF1A6401465D
:106A10001A4643F8083CE5E700293FF400AF53F875
:106A20000C2C014600293FF4FAAE81427FF4F7AE08
:106A3000106CC56B0135C563186493641A46D1E7C1
:106A4000012469E7344A0226294613E0D36B166312
:106A50005B01C2E9041120D003F6FF7300EB13338E
:106A600018465363C31A906352F84C7F461C1D446A
:106A70000134C7B11379701E002BE7D11369166377
:106A80007BB103F6FF7300EB13335769536337B1E0
:106A900007F6FF7700EB1730E4E73346E0E73046D0
:106AA000E0E73346F1E7DFF880E00138CEF88C43C9
:106AB000820F1B4C8300CEF880533F25CEF86443F1
:106AC0004024CEF87C03CEF870433E24CEE9DA456C
:106AD000D0B140F2FF141B1942F100025B0A43EAF5
:106AE000C25303F140020C491344CEF8742303EB64
:106AF000C000CEF878334202CEF86003C30DCEE971
:106B0000E111CEE9D6238AE60123EAE7000000245A
:106B10003C04002480510100003500240068214C11
:106B2000F4B00908E8B00908801A002410B58C18E0
:106B3000A14215D001F1FF3E013C41F2210C1EF8AB
:106B4000012F082380EA022002B24000002A8CEACA
:106B5000420180B2B8BF88B2013BF5D17445EED195
:106B600010BD00BF704700BF2DE9F047002BDDF8D6
:106B700020A0884607460CBF4FF020094FF030098F
:106B80005646002A144616F8011B23DD11B333467E
:106B900001E0002C05DD13F8012B2546013C002AFD
:106BA000F7D1023D3CB149463846C047013DFAD2D3
:106BB0009AF8001059B13846C047334616F8011B01
:106BC0000029F8D1A4EB0A041819BDE8F087204683
:106BD000BDE8F087002C04F1FF35E4DC0024002937
:106BE000E9D1F4E703685A1C02601970704700BFCE
:106BF00010B56FF000440246044404E0B3EB0E000D
:106C000015D1A24214D012F8013BA3F1410019287A
:106C100011F8010BA0F1410C98BF203300F1200EB8
:106C2000BCF1190FEAD91B1A04D10028E9D110BD13
:106C3000002010BD184610BD884230B54FF0010449
:106C40003AD301FB04F4B0FBF4FC8C45F9D2BCB19F
:106C500002BB06E0A14203F8015B11D81446B0FB69
:106C6000F2FCBCF1090F0CF157050CF1300E04FBDE
:106C70001C00B4FBF1F2EDDCA14203F801EBEDD90D
:106C800000221A7030BDA14203F8015BF8D8144607
:106C9000B0FBF2FCBCF1090F0CF137050CF1300E22
:106CA00004FB1C00B4FBF1F2EDDCA14203F801EBA4
:106CB000EDD900221A7030BD8446002AEAD1D0E70F
:106CC000002870B503DA2D23404201F8013B092862
:106CD00086464FF0010307DD03EB83035B00B0FB47
:106CE000F3F2092AF8D89BB10F4CA4FB030CBEFBAE
:106CF000F3F2092A4FEADC0C02F1570602F13005E3
:106D000003FB12EE07DD092B01F8016B6346ECD89B
:106D100000230B7070BD092B01F8015B6346E4D8BA
:106D200000230B7070BD00BFCDCCCCCC0378202BE2
:106D300003D110F8013F202BFBD0092BF9D02D2BCC
:106D400000F0A9802B2B75D0B7EE000AA3F130021A
:106D5000D1B2092977D8F2EE046ADFED5F7A07EE47
:106D6000102A10F8013FB8EEC77AA3F13002D1B271
:106D7000A7EEA67A0929F0EE477AF0D92E2B66D035
:106D800003F0DF03452B40F0838010B442782D2AB6
:106D900000F096802B2A00F08380A2F130030130AE
:106DA000092B00F284800024002303EB830302EB11
:106DB000430310F8012FA2F13001303B0929F4D927
:106DC000B3F59A7F1A46B7EE007A28BF4FF49A724D
:106DD000072B09D91346DFED416A083B27EE267AD7
:106DE000072BFAD802F00702DAB1F2EE046A012AA0
:106DF00027EE267A15D0022A27EE267A11D0032A0A
:106E000027EE267A0DD0042A27EE267A09D0052A05
:106E100027EE267A05D027EE267A062A18BF27EE17
:106E2000267A002C45D0C7EE877A5DF8044B20EE19
:106E3000270A70474378B7EE000A0130A3F1300209
:106E4000D1B2092987D92E2BDFED237A98D1437847
:106E50000130A3F13002D1B2092991D8B2EE047AFF
:106E6000F0EE475A06EE902A10F8013FB8EEE66AB7
:106E7000A3F13002D1B2C6EE076A092927EE257ABE
:106E800077EEA67AEED903F0DF03452B3FF47DAF12
:106E900020EE270A70474378BFEE000A013055E71D
:106EA00082780230A2F13003092B7FF67CAFB7EE77
:106EB000007A67EE877A5DF8044B20EE270A704768
:106EC00082780230A2F13003092B01D801246BE74C
:106ED000B7EE007AA7E700BF0000000020BCBE4C60
:106EE000F8B5164D6B78BE2B25D1AC1C144F022281
:106EF00029464FF6FF70FFF719FE22884AB1A618FF
:106F0000BE4218D2052A16D921463446FFF70EFE96
:106F1000F3E721460222FFF709FE0222A1180634F8
:106F2000FFF704FE074B641B1C8041F60F53C31A86
:106F300058425841F8BD0020FCE700BF000002089D
:106F40000000040898530024F0B5067906F0E00329
:106F5000402B03D145794FF0FF3406E0602B4FF012
:106F60000105F8D1447905FA04F40023012006F064
:106F70000706AB4200D1F0BD052E0FD8DFE806F0C2
:106F80000308101D242448B1C85CD75C78400FE08A
:106F900020B1C856D756C71B784278410133E8E77D
:106FA0000028FBD031F8130032F81370784080B21B
:106FB00020420CBF01200020F0E70028EED031F97C
:106FC000130032F91370E6E70028E7D051F82300E8
:106FD00052F82370DAE7037903F01803102B1DD061
:106FE00003D833B9B0F80B007047182BFAD0002043
:106FF0007047114BB0F80B0093F90030591C0BD1BE
:107000000E4B1B7903EB430203EB820303EBC30339
:1070100000EB430080B27047DBB2F3E7064BB0F8F9
:107020000B0093F901305A1C04D1044B5B7900EB3F
:107030004310EFE7DBB2FAE78C04002498530024F6
:10704000032870B518D80D4BC943C60003EBC00028
:1070500001F00101057E427E81EA0504A2420BD0C7
:1070600042693AB14D1B1068928869426941090131
:107070008A40826133445C7670BD00BF985300241F
:107080000379062B0FD1C9B20D290AD8074B5956DF
:107090000123C2688B40134214BF08464FF0FF30F3
:1070A00070470021F4E7481C704700BF10B1090881
:1070B000B5EEC00ADFED357A0023F1EE10FA30B5F7
:1070C000C8BF30EE270A87B0D8BF30EE670ADFEDC1
:1070D000307A054603A9029320EE270ACDE9003352
:1070E000FDEEC07A17EE904A84EAE470A0EBE470FB
:1070F00040F068F8002C03A8B4BF2D2320238DF89E
:10710000003049F085FD01282AD0022834D0032818
:107110001ED003A968464BF0B5FD684649F078FDDE
:10712000044669462846033CE4B222464BF044FD3F
:10713000002328462B5549F06BFD2E22431C0DEBF6
:1071400004012A54E8184BF0CAFD284607B030BDA8
:10715000302303A968468DF801304BF093FDDCE73E
:1071600043F23002302303A96846ADF801208DF8C0
:1071700003304BF087FDD0E743F2300303A96846A4
:10718000ADF801304BF07EFDC7E700BF6F12033A48
:1071900000007A4409F002BC38B5054658B14C1ECF
:1071A00014F8011F284619B9BDE8384009F00ABC97
:1071B00009F0F4FBF4E738BD70B50546B0F80900F6
:1071C0003AF0D6FD064B0446284693F83460FFF7A4
:1071D00002FF16B1E368184470BDA368FBE700BF67
:1071E0009853002438B505460C46FFF7E5FF2A7989
:1071F00002F0070302F0E002602A29D1052B0CD827
:10720000DFE803F0030B0F0B1B1B6A79012393408C
:107210000278DBB214B11343037038BD22EA0303D2
:10722000FAE76A790123934002889BB214B11343B1
:107230000380F2E722EA0303FAE76B7901229A401E
:10724000036814B113430360E7E723EA0203FAE794
:10725000052BE2D8DFE803F00303050507070470F8
:10726000DBE70480D9E70460D7E708B520214BF0BD
:1072700018FD034618461BB102780133202AF9D0C5
:1072800008BD08B5CB0701D4FBF740FC08BD2DE9CC
:10729000F3410023124D044600EB8106114F05F81F
:1072A000353FB44203D1104802B0BDE8F081394601
:1072B00028464FF000084BF0E5FC214668464BF0AD
:1072C0000EFD202168464BF0ECFC28B969462846A3
:1072D00004344BF0D7FCE4E780F80080F1E700BF0E
:1072E00098530024D31F0A08CD5300242DE9FF47EB
:1072F000914604468A461E46FFF7C2FE421CBDF870
:1073000030700546DDF834801FD0B9F1FF3F1FD043
:10731000154A3146CDE9000938462368C0474A4638
:107320005FFA8AF12079FAF761F9024600B1028822
:10733000D3B2314638460393C2F30323120B0293B0
:10734000CDE90052094A2368C04704B0BDE8F08780
:107350007B06FAD40C90314623683846044AC4466A
:1073600004B0BDE8F0476047CE1E0A08DB1E0A08DD
:10737000FF1E0A082DE9F043154685B089461946D7
:107380006A1CBDF830600D9F28D04FEA101800F03D
:107390000F04194A304608F14008CDE9004543463C
:1073A000B847C0B1EBB2D9F8000099F805100F2B1F
:1073B00011D82A46FAF762F968B1038800210278E9
:1073C00030460392C3F303221B0B02920B4ACDE912
:1073D00000434346B84705B0BDE8F0837306FAD4CE
:1073E000030900F00F00064ABC460C9040333046BB
:1073F00005B0BDE8F04360470E1F0A08201F0A08C9
:10740000491F0A082DE9F043070987B091461E4637
:10741000DDF83880403700F00F0439B30AF0E2FBA2
:10742000C3790546164A49463046CDE900433B46F6
:10743000C047C0B12868FAF7C3F9AA796B7912F08E
:10744000020F10494FEA93030F4A18BF0A46E97921
:1074500001330094CDE90321CDE901030B4A3B46FA
:1074600000213046C04707B0BDE8F0833B46084ADC
:1074700049463046C4460E9407B0BDE8F043604725
:107480005D1F0A08BD200A08B32B0A086F1F0A08EF
:10749000911F0A080823484041B240000029C0B2A9
:1074A000B8BF5040013BF7D1704700BF30B5056809
:1074B00004468D4218D901F1FF3E681E00231EF8D4
:1074C00001CF082183EA0C034FFA83FC5B00BCF177
:1074D000000FDBB2B8BF53400139F5D17045EED192
:1074E0006A1C22602B7030BD00236A1C22602B7046
:1074F00030BD00BF9FED067AF7EE007A60EE870A96
:1075000060EE800A30EEA70A80EE800A704700BF66
:10751000DB0FC94010B52DED028B08EE101ADFED20
:10752000807ADFED800A0446B8EE488A28EE008AA9
:1075300028EE278AB0EE480A4AF034FE9FED7A7AA8
:10754000F0EE407AB4EEC70AF1EE10FA40F3BD80D7
:107550009FED746ADFED756AB0EE677A77EEC67AF2
:10756000B4EEE67AF1EE10FAF6DC9FED717AF4EE05
:10757000C77AF1EE10FA40F3C5809FED6B7A77EE93
:10758000677A27EEA76ADFED6B5ADFED6B6A9FED36
:107590006B7AE6EE256A9FED660A67EE865ADFEDA6
:1075A000610A38EE000AA6EE267AE5EE877AB0EE9A
:1075B000678A4AF0F7FDDFED5C7AB4EEE70AF1EE98
:1075C00010FA5BDDDFED576A9FED587AF0EE407AF6
:1075D00030EE660AF4EEC77AF1EE10FAF6DCDFED73
:1075E000547AB4EEE70AF1EE10FA62DDDFED4E7A7E
:1075F00037EEC00AF7EE007A9FED517A20EE004A8E
:10760000DFED4C6ADFED4C4A0023B0EE673A9FEDA8
:107610004B5AE4EE264AC4ED097A60EE043AA361BF
:10762000A8EE073A6361F0EE675A2362F8EE006A4B
:10763000E361A4EE245AE8EE475A87EE836AA3EE8C
:10764000850AB6EE007ABDEC028B77EEC07A26EEA4
:10765000077A66EE266A27EE865A67EE277A25EEC7
:10766000866A26EE807A84ED015AC4ED007A84EDB4
:10767000046AC4ED027A84ED037A10BDDFED317A3D
:10768000B4EEE70AF1EE10FAA9D5DFED266A9FED18
:107690002E7AF0EE407A30EE260AF4EEC77AF1EE5A
:1076A00010FAF6D4DFED227AB4EEE70AF1EE10FA22
:1076B0009CDCDFED267AB4EEE70AF1EE10FA99D5FC
:1076C000DFED207A37EEC00A94E79FED1E7AB4EE24
:1076D000C70AF1EE10FA7FF548AF9FED126ADFEDB1
:1076E0001A6AB0EE677A77EE867AB4EEE67AF1EE51
:1076F00010FAF6D49FED0E7AF4EEC77AF1EE10FA96
:107700003FF73BAF9FED117AF4EEC77AF1EE10FA36
:107710007FF537AF9FED0B7A77EE677A31E700BFE1
:1077200027D4D236DB0FC940DB0F4940E4CB1641EA
:10773000DB0FC93F92E741B99730083C15A82ABE34
:10774000F304353FDB0F49C0E4CB16C1DB0FC9BFE3
:10775000DFED2D0A08B54AF025FDDFED2C7AB4EEF9
:10776000E70AF1EE10FA28DDDFED276A9FED287AAF
:10777000F0EE407A30EE660AF4EEC77AF1EE10FAD7
:10778000F6DCDFED247AB4EEE70AF1EE10FA2FDD35
:10779000DFED1E7A37EEC00A20EE007A9FED1E6AFA
:1077A000DFED1E6ADFED1E7AE7EE066A20EE076A5D
:1077B000E6EE877AA6EE270A08BDDFED1A7AB4EE68
:1077C000E70AF1EE10FADCD5DFED0F6A9FED167ACD
:1077D000F0EE407A30EE260AF4EEC77AF1EE10FAB7
:1077E000F6D4DFED0C7AB4EEE70AF1EE10FACFDC56
:1077F000DFED0E7AB4EEE70AF1EE10FACCD5DFED4C
:10780000097A37EEC00AC7E7DB0FC940DB0F4940F2
:10781000E4CB1641DB0FC93F92E741B99730083CF2
:1078200015A82ABEDB0F49C0E4CB16C1DB0FC9BFC8
:10783000B0EEC07AF0EEE06AF0EE407AC6FE875A0B
:10784000F5EE405AF1EE10FA3BD086FEC75A85EEAF
:10785000256A9FED1D2A9FED1D3A9FED1D4ADFED24
:107860001D4ADFED1D2AF7EE005ADFED1C3A9FEDB1
:107870001C5AA6EE423AE6EE223AA6EE034AE6EE9D
:10788000235AE6EE044AA6EE245A85EE250AF4EEC3
:10789000C76AF1EE10FA03D59FED127A37EE400A6F
:1078A000F5EEC00AF1EE10FA03D59FED0F7A37EE30
:1078B000400AF5EEC07AF1EE10FA48BFB1EE400A88
:1078C00070479FED070AE2E739094E3DE3B59E3E5A
:1078D00088FA163E45FE7F3F99FB243F69A2163E7B
:1078E000A7DFA834DB0FC93FDB0F49402DE9F04F7C
:1078F000884689B01E461178531C0393002900F076
:107900001681002514460746A94609E03846013588
:10791000C047039C621C21780392002900F08F80ED
:107920002529F3D16078A31C3028CDE9033923D071
:10793000A0F130034FF0000ADBB2092B26D96C28E6
:107940002AD078287FD8572878D9A0F15803202B3F
:1079500079D8DFE803F0BD78787878787878787827
:107960007882AF787878787878787878AA78787824
:10797000789E788A7878BD00E31CA0784FF0010AE1
:107980000393A0F13003DBB2092BD8D804AA03A9D2
:1079900040F058FF6C28D4D1039B1A785C1C782ADD
:1079A0000394B7D8572A40F28E80A2F15803202BB7
:1079B000B0D801A151F823F0EF7A04081579040832
:1079C000157904081579040815790408157904084F
:1079D000157904081579040815790408157904083F
:1079E000157904085D7A04080B7B040815790408EE
:1079F000157904081579040815790408157904081F
:107A0000157904081579040815790408157904080E
:107A1000AD7A040815790408157904081579040865
:107A200015790408957A0408157904081B7B040865
:107A30001579040815790408EF7A040828B928464E
:107A400009B0BDE8F08F039C64E72528FBD1039CB7
:107A5000252138460135C0475CE7039C56F8041BD6
:107A600038460135C9B2C04754E70DF1140B002266
:107A70000A2156F8040B5B46039CFFF7DDF85346DA
:107A8000049A41463846CDF800B0FFF76DF805443A
:107A900040E7039C56F8040B0023049A41460090EB
:107AA0003846FFF761F8054434E7039C56F8043B79
:107AB0001D602FE70DF1140B56F8040B039C59467B
:107AC000FFF7FEF8DBE7002AB9D0252AC0D021E76E
:107AD000A0F158020DF1140B102156F8040BB2FA64
:107AE00082F25B465209FFF7A7F8039CC7E7A2F1B1
:107AF00058020DF1140B102156F8040BB2FA82F261
:107B00005B465209FFF798F8B9E70DF1140B56F8E8
:107B1000040B5946FFF7D4F8B1E70DF1140B00221E
:107B20000A2156F8040B5B46FFF786F8A7E70D46D7
:107B300085E7F8B5104C07460D461646A06DA0B176
:107B40000E49FFF729FB3946A06DFFF725FB0C49CD
:107B5000A06DFFF721FB0B4933462A46A06DFFF7C6
:107B6000C5FE0949A06DFFF717FB94F85C3013B10F
:107B7000012384F85D30F8BD98530024A31F0A0840
:107B8000C7370A0895710408B01F0A080EB400B57B
:107B900084B0084905AB019001A853F8042B039366
:107BA000FFF7A4FE0022019B1A7004B05DF804EBFD
:107BB00003B07047E56B0408F7B5114E0746002384
:107BC0000C46304615460F495E3600F85E3F04EB22
:107BD00045050D4B002F18BF19460C4F4BF052F8BE
:107BE000AC4202D10A4803B0F0BD394634F8022B4A
:107BF0006846FFF7CBFF694630464BF043F8EFE7A6
:107C000098530024BD1F0A08B41F0A08C61F0A089B
:107C1000F6530024F7B500230B4E044600EB410554
:107C20000A4F06F88F3FAC4202D1094803B0F0BDBD
:107C3000394634F8022B6846FFF7A8FF69463046FC
:107C40004BF020F8EFE700BF985300246A200A08A1
:107C500027540024F8B54E1E054601F11F04054FB8
:107C600016F8012F284639460235FFF78FFFA64246
:107C7000F6D1F8BDCB1F0A0802460846531C05D1B1
:107C8000034B1A681B790A600B71704701497DE745
:107C9000091F0A086B200A0810B50131144609F0C3
:107CA000A1FF28B9054B1A681B792260237110BD0A
:107CB000C27920460249BDE8104067E7091F0A085B
:107CC0006A1F0A0803685A1C02601970090A0368CF
:107CD0005A1C02601970704702681346511C0160FB
:107CE00013F802CB0360D31C5178036093781B0414
:107CF00043EA0123111D43EA0C030160D07843EAF3
:107D000000607047A0F13003092B07D920F0200054
:107D1000413819288CBF002001207047012070478E
:107D2000303809288CBF00200120704741381928BD
:107D30008CBF002001207047613819288CBF0020BB
:107D40000120704720280BD0092809D00A2807D025
:107D50000D2805D00B3801288CBF0020012070476A
:107D600001207047A0F14103192B98BF20307047C4
:107D7000A0F16103192B98BF2038704702B38446E5
:107D800010B5841803E0981A15D1A44514D01CF836
:107D9000013BA3F14100192811F8010BA0F1410E9C
:107DA00098BF203300F12002BEF1190FEBD91B1A46
:107DB00004D10028E9D110BD002010BD184610BD27
:107DC0001046704770B5044608460D4648F020FF3F
:107DD000064602E014F8013F43B1324629462046E8
:107DE000FFF7CCFF0028F5D1204670BD1C46204689
:107DF00070BD00BF2DE9F043064686469EF800C0E0
:107E000074460EF1010EBCF1200FF7D0BCF1090F42
:107E1000F4D0BCF10A0FACF10B00EFD0ACF10D05C2
:107E2000B5FA85F56D09002DE8D10128E6D9BCF138
:107E30002B0F3DD0BCF12D0F39D0102A3ED04FF082
:107E4000FF3E9046BEFBF2FE02FB0EF7FF43FFB281
:107E5000002014F801CBBCF1390F4CF02009ACF133
:107E6000300C0DD85FFA8CFC944510DA704526462C
:107E700002D819D1674517D21D404FF0FF30E8E70F
:107E8000A9F1570CB9F1600F5FFA8CFCECD801B185
:107E90000E6003F00103D5B9002803DA002B18BFE8
:107EA0006FF00040BDE8F08300FB08C0D1E701257A
:107EB000102A94F801C004F10104C0D1BCF1300FC4
:107EC00010D06FF0704E0F274FF01008C0E7B0F1E0
:107ED000004F04D91BB14FF00040BDE8F083404291
:107EE000BDE8F08360786FF0704E0F274FF01008F8
:107EF000A0F14106192E04F1010698BF2030782820
:107F00000CBF02343446A3E773B50E46104905464C
:107F1000FEF76EFE18B93070012002B070BD2C78EB
:107F2000602C8CBF613C413C082C0FD801350123EB
:107F30000A2201A92846FFF75DFF019BAB4205D04D
:107F40000F2803D8013440EA0410E4E70020E4E7F6
:107F5000091F0A0801230A2200214BE770B50D46CC
:107F60001446FFF782F90646A0B1FFF7F3FF40F68B
:107F7000340319229842A8BF1846B0F5617FB8BFF4
:107F80004FF46170A0F56173B3FBF2F32B702378AB
:107F9000013323703046FFF768F90646A0B1FFF7BA
:107FA000D9FF40F6340319229842A8BF1846B0F50D
:107FB000617FB8BF4FF46170A0F56173B3FBF2F35A
:107FC0006B70237801332370304670BD2DE9F0418A
:107FD00016461F46404D0446394630464FF47A72E5
:107FE000002349F073FA3D4B05443D4F3D4E83FB62
:107FF0000510E9172844C1EB601183FB0103C81782
:108000000B44C0EB631087FB003CC317C3EBAC030E
:1080100086FB03764FEAE37ECEEBE61EC1EB01164C
:10802000A5EB860CC0EB00154FEA8E0684F806C05F
:10803000A1EB8501617103EB4301A0EBC10040F2AC
:10804000B55101FB1E332071B3F5896F33DA40F26D
:10805000DA218B4237DCB3F5B77F234FB4BF4FF043
:10806000000E4FF0010E0EEB4E0175464FEA4E0822
:1080700007EBC101C88A08EB0E0C0B2107EBCC0CF7
:108080000CF1160C01E03CF8020D984210DD0139AC
:10809000F9D1F044012137F8380006F5FA6E0133C2
:1080A000A17075441B1A22812580E370BDE8F08120
:1080B0000131C9B2F1E7032540F296500A4F4FF063
:1080C0000608AE46D7E7022540F22940064F4FF09A
:1080D0000408AE46CFE700BF80BC92C78988888875
:1080E000ABAAAA2A73B06D16AC4209080D4B10B5A5
:1080F000D3E9004354EA03020AD10146002340F2C7
:10810000011218460B80C1F802208B710B8110BD43
:10811000054A1268121943F10003FFF757FF0120C7
:1081200010BD00BF482F0024B81D00242DE9F041E8
:108130000446154608469442B4FBF2F607D205FB06
:108140001644134B1B5D00F8013BBDE8F0819642DD
:10815000B6FBF2F70CD20E4B05FB176705FB164476
:10816000DA5D1B5D00F8012B00F8013BBDE8F081F2
:10817000BA42B7FBF2F807D905FB1878044B13F89D
:10818000082000F8012BE7E74046FFF7CFFFF3E7B1
:108190002CB1090830B56D4C83B0B4F8E434B3F5B4
:1081A0007A7F03D94FF47A73A4F8E434B4F8E63450
:1081B000B3F57A7F03D94FF47A73A4F8E634B4F8B0
:1081C000E814B1F57A7F04D94FF47A731946A4F80C
:1081D000E834B4F8EA04B0F57A7F03D900231846EE
:1081E000A4F8EA34B4F8EC34B3F57A7F4AD94FF402
:1081F0007A73B4F8EE249A42A4F8EC3447D90023F9
:108200008842A4F8EE3480F08B80B4F8FA24B4F8F5
:10821000FC349A4202D90023A4F8FA344C4B1B8850
:10822000EBB14C4DAA78062A4ED9297900297AD18A
:108230009FED497A94F8042507EE903AAB7906EE63
:10824000902AF8EEE77AB8EEE66AC6EE276A0BB136
:1082500037EE077AB4EEE67AF1EE10FA42DC627994
:10826000032A23D83D4B03EB42132279C4F80C3583
:10827000032A14D8EA213A4B02FB0133C4F8103523
:1082800003B030BDB4F8EE24B2F57A7F16D8884238
:1082900010D29A42B9D30023A4F8EC34B5E70022F7
:1082A0002F4B2271C4F8103503B030BD00222B4B88
:1082B0006271DAE70021A4F8E814EAE700228842B4
:1082C000A4F8EE24E5D3F5E7264901EB820191ED10
:1082D000187A29790029ADD0531F032BBFD9002A62
:1082E000BDD025E067EE877ABCEEE77A8DED017AA6
:1082F0009DF8043007EE103AB8EEC77AF4EEC77A6C
:10830000F1EE10FA01DD0133DBB2EBB1102BA8BFA7
:108310001023DBB2934238BF134684F804359EE73E
:10832000A4F8E83471E7053A032A98D99FED0A7A50
:10833000B7EE000A80EE070A49F066FF2B888342F9
:1083400028BF03462B808AE70123E2E798530024E5
:10835000481C00201C2A00246F12033850540024AB
:10836000D0540024AC4209082DE9F04F9C4E83B054
:1083700096F8143500AFA3F11702022A00F2BC826E
:10838000984B7B6096F824350024DFF874A23B609C
:10839000954B03F178099846D8F800B01BF0010519
:1083A00040F08B8298F90410142911D058464AF0F5
:1083B00011FE1BF4003F00F07382012808D008284A
:1083C00006DC002D00F07C821BEA0A0F40F06B8275
:1083D0008549864839F0E2FC0023022086F8CC3536
:1083E00013F0D0F996F8D435D6F8D095022B00F0DA
:1083F0000C83002800F068837D4B4FF47A7C96F85C
:1084000031A6002503F56A7E4FF0640B33F8082C83
:10841000B2F57A7FB3F8462088BF23F808CCB2F5CE
:108420007A7F33F8062C88BFA3F846C0B2F57A7F6E
:1084300033F8042C88BF23F806CCB2F57A7F02D932
:10844000002223F8045C33F8061C9142B3F85A105A
:10845000B3F85C2098BF23F8065C914293F86B2038
:1084600003F1650102F1FF3288BFA3F85A50632A75
:1084700093F86C2002F1010288BF83F86BB0D2B28E
:10848000092A4FF0000288BF83F86C5013F83200BD
:10849000013211F8014F844238BF0D70032AF5D123
:1084A000BAF1010F03F1EA0318BF03F8645C9E45BB
:1084B000ACD1DFF850A19AF80230042B00F0E28230
:1084C0002BB9BAF80030B3F5F07F00F22782FFF73E
:1084D00061FE96F84B36092B1AD0B3FA83F2520993
:1084E000B3B1013BA6F84C265A0003F00303C3EBDB
:1084F000031302F00802C3EB03139B00A6F85036E7
:108500009300A3EB9203C3EB03139B00A6F84E3634
:10851000B6F85A26B6F858361343B6F85C26134315
:108520001BB213B10123A6F85E36324B09EA0303EE
:10853000002B00F0D68219F0010F40F09E8219F452
:10854000804F40F0F08119F0080F00F058822A4A5D
:10855000D6F8243609EA02091340C6F8D095C6F8C1
:10856000243619F4004300F02D82002386F82B35C1
:1085700086F83B3519F4805F00F02F8296F86B3651
:10858000012B02D9012386F86B36DFF870904B4639
:1085900009F1780402E006339C420CD01A780A2ACA
:1085A000F9D19978DA78914202D35A79002AF2D037
:1085B0000A201DF0D7F800234FF4806086F8CC35F0
:1085C00013F0E0F8002800F072820C4DAB469BF8E7
:1085D000051021B39BF80000F8B14B4617E000BF2F
:1085E00098530024AC420908E8580024A4830A08E0
:1085F000DA54002409600002FE9FFFFD085A00249F
:10860000BC0202001C2A002406339C4207D01A78C0
:108610008A42F9D15A79002AF6D01DF0A3F80BF15D
:10862000060B5C45D3D19AF80290B9F1080F00F01F
:10863000FA8196F8313696F8E124A3F10103032A72
:10864000B3FA83F34FEA531386F8E83696F83236D6
:10865000A3F10103B3FA83F34FEA531386F8EE361E
:10866000D6F82436C3F3C03186F8EB1602D90022BF
:1086700086F8E124BB4A03EA0201D6F8D0351A4055
:10868000B37CC6F82416C6F8D025002B00F0D9819B
:10869000B6F80437002B40F0E081D6F80837B3F580
:1086A000000F02D30023C6F80837D6F81037AE4AB9
:1086B0001A401AB140F20223C6F8103796F80C3768
:1086C000013B042B02D9012386F80C37A9F10509D7
:1086D000A64BB9F1030F93F8F48340F26981B8F126
:1086E000000F1CD000233B60DFF8A49206E0ABF142
:1086F000060BABEB0A0BD84540F21781CB4619F8B5
:10870000010F0028F3D009F091FA0028EFD0817909
:108710008B07ECD53B680122002B40F00B819AF8C7
:10872000063013B100238AF80630B6F81A3703F082
:108730000F02042A03D8C3F30313022B03D94FF407
:108740002063A6F81A37B6F81C3703F00F02042A84
:1087500003D8C3F30313022B03D940F60123A6F871
:108760001C3796F8891796F8952796F8883791421E
:1087700005D9002286F8892753B1A6F88C2796F8E8
:1087800094279A4204D2002386F88837A6F88C37BB
:1087900096F88A2796F87E389A4202D9002386F8FE
:1087A0008A37DFF8F0C10CF1800B6346796813F863
:1087B000032D02EB42020A4492F85CA192F85D910B
:1087C00092F85EE113F8010F99795045DA78A8BF65
:1087D00050464945A8BF494672451870A8BF724621
:1087E00063459971DA70EDD103F1200CDC45DCD1E1
:1087F000D6F84825002A00F03A810020012102E045
:108800000635AC420ED02B782B2BF9D16B78043384
:1088100001FA03F31342F3D0063522EA03020120E2
:10882000AC42F0D108B1C6F84825514C6D4604F170
:108830000808234602E0434500F08A8013F8012F20
:10884000072AF8D9002304F8013F0133082BFAD195
:10885000B6F82A26AD46B6F828369A4202D3454BDA
:10886000C6F82836444BFF22444C03F1780086F8C2
:10887000B02813F9082C142A05D053F80C1C34EA3C
:10888000010100F0FC800C339842F2D13C4B5A7944
:10889000022A01D100225A710C37BD46BDE8F08F83
:1088A00001283FF78CAD08F10C08C1457FF474AD89
:1088B000013C022C7FF690AD8AE50134E4B275E507
:1088C0001BF0400F3FF484AD1BF4057F09D03B68DB
:1088D0000F2BE8D0012BE6D0991E0529E3D9102BE8
:1088E000E1D0284931EA0B017FF472AD08F10C08A0
:1088F000C1457FF451ADDBE7234A02EBC3037A6045
:1089000093F87C20002A3FF43DADD3F88030002B53
:108910007FF438AD172386F8143533E54FF4F07340
:10892000AAF80030D3E5194A12E63B680022002B72
:108930003FF4F5AE9AF81130002B7FF4F6AE9AF8BA
:108940000530012B3FF4EBAE002A7FF4E8AEECE6F5
:1089500088B02022FF21E94648464AF08BF9044AB4
:108960001FE000BF9CD74518FDFDFFFF481C0020FD
:108970002E2A0024AE014A01F4580024010002000E
:10898000582C002440000200AC420908F6DFFFFD2D
:10899000232A002455540024424549F823303FF44B
:1089A00057AF12F8013F59F823100131F4D049E7CD
:1089B00000238AF80430B8F1000F00F09080012302
:1089C0003B6091E696F82B25002A3FF4D3AD19F4CD
:1089D000805F86F83B357FF4D1AD19F0800F3FF40E
:1089E000CDAD96F81425182A04D8424BD340DA07A7
:1089F0003FF5C4ADDFF80C9109F17804DBE519F41B
:108A0000005F3FF4AEAD3C4AA2E500283FF4F4AC71
:108A100090F90440FF2500E00572204610F030FA7E
:108A20000028F9D1E8E49AF80630002B3FF401AEB3
:108A30009AF81130012B7FF4FCAD02238AF8113033
:108A4000F7E52E4B1A430B43C6F82436B6F8043725
:108A5000C6F8D025002B3FF420AE96F8000709F0A9
:108A6000E5F800287FF419AEA6F8040715E62B20D8
:108A70001CF078FED6F84825BFE6214A68E586F85E
:108A8000B02803E7D6F8243629F4805923F480531C
:108A9000C6F8D095C6F82436BAF82030B3F57A7FF8
:108AA000BFF415AD4FF47A73AAF820300FE5D6F86D
:108AB000D03523F00063C6F8D035D6F8243623F03D
:108AC0000063C6F8243680E5D6F8243629F08009FC
:108AD00023F08003C6F8D095C6F824368CE44246CD
:108AE00028E7D6F8243649F0080943F00803C6F809
:108AF00024362CE500410001F6BFFFFD000405000F
:108B0000F79FFFFD085A00242DE9F04F724E83B005
:108B1000724BD6F8C428DFF8E08102F2DC524345FC
:108B2000C6F8C42880F0D480DFF8D09101229B469B
:108B30006B4D09F102070192B9F80210002900F00B
:108B4000B2807A18AA4280F0AE80052940F2AB804C
:108B5000BBF800003C46C0F30B000BE01188144644
:108B60000A44002900F09F80AA4280F09C800529D9
:108B700040F2998061888142F0D161798B07EDD113
:108B800023885846DBF8081094F804A0009339F0C5
:108B900005F9BBF80010BAEB113F00F08A80002302
:108BA0000193BBF804100BF11C0B5BF8140CC1F320
:108BB0000B015BF8044C3FF0DDFAC3452060BBD3EA
:108BC000D6F8D035474CC6F82436FFF7CDFB3379BD
:108BD000EA22454D03FB0242A4F18003C6F81025AA
:108BE000727903EB4213C6F80C351BF063F84FF0B3
:108BF000FF33D6F810056B6023F0AEFD1CF0F8FDD6
:108C000004F5A76304F5B66102E0063399425AD031
:108C10001A78002AF9D19C78D878844202D35879FE
:108C20000028F2D096F8683664212A7203EB830399
:108C3000B6F86C2603EB830301FB02F22B499B0081
:108C4000642AB8BF6422642BC6F8C028B8BF642366
:108C5000C6F8D8280022C6F8BC3886F8DC2886F882
:108C6000DE28A1F51A72224BC3F8742500220023D6
:108C7000C1E90223C1E9042324F004FFB6F8E008A7
:108C800096F8E2181EF09CFC2FF068F815F06CFBCB
:108C9000184B012201981B6886F8DD28C6F8C438F5
:108CA00003B0BDE8F08FDBF80810584639F076F8CD
:108CB00075E7009BA11D58469A1F39F0A5F80028BA
:108CC0007FF46FAF6BE7F27C003A18BF0122A9E78F
:108CD0000123019374E700BF98530024FC820A0823
:108CE00000000408D05400248C040024585C0024A4
:108CF000481C0020B81D0024148B0A08000002083C
:108D0000114B0122032810B5044683F87C2505D9B0
:108D1000601CBDE81040C0B20AF070BD0B4BEA22E7
:108D200003F59C701C7104FB0200C3F8100523F0CE
:108D300013FD21F0B0F921F091FA601CBDE810405C
:108D4000C0B20AF05BBD00BF481C0020985300244D
:108D5000054B0121D3F8E82883F8E41842F4001207
:108D6000C3F8E828704700BF9853002470B5046822
:108D700086B005460E46C4F310033BBB01220393A5
:108D8000CDE901332023CDE9042304F17843B3F581
:108D9000801F19D3A4F10163B3F5801F10D2A4F58D
:108DA0008013022203F17843694601A802925B0C0A
:108DB00003933AF071F948B14FF0FF3006B070BD3F
:108DC0000520FCF755FBFBE72346EBE73146204641
:108DD0003FF0A0FF18B92B6820332B60EEE76FF04F
:108DE0000200EBE72DE9F0416A4E90B03378B12BE9
:108DF0007ED1FEF775F880F00104E4B2664B04F012
:108E00000104664DB3F86B31654FADF80030BD42DB
:108E100070D3002C00F0BC802822002106A849F065
:108E200029FF604B04969B1B05935F4BDA68D407C0
:108E300070D45D4BD3F80C21D00774D44FF48073F9
:108E40000222694604A8ADF83C3047F0C3F902227B
:108E500069464FF6FF70514DFDF768FE4FF0000870
:108E60000446BD4269D30025022201A904A8ADF839
:108E7000045047F0AFF9022201A92046FDF756FE43
:108E800040BA022202A9C043ADF8080004A847F086
:108E9000A1F90E9888B106ABC0F12002294618440A
:108EA00049F0E8FE9DF93C0018B906A904A8FFF7AF
:108EB0005DFF00238DF83C000E939DF83D307BB1A3
:108EC000394BDA6842F00102DA60DA68D20707D576
:108ED000D3F80C2142F00102C3F80C21D3F80C3175
:108EE0009DF93C00B0FA80F0400910B0BDE8F08177
:108EF000012483E7AB691C3535F8181CD3F80080D2
:108F000055F8140CC1F30B013FF034F9804518BF3C
:108F100001247CE7254A5A6002F188325A60DB68F6
:108F2000D90786D58AE7214AC3F8042102F188329D
:108F3000C3F80421D3F80C3180E7AE8802A904A855
:108F40008DF80D80C6F30B061C35B31DADF8083047
:108F500035F81C3CC3F30B021B0BADF80A200622AC
:108F60008DF80C3047F036F9062202A92046FDF7AD
:108F7000DDFD044655F8141C324604A847F02AF9D2
:108F8000204655F8141C3246FDF7D0FD044668E72C
:108F90000120AAE700000208AC420908FC820A0886
:108FA000148B0A08000004080020005223016745C2
:108FB00038B50324134DFFF7D7F9FFF713FF58B166
:108FC0002B78B12B08D1FDF78BFF013C17D040B9AE
:108FD000FFF708FF0028F3D1013CEED10520FCF794
:108FE00047FA09490022094B0120096883F8EC2857
:108FF00083F8DD08C3F8C41883F8ED2838BD0028CD
:10900000EFD1EBE700000208B81D002498530024BC
:1090100010B5074A0124074B82F87C459C74FFF782
:10902000C7FFFFF771FD2046BDE810400AF0E6BB20
:10903000481C00209853002490F89230B7EE007A34
:10904000DFED6A6A014607EE903A90F89630684A7A
:10905000B0EE476A05EE103A90F89430F8EEE77AF1
:1090600004EE903A90F89530B8EEC55A05EE903A75
:1090700090F8983067EEA67A04EE103A25EE265A5C
:10908000F8EEE44AF8EEE55AB8EEC44A25EE275A5F
:1090900064EEA64A65EEA65A24EE264A64EE854A98
:1090A00065EEA75A24EE274AB0EE473AF0B590F89D
:1090B000917000F16F0602F118050024137807EE95
:1090C000903AF8EEE77A67EE857A67EE867AFDEEFB
:1090D000E77A17EE903AFA2BA8BFFA2323EAE37354
:1090E0000B72537807EE903AF8EEE77A67EEA47ABF
:1090F00067EE867AFDEEE77A17EE903AFA2BA8BF74
:10910000FA2323EAE3734B72937803EE903AF8EE76
:10911000E33A63EEA57A67EE877AFDEEE77A17EE1B
:10912000903AFA2BA8BFFA2323EAE3738B72938851
:1091300007EE903AF8EEE77A67EE847A67EE867A81
:10914000FDEEE77A17EE903AD5ED007AB3F57A7F27
:10915000F8EEE77AA8BF4FF47A7323EAE3738B81C2
:109160002B68002B3FDD90F89730B0EE436A02EE9B
:10917000903AF8EEE22AA2EEE66A63EE863A83EED1
:10918000A76AA2EEA66A65EEA77A013467EE877A2F
:1091900067EE867AFDEEE77A17EE903AFA2BA8BFD3
:1091A000FA23BC4223EAE37306F8013F00DDF0BD79
:1091B000012C13D190F8933007EE103A90F89B30C1
:1091C00006EE103AB8EEC77AB8EEC66A27EE267AEF
:1091D00026EE266A0435083208316FE7B7EE007ACA
:1091E000B0EE476AF6E7B7EE006ACCE70AD7233C51
:1091F0008048090890F899306BB3B0F864308BB1AF
:1092000090F89A20642102EB8203C3EB0313B3FBB3
:10921000F1F3A0F86430962312FB03F3B3FBF1F3F0
:10922000A0F8663043884BB190F89A30642203EB83
:109230008303C3EB0313B3FBF2F34380B0F8503066
:109240004BB1962290F89A3013FB02F36422B3FBE1
:10925000F2F3A0F85030704790F821304BB3438BB5
:1092600083B190F82230FA22642113FB02F203EB5F
:109270008303B2FBF1F2B3F57A7F4283A8BF4FF4C8
:109280007A738383838843B1FA2290F8223013FBE8
:1092900002F36422B3FBF2F38380C3884BB190F8EE
:1092A000223003EB8303B3F57A7FA8BF4FF47A73C0
:1092B000C380704770B50B4C002504F56A7694F8AE
:1092C000913013B12046FFF7B7FE20460135FFF776
:1092D00091FF3046FFF7C0FF042D04F1EA04EED100
:1092E00070BD00BFD054002410B5064C4FF48072FE
:1092F000002104F61C6049F0BDFC0023C4F81C3FAB
:1093000010BD00BF98530024034BD3F8200F08B1C1
:1093100007F058BB704700BF9853002408B50B46B0
:1093200005490246D1F8200F28B10449FEF7DEFABC
:10933000BDE80840E8E708BD98530024957104088B
:10934000024B0146D3F8200FFDF726BF98530024A7
:109350000048F5E7B12B0A080CB4C30607B500D5E1
:1093600061B905A904980191FFF7D8FFFFF7F0FF55
:10937000012003B05DF804EB02B070470020F8E76D
:1093800008B5FFF7DDFFBDE80840E1E710B504468A
:109390000348FFF7D5FF2046BDE81040F0E700BFC7
:1093A000D01F0A0810B508460749FDF721FC002820
:1093B00015BF0124002405480548FFF7E7FF2046B4
:1093C000BDE8104006F00EBCD51F0A08DE1F0A08D3
:1093D00005200A08034B0146D3F8200F08B107F017
:1093E000DDBA7047985300240CB407B510F0200084
:1093F0000BD079B92320FFF7EDFF05A9049801915F
:10940000FFF78CFFFFF7A4FF012003B05DF804EB2A
:1094100002B070470020F8E70FB407B504A951F86F
:10942000040B0191FFF77AFF03B05DF804EB04B081
:109430007047194B1B682DE9F04153B30025174FB6
:10944000DFF864801648FFF79BFFFFF75DFFFCF72E
:109450006DFDFCF7ABFD044640B1132009F036FC6E
:10946000FFF776FF0F48BDE8F04189E73B78012B15
:10947000F3D040466E1CFFF7CFFF792D02D1264670
:10948000FFF766FFFFF740FF64203546FBF7DEFE7F
:10949000DFE7BDE8F08100BF801D0024562C0024CA
:1094A00021200A083B200A08F9390A0838B50B4D73
:1094B0000C4605EBC00595F9F80507F00DFC0146D3
:1094C0000748FFF7A9FF95F8FE352BB1611C054849
:1094D000C9B2BDE838409FE738BD00BFAC420908BB
:1094E00084370A086A200A080FB407B504A951F89E
:1094F000040B0191FFF712FFFFF72AFF03B05DF89D
:1095000004EB04B070472DE9F041037903F0E00269
:10951000402A4AD009D82ABB03F00703052B1CD8E0
:10952000DFE803F0161B161B090F602A44D0802ABF
:109530003ED0BDE8F081D0F805102148BDE8F041EB
:10954000D2E7D0F8052051421E48BDE8F041CBE7F4
:10955000B0F80720B0F80510F6E7B0F90720B0F929
:109560000510F1E746790024174D184805EBC605AC
:10957000FFF7E6FE012395F8D476A74202D8BDE8AE
:10958000F041E5E6D5F8D0664FEA840856F8242085
:109590004AB113B90E48FFF7D3FE56F808100D482C
:1095A000FFF73AFF00230134E7E741790A48C5E7AE
:1095B000827941790948C8E70948BDE8F04193E755
:1095C00041200A0857200A08AC4209086E200A0800
:1095D000B8220A0884370A087F200A0890200A085F
:1095E000A7200A082DE9F04385B0224EFCF78EFC37
:1095F0000269838900250188044602928268DFF8A7
:10960000888001924288DFF884901B4F0092426864
:109610001A48FFF769FF15B91948FFF7B1FED8F8E6
:1096200000309D4212DA3378052B20D809EB8303F2
:10963000D3F88828B3882946013538460093063682
:1096400036F8043CFFF750FF062DE4D13FF022F935
:109650004288838864689B1A03FB0444FCF7F2FC8D
:1096600002460848214605B0BDE8F0433CE7002229
:10967000E0E700BFBC62002429210A08BF200A08D5
:109680001D210A0838210A084C2C0024AC42090884
:109690000249034801F500610EC925E700E0F11F0A
:1096A00055210A0870B50022124C134D134E94F840
:1096B000033503F0010302B170BD002BFCD0012182
:1096C0002846FFF711FF752024F0F0FC01463046D4
:1096D000FFF70AFF1A2024F0E9FC01460848FFF7CB
:1096E00003FF1B2024F0E2FC01460648FFF7FCFEC6
:1096F0000122DCE79853002469210A0875210A0831
:1097000088210A089B210A08B64B42F201011A6817
:10971000B1EB124F4FEA12432DE9F04790B000F041
:109720005C8142F20302934200F0598141F203024C
:10973000991A4B424B41AC4A4FF00008AB4D1168AF
:10974000464605EBC303AA4AAA4CAB48AB4FB1FB54
:10975000F2F2D3F8A418FFF75FFEB4F8482F4FF4E5
:109760007A730A20B2FBF3F103FB1122B4F94A3FEA
:1097700092B2B2FBF0F2A248FFF7B6FEA14AA249AC
:10978000A248FFF749FEFFF7E3FDA17CA04A05EBE5
:109790008101A04BA048D31AD1F8C0182288FFF746
:1097A000A3FEFFF7D5FD9D48FFF7CAFD94F84C1FB7
:1097B0009B48FFF731FE9B48FFF7C2FDB4F84E2FE0
:1097C00094F8501F92B29848FFF726FEFFF7C0FDAD
:1097D00096499748FFF720FEDFF8C89294F8FF34C7
:1097E00003F00103B8F1000F00F06081002E40F09B
:1097F00091819048FFF7C4FD8F4F0126D4F8548F14
:10980000DFF8A49207F1180A0123B34013EA080F06
:1098100015D019F8062057F826305AF8261053F8B4
:1098200022208648FFF7F8FD012E06D1734B93F8EE
:10983000A91511B18248FFF7EFFDFFF789FD013649
:10984000062EE1D17F48FFF77BFDD4F824361B06B6
:1098500040F1948194F8743F032B8CBF7A487B4885
:10986000FFF76EFD94F8D435022B40F0568178480E
:10987000FFF766FD94F8743F042B00F2768175487B
:10988000FFF75EFD94F8843F002B00F0758105EB37
:10989000C303D3F89C197048FFF7BEFDFFF758FDCE
:1098A00094F86B3DD4F86C6D05EB83036B48D3F8EB
:1098B000D019FFF7B1FD26B1327A717A6848FFF707
:1098C000ABFDFFF745FDFCF721FB016921B1826883
:1098D0006448120DFFF708FEFFF73AFD624963483E
:1098E000FFF79AFD62496348FFF796FDFFF730FDE9
:1098F000FFF72EFD604B614819684FF47A73B1FB96
:10990000F3F1FFF789FD05A8FEF7F0FB38B105A9D3
:1099100008A847F02FF808A95948FFF77DFDFFF781
:1099200017FD584BD3F81080B8F1000F00F02A81D2
:1099300007EE908ADFED546AB8EEE77AC6EE877AD2
:10994000FDEEE77A17EE903A504F97F8100630B1D7
:109950004F4A039392ED2B0A48F056FC039BD4F830
:10996000906F5EB107EE906ADFED476AF8EEE77A36
:1099700086EEA77AFDEEC77A17EE906A1F4AB2F814
:10998000F81542466429CDE90006A8BF6421414884
:10999000FFF7AAFDB7F8142664233F483F4EB2FBF9
:1099A000F3F103FB112297F8253605EB830592B2FC
:1099B000D5F8E4390125009397F82436FFF794FD94
:1099C0003748FFF7BDFCD4F8E848002C40F0DC80B5
:1099D000FFF7BEFC10B0BDE8F0870223ABE603231F
:1099E000A9E600BF0010005CA4030024AC420908F3
:1099F00040420F0098530024B6210A08481C00205A
:109A0000C8210A08F8FF012000080000EA210A081E
:109A10000000040800000208FC210A0813220A08BA
:109A200025220A082D220A082F220A0843220A08A2
:109A300048220A0867220A08D44B0908F2330A08A8
:109A40006C220A0870220A0876220A0882220A0872
:109A500092220A08343A0A08D6220A08F2220A0890
:109A6000FB220A0805230A0820230A0841230A08C2
:109A70004F230A08082B0A08B81D002459230A0896
:109A800073230A0898630024002474499064002416
:109A90008C04002486230A08CC230A08E2220A0840
:109AA000F1230A08B8220A0830050024002B3FF4ED
:109AB0009DAE16B14846FFF743FC01213A48FFF737
:109AC000ABFC94F8143A394805EB8303D3F8C81873
:109AD000FFF7A2FC97F8CE33DA0702D53448FFF738
:109AE0009BFC97F81831032B09D03248FFF794FC00
:109AF00097F81831012B02D12F48FFF78DFCFB6C32
:109B000001265B7BB046B3427FF668AE2B48FFF779
:109B100083FC61E6FFF71CFC6EE6022011F050FEAC
:109B2000064608B92648A3E690F904003DF034FB48
:109B300007462EF0FDF805EB80003946D0F858298D
:109B40002048FFF769FC94F8D735012B04D11E4853
:109B5000FFF7F6FB1D488BE6B3791D4805EB830341
:109B6000D3F85819FFF758FCF4E794F8D6350BB939
:109B7000184885E6184883E618498CE61848FFF728
:109B8000DFFB8BE64346DFE694FAA4F0B0FA80F000
:109B900005FA00F024EA000409F07EF80146304698
:109BA000FFF73AFC11E700BF4D220A08E2220A083B
:109BB00072370A0852220A085A220A085F220A0843
:109BC00098220A08A2220A08B2220A08B7220A0822
:109BD000212E0A08BB220A08CB220A08AE210A0855
:109BE000E6220A082DE9F04FDFF8748199B098F861
:109BF0000730002B00F0978050480025504EDFF8CA
:109C000064B1FFF7BDFB2F46DFF85C91DFF85CA184
:109C10000BA9E8B216F0BCFC9DF83430002B53D0F1
:109C2000139C54B107EE904A9FED460AF8EE677A0E
:109C300080EE270A48F0E8FA04460B9A294658466F
:109C4000FFF7EAFB109A002A6FD002FB04F04FF4F2
:109C50007A73B0FBF3F30993DDF848C0BCF1000F51
:109C600065D00CFB04F142F21073B1FBF3F1082D47
:109C700098F8073018BF7F18002B5AD017984FF468
:109C80007A7E0A23079015980690169805901198E9
:109C9000B0FBFEFECDF810E00998B1FBF3FE03FB2C
:109CA0001E11CDE902E10999B1FBF3F103FB1100AB
:109CB000BCFBF3F3CDE9001021465046FFF714FC3E
:109CC0000023B362C6E90D33013540361E2D9FD106
:109CD00098F8073023B31C4C4FF47A731B48D4F820
:109CE0002816D4F82C26B1FBF3F3D208D4F830169A
:109CF000FFF7FAFB0A22164897FBF2F102FB1172FA
:109D0000FFF7F2FB134B1B78432B06D1D4F8342614
:109D1000D4F838161048FFF7E7FB0023C4F83036B4
:109D200019B0BDE8F08F0D4867E7099294E76146E6
:109D30009DE721464846FFF7D7FBC1E707240A08FD
:109D4000206300248096184B90640024AE240A08F7
:109D5000CE240A08142B0024F2240A0865240A08D9
:109D6000985300246F240A0820370A087E240A0822
:109D7000234870B5FFF7E4FA224B93F81036002B16
:109D800038D0214B93ED2B0A48F03EFA01461F488C
:109D9000FFF7AAFB1E4C1F48FFF7D2FA1E4B94F8A0
:109DA0003D051E4A00280CBF10461846FFF7E8FA8A
:109DB00094F83D3513B31A4C1A48B4F88E16FFF7D1
:109DC0002BFB194E94F88C06184D00280CBF30461A
:109DD0002846FFF7D5FAB4F890161548FFF71CFB94
:109DE00094F88D0600280CBF30462846BDE8704028
:109DF000FFF7C6BA0F48FFF7C3FACBE770BD00BF45
:109E00002C250A08906400248C04002446250A08A6
:109E10009853002455250A08BC200A08643F0A0804
:109E2000481C002066250A0825250A081C250A0862
:109E30008D250A084B250A080EB403B503AA52F86B
:109E4000041B0192FDF775FE064BD3F8202F1AB9BB
:109E50000549986DFDF7A0F902B05DF804EB03B079
:109E6000704700BF98530024B12B0A082DE9F04732
:109E700098460B7981460F4603F0E0051646402DC3
:109E800032D10024634DDFF8A881DFF8B09116E0ED
:109E90003B7903F00703013B042B04D8DFE803F010
:109EA00014171A1D2100315D5A48FFF7B5FA7B7966
:109EB000013BA34202DD4846FFF742FA01347B79B9
:109EC000A342E5DCBDE8F08731572846EDE736F8D8
:109ED0001410FAE736F91410F7E756F82410404644
:109EE000E3E756F82410F0E703F00703052B57D8F3
:109EF000DFE803F0031F27292C3E3478602D55D06E
:109F00002CD8002D75D1B7F80550B7F80760214659
:109F10004048FFF781FAAC4239DBB44237DCB8F194
:109F2000000FCFD0324629463B48BDE8F047FFF747
:109F300073BA96F90040602D38D00FD8002D58D153
:109F400051E03488DAE7B6F90040F4E7D6F800A02B
:109F5000202D54464DD034D9602D27D0802DB1D13D
:109F600032782E4B2E48002A14BF3146194635E070
:109F7000202D34683DD0EFD821462648FFF74CFA13
:109F8000D7F80510A14202DB4B42A34221DDFFF7C7
:109F9000DFF923463A6848462249BDE8F0474BE7D7
:109FA000202D25D01ED9602DD8D100247B7944FAEC
:109FB00003F3DB07BDE8F0474CBF1B481B48FFF726
:109FC0002BBA51461A48FFF727FAD7F805108A45E9
:109FD000DDD8B8F1000F3FF475AF1648BDE8F04783
:109FE000FFF71ABA0024B7F90550B7F907608EE7F2
:109FF00000247A79104B03EBC20393F8D426A242D3
:10A00000C5DDD3F8D03653F82400BDE8F047FFF79C
:10A0100097B900BF6B200A08D41E0A08253B0A081E
:10A0200084370A08B3250A08BC200A08643F0A08D6
:10A0300054200A08AD250A08AC4209082D220A0856
:10A0400070B5164605460C460846FDF7B5F833468A
:10A05000024621462846BDE8704007E70EB403B526
:10A0600003AA52F8041B0192FDF763FD044B054956
:10A07000986DFDF791F802B05DF804EB03B07047FE
:10A0800098530024B12B0A080049E7E7CD250A08B8
:10A0900038B50C46054615492046FCF7A9FD30B9F0
:10A0A000FFF708F91248BDE83840FFF769B91149D0
:10A0B0002046FCF79DFDA0B90F4B83F8C90183F83A
:10A0C000D10183F8B30283F8BB0283F89D0383F8C0
:10A0D000A50383F8870483F88F0483F801050748F4
:10A0E000E1E72846BDE83840CEE700BFDC250A0896
:10A0F000E2250A08FD250A089853002405260A08C7
:10A100000049ABE721260A08F8B50C460646084682
:10A11000FDF720FF20210546204648F0C2FD0446F9
:10A1200018B93046BDE8F840EAE7114F0134114E46
:10A130003B7832789A4201D0FCF784F80E4B2046E7
:10A140001D6046F065FD012201462046FCF718F827
:10A150003B7832789A4201D0FCF774F8204646F0FA
:10A1600057FD2A4601460548BDE8F840FFF7BCB94F
:10A170007C1D0024572C0024781D002438260A0852
:10A180002DE9F0410D4688B006460846FDF7E2FE8F
:10A1900020210446284648F084FD20B9304608B006
:10A1A000BDE8F041ACE7FDF7D5FE22460546014685
:10A1B0000F48FFF799F985B1202D2A4669462046B8
:10A1C00028BF2022E846FCF785F800270646B7425C
:10A1D00008DBAD1B3444002EEDD1FFF7B9F808B011
:10A1E000BDE8F08118F8010B0137FFF7F3F8EEE74F
:10A1F0004E260A082DE9FF47074608460D4646F059
:10A2000007FD082846D105F1FF3801AE0735314674
:10A210004246B14612F8010FFDF7AAFD01F8010B05
:10A22000AA42F7D10023DFF880A08DF80C30A845B2
:10A2300018D11C49484623F07BFB1A4808231A49C9
:10A2400010F8012B013B11F8014B02F110026A4496
:10A2500002F80C4CF4D101A914488DF80C30FFF72A
:10A2600043F914E018F8010FFDF782FD044601469A
:10A2700006F8010B504648F014FD28B1214630463F
:10A2800048F00FFD0028D2D03846FFF7FDFE04B09D
:10A29000BDE8F0870028D0D0384604B0BDE8F047CC
:10A2A0002EE700BFB4580024A0C0090866260A089B
:10A2B00007B5009313460A460249FFF7CFFE03B0E5
:10A2C0005DF804FB6D260A0810B504460748FFF741
:10A2D00057F8FCF72FF820B10548BDE81040FFF70C
:10A2E0004FB820460349BDE81040B7E686260A0865
:10A2F00090260A0898260A08154BD3F8643A2DE9E7
:10A30000F041044688B0F3B11A6804A91846D56A2A
:10A310006A46A847064688B104AC6D460027DFF8B8
:10A320003C80013735F8022B34F8021B4046FFF71A
:10A33000DBF8BE42F5DC08B0BDE8F08105492046F7
:10A34000FFF78CFEF7E7044908B0BDE8F04185E669
:10A3500098530024B9260A08D1260A089F260A081D
:10A3600070B5054608460C4646F052FC024668B1F8
:10A370000D2804D12146084848F06CFD30B128462C
:10A38000054B064A0649BDE8704067E602490548A4
:10A39000BDE87040FFF7A8B8D8260A08E6260A08E4
:10A3A000F1260A081B270A0870B5054608460C4620
:10A3B00046F02EFC024668B1042804D12146084824
:10A3C00048F048FD30B12846054B064A0649BDE82D
:10A3D000704043E602490548BDE87040FFF784B885
:10A3E00029270A082E270A08F1260A083E270A0804
:10A3F0002DE9F04307469BB008460C4646F008FCA2
:10A4000006462022002101A848F034FC2EB3402E3D
:10A4100007D0402332463A4938461BB0BDE8F043E6
:10A420001CE601AD04F140084FF00009022221466C
:10A43000684648F021FD0023102209A968468DF8DE
:10A440000290FDF7D7FC099B0DF10202934223D144
:10A45000023405F8010BA045E8D109AC41220021E6
:10A46000284D204648F006FC002E3DD095F83C666D
:10A47000D6B1202205F23D6101A848F04FFD98B108
:10A4800005F23D612046FDF7E5FB23461E4A3846AE
:10A490001E49FFF7E3FD04E01A7838461C49FFF730
:10A4A000DDFD1BB0BDE8F0831A4B93F83430DBB907
:10A4B000D6B901AB184E1A46083603CAA24246F86E
:10A4C000080C46F8041C1346F5D101232046124916
:10A4D00085F85D36FDF7BEFB1048FEF757FF2146B5
:10A4E0000F48FFF701F8DCE795F85D361BB995F8E2
:10A4F0003C36002BF3D008492046FDF7ABFBEEE7D6
:10A5000051270A08906400248F270A08F1260A08B8
:10A5100073270A0898530024CD6A002499270A0853
:10A52000A8270A082DE9F74FDFF82081834608465F
:10A530000C4646F06DFBD8F8D075064628B10246A9
:10A5400033492046FDF71AFC80B9394631483CF0C2
:10A55000A9FD3149314821EA07013CF0A3FD30490A
:10A56000304803B0BDE8F04F3CF09CBD23782D2B64
:10A5700023D10134013E4FF0010A2B4B4FF000096B
:10A580004FF0FF3553F8041B51B13246204601937A
:10A59000FDF7F4FB0028019B0ABF4D460021012175
:10A5A00009F10109A1B9B9F11D0FEBD122461F49EB
:10A5B000584603B0BDE8F04F50E54FF0000ADCE725
:10A5C0003B431B49C8F8D0351A4B12E01A4913E037
:10A5D0000123114AAB401A40002AF7D007EA0302D0
:10A5E000BAF1000FECD027EA03031449C8F8D035BC
:10A5F000134B002A18BF1946124B134803EB85036F
:10A60000D3F8F82903B0BDE8F04FFEF76DBF00BFE7
:10A610006A240A08E0270A089CD74518EA270A088E
:10A620006328BAE7F6270A08A44C090804280A0890
:10A63000D8270A08D1270A08B5270A08C1270A0817
:10A64000C8270A08AC420908562E0A089853002465
:10A650002DE9F74F019008460E461746984646F0FA
:10A66000D7FA0446E8B93F4D3F48FEF7D5FE2046ED
:10A670000EF06EFB3B68184206D020460EF07AFBC7
:10A6800001462846FEF7C8FE0134172CEFD13B687F
:10A6900013B93648FEF754FE03B0BDE8F04FFEF79D
:10A6A00057BE024632493046FDF768FB0546A8B959
:10A6B0002C46304D3048FEF743FE20460EF048FB56
:10A6C00010EA080F06D020460EF054FB014628463B
:10A6D000FEF7A2FE0134182CEFD1DDE733782D2BE5
:10A6E00029D10136013C01254FF0000948F4000B47
:10A6F00048460EF03FFB2246824601463046FDF7B3
:10A700003DFB18BB48460EF023FB1BEA000F1DD093
:10A710009DB1B9F1170F02D03B6840EA0308174812
:10A72000C7F80080FEF70CFE5146124803B0BDE8A2
:10A73000F04FFEF7D9BE0025D6E7B9F1170F02D0CA
:10A740003D6825EA00050E483D60EBE709F1010987
:10A75000B9F1180FCCD132460A49019803B0BDE8CF
:10A76000F04F7BE4E1220A0815280A081F280A088E
:10A770006A240A08E2220A0826280A08C8270A08C2
:10A78000D8270A0804280A0840F20223004A5FE793
:10A79000A85A0024014B024A5AE700BFFFFF7F007E
:10A7A000A05A002410B5044623F036F920B92046FB
:10A7B0000449BDE8104051E40348BDE81040FEF7ED
:10A7C00093BE00BF31280A0840280A08064B10B57E
:10A7D0000446D3F860062DF023FA20B92046034939
:10A7E000BDE810403AE410BD906400244B280A08EC
:10A7F00070B5054608461646FDF7ACFB0D4B041E2A
:10A8000093F8F4230EDB944205DA21460A48FEF75A
:10A810006BFE204670BD2EB1FF2C03D10748FEF71A
:10A8200063FEF6E7013A064928464FF0FF34FFF78A
:10A8300015FCEEE7481C002061280A0872280A0867
:10A8400085280A082DE9F04F074691B082480E4648
:10A85000824DFEF749FE002381494024062285F8F7
:10A8600068363046012391F8F413C5F864D685F8AC
:10A87000694606F061F80A20FAF7E8FC95F86836B0
:10A880000C2BDAB240F2E4809DF80C60FE2E2CD046
:10A89000FF2E15BF0F24152400250125944240F0FA
:10A8A000D780611E6846C9B232F096FA04F14003BF
:10A8B0000DEB030414F8413C834240F0C4806A1E4F
:10A8C0009DF80D30012A12D903F01F075C0961378A
:10A8D0006448FEF735FD022D39D0013C042C34D8F4
:10A8E000DFE804F00B2D2F3331000225D6E79DF869
:10A8F0000E701E469DF80F40EAE75B486C464FF02D
:10A900000008DFF8BC91FEF73BFDDFF8B8A1DFF8E7
:10A91000B8B15648FEF714FD08F1010814F8011B00
:10A920004846FEF779FDB8F10C0F16D00AFB08F384
:10A93000B3F1553FF0D85846FEF702FDECE74C481E
:10A94000DCE74C48DAE74C48D8E74C48D6E7002328
:10A950000DF11F008DF83F30D0E7FEF7F9FC022D16
:10A960003AD064223B464648B6FBF2F102FB116244
:10A97000C9B2D2B2FEF7B8FD85F001035B42DBB28B
:10A98000012B59D83F4A404B9DF810103F480029F1
:10A990000CBF114619463E4EFEF7A6FD9DF811105C
:10A9A0003C4B3D4800290CBF31461946FEF79CFD43
:10A9B000022D41D19DF812403848FEF7C1FC8CB100
:10A9C000FF2C1FD00A233648B4FBF3F103FB1142DE
:10A9D000D2B2FEF789FD08E03A4631463148FEF72B
:10A9E00083FDCFE73046FEF7CBFC9DF813402E48A1
:10A9F000FEF7A6FC44B1FF2C21D021462B48FEF7E0
:10AA000073FD04E02A48EEE72148FEF7B9FC0DF19A
:10AA1000130500241E4E1F4FDFF8948015F8013FE8
:10AA20007BB1FF2B14BF3A464246214601342148F0
:10AA3000FEF75AFD042CF1D111B0BDE8F08F1C488F
:10AA4000E3E73246F1E71C493846FFF707FBF3E737
:10AA50001A48FEF795FCEFE7CB280A08906400241B
:10AA6000481C0020DC280A08E7280A080D290A08E3
:10AA7000EE280A08F6280A08FE280A08AE210A0865
:10AA80001F290A08B4280A08AB280A0856290A0808
:10AA9000BB280A08C8380A086D290A0874290A0858
:10AAA00088290A083B290A0890290A086B200A0805
:10AAB000BF280A08A0290A08AB290A08BB290A08E6
:10AAC000CB1F0A08ABAAAAAA253B0A082DE9F8431E
:10AAD00007460C46DFF8A490204646F099F8064653
:10AAE00060B91E4B1E4893F814251E4B03EB8203DE
:10AAF000D3F8681ABDE8F843FEF7F6BC02464946AB
:10AB00002046FDF73BF960B1DFF86080002558F87A
:10AB1000041BB1B9224638461349BDE8F843FFF794
:10AB20009DBA124C124D1348FEF70AFC54F8041B50
:10AB300019B12846FEF770FCF8E7BDE8F843FEF7C8
:10AB400007BC324620460135FDF718F90028DED152
:10AB5000024B094C83F81455BEE700BF98530024FC
:10AB6000C4290A08AC42090804280A08184D090833
:10AB7000E2220A0826280A08B32B0A086A240A08CF
:10AB800038B50D460446052219492846FDF7F6F862
:10AB900068B9184B93F85C2022B9012183F85D2035
:10ABA00083F85C101448BDE83840FEF7E9BB032287
:10ABB00012492846FDF7E2F8A0B90E4D95F85C3031
:10ABC00063B195F85D304BB10D492046FFF746FA69
:10ABD000002385F85C3085F85D3038BD0948FEF704
:10ABE000CFFBF5E720460849BDE83840FFF736BA05
:10ABF00026380A0898530024CE290A0871390A0811
:10AC0000E4290A081B2A0A082F2A0A0870B5194CD9
:10AC1000054694F85C307BB194F85D3063B1164919
:10AC2000FFF71CFA28461549FFF718FA002084F8A8
:10AC30005C0084F85D0070BD114B93F85D26B2B1E5
:10AC400093F83C269AB903F23D6203F26C6503F275
:10AC50005D661068083252F8041C2C46B24203C4E8
:10AC60002546F6D1012283F8A72607F0EFFD012043
:10AC7000E1E700BF98530024E4290A083E2A0A08A5
:10AC80009064002408B5034610460AB9002008BDA8
:10AC9000DB0601D50029FAD0FEF778FBF6E7F8B518
:10ACA0000D4E054696F8343093B9F8BD25B123888A
:10ACB000C3F30B039D4204D0A288D4E9020147F0FC
:10ACC0007BFF1C34BC42F1D3002386F83430ECE720
:10ACD000024C034FF6E700BF98530024FC820A0899
:10ACE000148B0A082DE9F04F164685B0334C1A46EE
:10ACF0004FF00009A246CDE9010100213046FFF7DF
:10AD0000C1FF06F0100300900393FEF7FDFA2379CC
:10AD1000029A03F01803934203D0002A44D1182B5F
:10AD200042D14FF00D0B0BFB09A3B3F8090037F02C
:10AD30001FF880462046FCF74EF90746D8E9022165
:10AD4000024401442046FCF7FFF880F0010105466B
:10AD5000009AC9B23046FFF795FF039B009003B1FC
:10AD600015BB0BFB09FBB3065AF80BB00ED56DB93A
:10AD700059461348FEF750FBD8F808202B462146C9
:10AD80003A440198FFF772F8FEF7E2FA59460D4887
:10AD9000FEF742FBD8F80C20002321463A440198E4
:10ADA000FFF764F8FEF7D4FA09F1010940F24923EC
:10ADB0000D349945A9D105B0BDE8F08FE05A0908D6
:10ADC0005C2A0A085D2A0A0820B10078B0FA80F0EF
:10ADD00040097047012070472DE9F74F814608462A
:10ADE000FFF7F2FF0E46054670B1002401A9204688
:10ADF00001343CF0E7F901464846FFF7EDFF122C1D
:10AE0000F4D103B0BDE8F08F0846FDF7A3F8C4B253
:10AE1000112C72D83D4D701CFCF727FA3C4E05EB07
:10AE200044088346670098F8A8A6B8B9AAF10201B9
:10AE30004B424B413D4495F8A826B25C002B55D0BF
:10AE400095F8A936192040F2EE2100FB03132146A4
:10AE5000304803B0BDE8F04FFEF746BB01783046FE
:10AE600047F01FFF80B1032C2B49A0EB060394BFD2
:10AE70000022012202EB42020A4452FA83F393F8C1
:10AE8000DCAABAF1030F05D1484603B0BDE8F04F84
:10AE9000FFF7FAB85846FCF7E8F9F0B1BAF1020F3B
:10AEA000F2D1FDF757F840F6CA0380B29842A8BF26
:10AEB000184640F2EE239842B8BF18461923A0F274
:10AEC000EE20B0FBF3F088F8A906AAF10202534283
:10AED0005341EA1982F8A8A6ACE7BAF1020FF4D1FF
:10AEE000484603B0BDE8F04FFFF70AB921460B48CA
:10AEF00003B0BDE8F04FFEF7F7BA11232A46084920
:10AF0000484603B0BDE8F04FFFF7D2B99064002483
:10AF1000B0C20908672A0A08AC420908772A0A0859
:10AF2000842A0A082DE9F04F0346A1B00846FFF72E
:10AF30004BFF054628B1184621B0BDE8F04FFFF79A
:10AF4000DFB8FF23DFF8C09207464FF0FF388DF8D7
:10AF50002830D9F860360B9093F83820ADF83000DF
:10AF60000D908DF838200F90ADF8400011930991A5
:10AF7000CDE90500934909A847F02CFE044618BB0B
:10AF800001460AAC904F0B0190481A57002310F964
:10AF9000016BB24240F0D2804E1C10463CF0FCF8EF
:10AFA000024631463846FEF79FFA022E4FF0010165
:10AFB000E9D19DF938A09DF92830534540F0C5806E
:10AFC0008348FEF791FA4DE02378002BD2D0032F6F
:10AFD000D4BF00260126062F00F2A980DFE807F083
:10AFE0000447509104475000042F10D0794920465F
:10AFF000FCF7E8FE58B14FF4806010F0E1FB002848
:10B0000000F0B58190F90400012306930AE072492B
:10B010002046FBF7EDFD70B9D9F8603693F938009A
:10B02000042F22D0119B119320AB03EB061606F8D8
:10B03000580C01379EE720463BF0A4FF0028EFDACA
:10B0400001230A2212A92046FCF7D4FE40B20028B0
:10B0500003DB129B1B78002BE2D02246711C5F4859
:10B06000FEF742FA21B0BDE8F08F0023DBE720466F
:10B07000FCF770FF20AB03EB061646F8540CD8E73C
:10B0800057492046FCF79EFEB0F1000A554920467C
:10B0900018BF4FF0010AFCF795FE08B14AF0020A0A
:10B0A0003301DFF868C1079320AB03EB0616BCE859
:10B0B0000F0006F850AC12AE0DF1480A0FC6BCE8FE
:10B0C0000F000FC6BCE80F000FC69CE8030086E81F
:10B0D00003000026B346DAF80010204647F008FFC8
:10B0E00010B19AF804301E430BF1010B0AF1080A63
:10B0F000BBF1070FEFD1079B80336B4403F84F6C14
:10B1000097E739492046FBF773FDA0B13749204640
:10B11000FBF76EFD00288CD02046FCF71BFF0328B0
:10B12000804686D901463248FEF7DEF99AE7224684
:10B130000821304894E7012305937AE701330A2B6D
:10B140007FF425AF01312C488AE70B9B1BB9AAF18C
:10B1500014025542554100235F1CE368002B62D165
:10B1600094F900B058460DF08BFED4F8049018B155
:10B170000668002E40F08B80B9F1000F237A14BFCF
:10B180004E464FF46146666023B91C48FEF7ACF9A1
:10B1900003232372627A2AB1394619480792FEF7CF
:10B1A000A3F9079A02925846237ACDE90063002357
:10B1B0001A46194610F079FBE06048BB3946114841
:10B1C000B2E700BFD31F0A080E2B0A08BB460908C6
:10B1D0002B2B0A08A72A0A08B22A0A08B62A0A0844
:10B1E000D12A0A08F5380A08D42A0A0821280A08A8
:10B1F000DA2A0A08F22A0A08192B0A08442B0A0834
:10B200005F2B0A087A2B0A0890640024904D0908E5
:10B2100058493346584A5948B9F1000F18BF0A46F1
:10B220003946FEF7F9F8022F04F110044FF001033C
:10B2300092D1119E0D9F4DB15148FEF7A1F8336890
:10B240001B6A1BB13A464F4930469847059B002B75
:10B2500050D04D49474BBAF1140F18BF19464B480F
:10B26000FEF742F9BAF1140F09D1059B002B43D028
:10B270003368DB691BB10022454930469847069B7D
:10B28000002B43D10022314638463BF093FEE66066
:10B29000B9F1000F2CD04946304603F051FA3D4A2F
:10B2A000B36839463C48FEF71FF994F80890B9F1A5
:10B2B000000F0CD03279914509D04B4639463748BA
:10B2C000FEF712F93368494630469B699847637A1E
:10B2D00023B1727939463248FEF706F9F36A002B3A
:10B2E000A1D039462F48FEF7FFF80023F3629AE712
:10B2F000204AD5E71F49B2E7B8F1000FBFDB33683A
:10B30000DB69002BBBD042462749B6E7DFF89C90AB
:10B310000025DFF89CA04FF0030B05F097FC0520FB
:10B32000F9F794FF9AF8F433AB42ABD919F8014F0F
:10B33000C4B1204606F07AFC804698B12046F7F763
:10B3400061F90446EBB210B180F806B0C371204633
:10B350000121F6F7C9FC98F806302046DB0703D533
:10B36000F6F7F4FA0135DDE7F6F7EAFAFAE74FF017
:10B37000FF3049E6B32B0A088C2A0A08962B0A08E4
:10B380004C2C0A0841E704089A2A0A08752C0A0876
:10B3900083720408952A0A08B42B0A08D92B0A08D4
:10B3A000FC2B0A08332C0A0841700408232A0024C5
:10B3B000481C00202DE9F74F05460846FFF704FD1D
:10B3C0000B46044618B9334A92F8CC762FB9284672
:10B3D00003B0BDE8F04FFEF757BE2646DFF8C89031
:10B3E000DFF8C8A001AA2C49184647F020FC10B984
:10B3F00005F038FC08E056B9012201462846FFF75F
:10B40000F7F9421C04461BD103B0BDE8F08FFCF7EE
:10B41000A1FD2F28834637D80FB105F017FCBBF1EB
:10B42000060F14D01D4901235FFA8BF291F8F41333
:10B43000E0B205F081FA002759464846FEF754F875
:10B4400001AA15490020013647F0F1FBCFE7DAF8F1
:10B4500024361B0114D5FF2C0ED0E1B22846FFF78D
:10B46000F1F9E8E701372846FFF7ECF9F9B298F867
:10B47000F4238A42F6D8DEE70027DFF82080F5E7DC
:10B480000748FDF77DFFD6E72F2206492846FEF73D
:10B49000E5FDD5E790640024D31F0A08481C00206E
:10B4A00031280A08A92C0A08982C0A089853002465
:10B4B0002DE9F74307460846FFF786FC0B4604468E
:10B4C00028B1384603B0BDE8F043FEF719BE01AA23
:10B4D0002E491846264647F0AAFBA0460546DFF847
:10B4E000AC9065B92A4B3246A1B2D3F860063EF063
:10B4F00045FF68BB27493846FEF7B0FD28E0B8F1A4
:10B50000000F06D0B8F1010F25D03846FEF7F8FD40
:10B510001EE0284645F07CFB1F49064602462846A9
:10B52000FCF72CFC50B332461C492846FCF726FC9D
:10B5300030B332461A492846FCF720FC10B3324695
:10B5400018492846FCF71AFCF0B13846FEF79CFD76
:10B5500003B0BDE8F083B31E294638465A425A412B
:10B56000FFF746F9421C0446F2D001AA49460020E2
:10B5700008F1010847F05BFB0546B2E74646F4E7F1
:10B580000126F2E70226F0E70426EEE7D31F0A08B9
:10B5900090640024D52C0A08C92C0A08CC2C0A086F
:10B5A000CF2C0A08D22C0A082DE9F743804608461A
:10B5B000FFF70AFC0B46054628B14046FEF7A0FD02
:10B5C00003B0BDE8F08301AA2C4918462F4647F086
:10B5D0002EFB2E460446DFF8A4907CB9022DECD158
:10B5E000A7F57A73B3F57A7F21D94FF4FA634FF454
:10B5F0007A7223494046FEF75BFEE1E74DB1012D2B
:10B6000010D001AA49460020013547F010FB04463E
:10B61000E3E7012221464046FFF7EAF8431C0646CD
:10B62000EFD1CDE72046FCF795FC0746E9E7154D3D
:10B63000B8B2D5F880355B689847FCEEC07AFF2E2B
:10B64000114B17EE902A0AD195F8F413B6EEC00A02
:10B65000A1420FDC11460D48FDF746FFB0E703EBB2
:10B66000860331460A48B6EEC00A83ED000AFDF7AC
:10B670003BFFA5E70134A3EC010AE9E7D31F0A0861
:10B68000E32D0A08481C0020606B0024002D0A08E6
:10B69000F32C0A08F8B507460846FFF795FBD0B12A
:10B6A000204BD3F8B0600136304634460DF062FBD3
:10B6B0000546F0B90134182CA8BF002420460DF02F
:10B6C00059FB0546A8B9B442F4D138461649BDE83D
:10B6D000F840FEF7C3BC0846FCF73CFC04460DF0FE
:10B6E00049FB054628B921461048BDE8F840FDF75A
:10B6F000FBBE0C4BC3F8B04008F002F92A462146C5
:10B700000B48FDF7F1FE172C09D80A4B0C2202FB5F
:10B71000043393F81C0BBDE8F84007F0D7BA0020BB
:10B72000F9E700BF8C0400240F2D0A08232D0A0816
:10B73000392D0A08AC42090838B50446114D0846AF
:10B74000FFF742FB68B1104B93F900104B1C06D178
:10B750000E4B19790E48BDE83840FDF7C5BEC9B299
:10B76000F8E70846FCF7F6FB032804D8C0B2FDF75B
:10B77000C7FA2946E3E7204603220649BDE83840D8
:10B78000FEF76CBCB32B0A088C04002498530024E9
:10B79000522D0A08622D0A0838B50446114D084694
:10B7A000FFF712FB68B1104B93F901104B1C06D147
:10B7B0000E4B59790E48BDE83840FDF795BEC9B229
:10B7C000F8E70846FCF7C6FB032804D8C0B218F017
:10B7D000F5FC2946E3E7204603220649BDE8384048
:10B7E000FEF73CBCB32B0A088C04002498530024B9
:10B7F0004E2D0A085D2D0A08444B2DE9F74FDFF85E
:10B80000249105461A79009189F800205A7993F815
:10B81000343089F801200BB904F002FA00263C4CC0
:10B8200036F0E0FAB0460D23394A0099734352F8D6
:10B8300003A05046FCF7C6FA002841D0B8F1000F2B
:10B8400001DDFDF785FD51463248FDF7E5FD00229B
:10B8500021462846FEF7F4FBFDF77AFD237903F035
:10B860001803082B45D0102B48D02046FDF74BFE7F
:10B870000D22274B02FB0633B3F8090036F078FAA5
:10B880008346D8B12046FBF7A6FB0746DBE9022139
:10B89000024401442046FBF757FB78B9514601901A
:10B8A0001D48FDF7B9FDDBF80810019A284613463C
:10B8B000CA192146FEF7DAFAFDF74AFD08F1010838
:10B8C000013640F249230D349E42ACD10020FFF7EF
:10B8D000E6F9FF2389F8003089F80130B8F1000F4C
:10B8E00011D1009A28460D4903B0BDE8F04FFEF78C
:10B8F000B5BB0B492846FFF71FFFB6E708492846A6
:10B90000FFF74AFFB1E703B0BDE8F08F985300247A
:10B91000E05A0908612A0A087D2D0A0804280A0845
:10B92000B32B0A088C0400242DE9F74F8046084603
:10B930000F4645F06DF9044620B1012824D13B782B
:10B940002A2B21D1A94E00254FF00D0AA84FB14650
:10B9500004F00104A748FDF713FD0AFB05F3384680
:10B96000013559F80310FDF757FD31462246404690
:10B97000FEF766FB0D36FDF7EBFC40F249239D42D6
:10B98000EBD103B0BDE8F08F3D21384647F089F98F
:10B99000002800F0248103469A4613F8012D202A3E
:10B9A000FAD0AAEB070A0130054610F8013B202B1C
:10B9B000FAD05FFA8AFA4FF00009DFF830B20D23AF
:10B9C0005246384603FB09F35BF803100BEB030404
:10B9D0000091FCF7D3F9064670BB0099084645F084
:10B9E00017F9824528D1277907F0E001402900F0B6
:10B9F0008A8012D871B366797F4A002702EBC606A7
:10BA0000BA463B4696F8D4260092009ABA4202D92A
:10BA1000BAF1000F63D02BB12DE06029ECD0802962
:10BA200000F0A58040467549FEF718FB204603B09C
:10BA3000BDE8F04FFDF767BD09F1010940F2492368
:10BA40009945BCD13A466E49404603B0BDE8F04F37
:10BA5000FEF704BB07F00703042B1CD10B460A2298
:10BA60002846FCF7C7F9D4F8053001468342D9D3FC
:10BA70002046FBF7B7FB0D23624803FB09F95BF88F
:10BA80000910FDF7C9FC00222146404603B0BDE87D
:10BA9000F04FFEF7D5BA052B0DD101230A22284617
:10BAA000FCF7A8F9D4F8053001468342BADB5B42C3
:10BAB0008342B7DCDCE72846FCF74CFA17F0050FA9
:10BAC000014607D1B4F80520B4F807309142A9DB4C
:10BAD0009942EEE7B4F90520B4F90730F6E7D6F855
:10BAE000D01651F8270060B129460193FBF780F882
:10BAF000019B30B94FF0010A39462046FBF772FB33
:10BB00005346013781E707F007076379013F009348
:10BB1000009BB342AFDDAA4615F8013B202BFAD0BB
:10BB20002046FBF749FB0546042F04D8DFE807F061
:10BB3000030E0E141D005046FCF70CFAA8552C21DC
:10BB4000504647F0AEF80136451CE1E75046FCF799
:10BB500001FA25F81600F2E700230A2200215046D8
:10BB6000FCF748F945F82600E9E70123F5E7284600
:10BB700045F04EF8E379064694F805A0DB07A7796F
:10BB80000AD52046FBF718FB0378014623B132465D
:10BB9000284647F05FF9E0B9DEB1B74219D3204635
:10BBA000FBF70AFB3A46002147F064F8B2453FF63E
:10BBB00062AF32461449284647F04CF900283FF45A
:10BBC0005AAF2046FBF7F8FA3246294646F0F4FF12
:10BBD00051E73A460D494046FEF740FA22E739461A
:10BBE000404603B0BDE8F04F06E600BFE05A090842
:10BBF000612A0A088D2D0A08AC420908DB2D0A08C3
:10BC000004280A08D02D0A08253B0A08A02D0A0896
:10BC10002DE9F04F914687B00C461A460021804628
:10BC20004D46FFF72FF800270646B9F1000F63D005
:10BC300029460622204647F071F900283246404640
:10BC400013BF012100214FF0010A4FF0000AFFF756
:10BC500019F80646287812F013FB8346F8B1687984
:10BC600012F00EFB4FF461714FF0190CAB78EA78CB
:10BC70009BF805E01CFB03131CFB021295F801B0B6
:10BC8000297900B14079CDE90410CDE9023251465D
:10BC90003B461A4A4046CDE900EBFDF7A5FB20786C
:10BCA00012F0EEFA8346F8B1607912F0E9FA4FF437
:10BCB00061714FF0190CA378E2789BF805E01CFB4A
:10BCC00003131CFB021294F801B0217900B14079F2
:10BCD000CDE90410CDE9023251463B46074A4046C1
:10BCE000CDE900EBFDF738FB013706340635142F9C
:10BCF0009BD107B0BDE8F08FCA46D0E7E92D0A080E
:10BD00002DE9F041054686B008460F46FFF75CF87E
:10BD1000064638B100235B4901201A4606B0BDE84B
:10BD2000F04175E70846FCF715F91328044600F3BF
:10BD3000A08006258DF81760534E4543781CFBF70D
:10BD400094FA074660B1FCF705F9C0B212F0B2FAF6
:10BD500030B17319027983F8702601238DF81730FA
:10BD60003846FBF782FA074668B1FCF7F3F80D286E
:10BD700009D8062303FB046383F871069DF8173086
:10BD800001338DF81730DFF8FC80A91C0DF1170284
:10BD900038464144FCF7E2F8FBF767FA074668B11A
:10BDA000FCF7D8F8012809D89DF81730062201338E
:10BDB00002FB04628DF8173082F874063846FBF7F0
:10BDC00054FA80B1FCF7C6F8C0B212F073FA50B161
:10BDD0009DF817300622017902FB0462013382F8D4
:10BDE00075168DF817309DF817200623042A2FD1D9
:10BDF00003FB04630022A3F87426062519F0F8FC5F
:10BE000005FB046595F8700612F03AFA95F873167A
:10BE100095F8727619234FF46172804695F875068D
:10BE200013FB012613FB072712F02AFA4379214658
:10BE300098F80520039395F8743614480097CDE9D7
:10BE4000016395F87136FDF74FFB06B0BDE8F08150
:10BE5000052A05D103FB0463002283F87526CCE78D
:10BE6000062ACAD0002308EB050248F80530938063
:10BE7000C3E7132332460649284606B0BDE8F04121
:10BE8000FEF716BA085A002498530024E92D0A0830
:10BE9000022E0A082DE9F04F904689B01A460C464A
:10BEA000002181464546FEF7EDFE3A4E08F1780343
:10BEB0000746DFF8E4B0079394F904000CF0E0FFC4
:10BEC00000285CD0B8F1000F61D029460C22204632
:10BED00047F024F800283A46484613BF01210021C4
:10BEE0004FF0010A4FF0000AFEF7CCFE074695F925
:10BEF00004003BF051F9EA790346514606EB820211
:10BF00004846D2F8582904922A7A06EB8202D2F8DF
:10BF100058290392AA7906EB8202D2F85829029294
:10BF20006A7906EB8202D2F8582901922A680092B7
:10BF30005A46FDF759FA94F904003BF02DF9E279DD
:10BF40000346514606EB82024846D2F8582904922D
:10BF5000227A06EB8202D2F858290392A27906EBE4
:10BF60008202D2F858290292627906EB8202D2F854
:10BF700058290192226800925A46FDF7EDF90C35D6
:10BF8000079B0C34AB4297D109B0BDE8F08FC24695
:10BF9000D1E700BFAC420908082E0A082DE9F04796
:10BFA00080468CB00846FEF70FFF054638B10023E7
:10BFB000594901201A460CB0BDE8F0476AE7CDE9BF
:10BFC00009000B9007A80791544946F003FE064666
:10BFD0003AF0D8FF431C04460CD12B460A2208A98C
:10BFE0003046FBF707FF089B1B781BB9C4B2132C24
:10BFF0000BD944B220460CF0FFFE054640B940463E
:10C00000FEF742F80CB0BDE8F087333464B2F1E7D4
:10C01000424907A88DF8284046F0DCFDB0B3002364
:10C0200002260A221946FBF7E5FE09900027DFF8F1
:10C03000EC90DFF8F0A0494607A846F0CBFDF8B138
:10C04000FBF788FF364A002352F8041B88421FD1B1
:10C05000DBB20AEB8302D2F85829904210D1022FAA
:10C0600020D0032F23D05A1E012FD2B215D00B2A75
:10C0700003D88DF829300136F6B20137042FDAD112
:10C08000052E1AD84046FEF73BF8BBE70126CDE760
:10C090000133102BD8D10023DBE7052AEDD88DF82A
:10C0A0002A30E8E7092BE8D88DF82C30E3E79A1E10
:10C0B0000D2AE2D88DF82B30DDE709AB03CB2860E1
:10C0C00018686960A86020463BF066F8154A9DF83C
:10C0D0002B10034602EB8101D1F8581904919DF809
:10C0E0002C1002EB8101D1F8581903919DF82A1008
:10C0F00002EB8101D1F8581902919DF8291002EB49
:10C1000081020021D2F8582908460192099A00922A
:10C11000054AFDF721F975E7E8580024D31F0A08FE
:10C12000044C0908AC420908082E0A082DE9F04F12
:10C1300090468BB000264FF0190A45464FF46179BE
:10C140000C461A4600210746FEF79CFD0990B8F1FF
:10C15000000F49D029460A22204646F0DFFE00287B
:10C16000099A384613BF012100214FF0010B4FF00F
:10C17000000BFEF787FD2A8909903346069259463F
:10C18000EA88384605922A790492EA780392AA78D6
:10C190001AFB029202926A781AFB029201922A78A2
:10C1A0000092124AFDF720F922893346013659469A
:10C1B00006923846E2880A35059222790492E2789E
:10C1C0000392A2781AFB0292029262781AFB029200
:10C1D000019214F80A2B0092044AFDF7BDF81E2EB6
:10C1E000B5D10BB0BDE8F08FC346DDE7252E0A08B8
:10C1F0002DE9F04380468BB008460F46FEF7E4FD7C
:10C20000044638B100235E4901201A460BB0BDE850
:10C21000F0438BE70846FBF79DFE1D28054600F31B
:10C22000A5800A268DF827404643781CFBF71DF8A9
:10C2300010B101238DF82730FBF717F8514C074652
:10C2400068B1FBF787FE0D2809D80A2303FB0543D5
:10C2500083F8F0069DF8273001338DF82730DFF89A
:10C260002091711C0DF1270238464944FBF776FEF8
:10C27000FAF7FBFF074668B1FBF76CFE232809D8E5
:10C280009DF827300A22013302FB05428DF8273042
:10C2900082F8F3063846FAF7E8FF074668B1FBF77D
:10C2A00059FE0D2809D89DF827300A22013302FBD8
:10C2B00005428DF8273082F8F4069DF82730062BCA
:10C2C0000CD0002309EB0602404649F806305360C3
:10C2D00013810BB0BDE8F043FDF712BF0A2600231F
:10C2E000384606FB0546A6F8F636A6F8F836FAF7FD
:10C2F000BCFF074618B1FBF72DFEA6F8F606384638
:10C30000FAF7B3FF30B1FBF725FE0A2303FB054321
:10C31000A3F8F8061C4B4FF0FF324FF461705A60DF
:10C320000A2303FB0542B2F8F8360693B2F8F63654
:10C33000059392F8F436049392F8F3360393192395
:10C3400092F8F21613FB0101029192F8F11613FB19
:10C35000010300210193084692F8F0360B4A00933E
:10C360002B46FCF7F9FF0BB0BDE8F0831D232246F6
:10C37000074940460BB0BDE8F043FDF799BF00BF49
:10C38000806B0024906400248C040024252E0A086D
:10C39000022E0A082DE9F04F804691461E460C46B3
:10C3A00015460027DFF81CA12DED088B95B094ED04
:10C3B000008AB5EE408AF1EE10FA7BD0D4ED019AF6
:10C3C00094ED029AD4ED038AB9F1000F49D0D5ED6E
:10C3D00000BA95ED01BAB4EE6B8AD5ED02AA95EDDF
:10C3E00003AAF1EE10FA6AD1F4EE4B9AF1EE10FACC
:10C3F00065D1B4EE6A9AF1EE10FA60D1F4EE4A8A91
:10C40000F1EE10FA0CBF0121002132468B46404666
:10C4100081F00101FEF736FCB0EE6B0A064611A86A
:10C42000FAF746FEB0EE4B0A07900EA8FAF740FE68
:10C43000B0EE6A0A06900BA8FAF73AFEB0EE4A0A86
:10C44000059008A8FAF734FE0599069A079B039011
:10C450004046029159460192524600933B46FCF7F2
:10C46000C3FFB0EE480A11A8FAF722FEB0EE690A3F
:10C4700083460EA8FAF71CFEB0EE490A06900BA8F8
:10C48000FAF716FEB0EE680A059008A8FAF710FE53
:10C49000069B059A002103904046029252461034B2
:10C4A0001035CDE900B33B460137FCF755FF082FA7
:10C4B0007FF47DAF15B0BDEC088BBDE8F08F002197
:10C4C000A3E700BF482E0A082DE9F14F06460C46A7
:10C4D000DFF894B12046FEF777FC074638B1002319
:10C4E0005A4901201A4601B0BDE8F04F52E7052233
:10C4F00057492046FBF742FC60B9544B00221A60B2
:10C500001A611A621A631A641A651A661A6701B008
:10C51000BDE8F08F042259462046FBF72FFC054664
:10C520002046002D45D1FAF7A0FE07460028EED0A0
:10C5300044F06EFBDFF834A15FFA80F85AF8049BF0
:10C54000B9F1000F07D122464249304601B0BDE89B
:10C55000F04FFDF783BD4246494638460135FBF7AB
:10C560000DFC84460028E9D1384A034600211746CD
:10C57000013342F8101B082BFAD1374B03EBC505EA
:10C58000D5F880E0BEF1000F05D149463348344C60
:10C59000FCF7AAFF9EE795F87C50AC45F5DA0EEB68
:10C5A0000C1307EB0C140CF1010C0FCB84E80F00FB
:10C5B000F3E7FBF7CFFC072805463DD82046FAF7FE
:10C5C00054FE074658B3FAF7B1FB204B012403EBA6
:10C5D000051383ED000A3846FAF747FE074638B1DF
:10C5E000FAF7A4FB194B013403EB051383ED010AA1
:10C5F0003846FAF73AFE074638B1FAF797FB134B7D
:10C60000013403EB051383ED020A3846FAF72DFED9
:10C6100038B9304601B0BDE8F04FFDF771BD0446B2
:10C62000D9E7FAF783FB094B032C03EB051383EDE2
:10C63000030A3FF454AFECE707233A460949304672
:10C6400001B0BDE8F04FFDF733BE00BF0C5D002424
:10C65000D42A0A0804280A08AC420908612E0A08EC
:10C66000B32B0A08022E0A085C2E0A08184D090886
:10C670002DE9F74F92460C461A4600218146564650
:10C68000FEF700FB00258046DFF864B0BAF1000F2A
:10C690002CD031460422204646F040FC0028424679
:10C6A000484613BF0121002101270027FEF7EAFABF
:10C6B000738880465A46019339463AF825304846F1
:10C6C00000932B46FCF790FE63885A46394648464D
:10C6D0000193043634F8043B00932B460135FCF7F4
:10C6E0003BFE042DD2D103B0BDE8F08F5746EBE7F7
:10C6F0006B2E0A082DE9F34105460846FEF764FB58
:10C700000C46074638B10023334901201A4602B0CF
:10C71000BDE8F041ACE731492046FAF769FA70B953
:10C7200004222D4B4FF47A704FF4FA61013A1880CD
:10C73000598003F10403F9D102B0BDE8F08120462D
:10C74000FBF708FC0328064641D82046FAF78DFD82
:10C75000074698B1FBF7FEFB4FF001080446384648
:10C76000FAF783FD20B1FBF7F5FBB8F1000F09D113
:10C77000284602B0BDE8F041FDF7C2BC40F2EE240D
:10C780008046ECE7A4F2EE2240F2DC539A4203D852
:10C79000A0F2EE229A420AD940F6CA0340F2EE22F3
:10C7A0000F49284602B0BDE8F041FDF781BD0D4BB1
:10C7B00000210D4A03EB8603A3F81C48A3F81E08CA
:10C7C0003346CDE900400846FCF7C6FDB4E7032335
:10C7D0003A460649E5E700BFAC6C0024D42A0A08B3
:10C7E0007C2E0A08906400246B2E0A08842A0A080A
:10C7F0002DE9F04F8FB08946174600211A460646AC
:10C800000024FEF73FFA0DF1240B0546DFF86CA07B
:10C8100059F82480594602A8CDF808803AF06CFCFB
:10C820004FB357F824302A4630469845039313BF38
:10C83000012100214FF001084FF00008FEF722FA15
:10C8400004A9054603A83AF057FC04A9234652461A
:10C85000009130464146FCF7C7FD2346013452465D
:10C8600041463046CDF800B0FCF776FD202CCFD104
:10C870000FB0BDE8F08FB846EFE700BF8A2E0A0878
:10C88000F0B5074689B008460E46FEF79DFA054604
:10C8900038B10023194901201A4609B0BDE8F0401B
:10C8A000A6E70846FBF756FB1F2804461DD830466E
:10C8B000FAF7DBFC014620462BF0A2FB78B103AE71
:10C8C0000E48314600EB84003AF016FC23460C4A31
:10C8D000294628460096FCF73FFD09B0F0BD3846D2
:10C8E00009B0BDE8F040FDF7CFBB1F232A4605493C
:10C8F000384609B0BDE8F040FDF7DABCBC6C002456
:10C900008A2E0A08022E0A082DE9F04F924685B0B9
:10C910000C461A46002181465546FEF7B3F900261B
:10C920008046DFF86CB0BAF1000F2FD02946042200
:10C93000204646F0F3FA00284246484613BF01213C
:10C94000002101270027FEF79DF9EB7880465A4623
:10C9500002933946AB78484601932B8800933346BF
:10C96000FCF742FDE3785A463946484602930435BF
:10C97000A378019334F8043B009333460136FCF767
:10C98000EBFC102ECFD105B0BDE8F08F5746E9E79C
:10C99000942E0A08F0B5074685B008460E46FEF705
:10C9A00013FA054638B100231C4901201A4605B088
:10C9B000BDE8F040A8E70846FBF7CCFA0F2804468C
:10C9C00023DC3046FAF751FC014620462BF0F2FBFF
:10C9D000A8B104F12002124B2946284603EB82033A
:10C9E00093F82F28029293F82E280192B3F82C384E
:10C9F0000C4A00932346FCF7AFFC05B0F0BD384667
:10CA000005B0BDE8F040FDF73FBB0F232A460649BD
:10CA1000384605B0BDE8F040FDF74ABC3C6D002447
:10CA200090640024942E0A08022E0A082DE9F04F83
:10CA300085B014461A46054602910021FEF722F9F8
:10CA40004FF00008064606234FF0000903FB08F7E5
:10CA5000C037029B13F807B0002C7AD0E35D324652
:10CA600028469B45039313BF012100214FF0010A83
:10CA70004FF0000AFEF706F9039B0646374A514677
:10CA80002846CDE900934346FCF7AEFC4346334AC3
:10CA9000514628460137CDE9009B09F10109FCF711
:10CAA0005BFCB9F1060FD4D108F10108B8F1060F0B
:10CAB000C9D1E427029BA7F1E40913F807A0002CD1
:10CAC00049D014F807B032462846DA450DBF4FF07A
:10CAD00001084FF0000801210021FEF7D3F80623DA
:10CAE00006461E4A41462846CDE9009BFCF77CFCE1
:10CAF00001370623194A41462846CDE9009AFCF73A
:10CB00002BFCEF2FD6D1029B93F8EF70ACB194F8C9
:10CB1000EF8032462846474513BF012100210124FA
:10CB20000024FEF7AFF800230C4A21460093284664
:10CB30000723CDF80480FCF757FC0023074A214661
:10CB40002846009307230197FCF706FC05B0BDE8D3
:10CB5000F08FA2469AE7A046CAE700BFA62E0A08B1
:10CB6000F0B5054685B008460B46FEF72DF904469C
:10CB700038B100231B4901201A4605B0BDE8F0403A
:10CB800054E701AE184F6A461749184646F04FF869
:10CB900088B1032C04D12846FDF7B2FA05B0F0BDE8
:10CBA000FBF7D8F96A4646F8040B394600200134F1
:10CBB00046F03DF8ECE7032CEDD1039FDDE901469B
:10CBC0003A463146E0B22BF02FFB18B92846FDF764
:10CBD0005BFAE3E73B46324621460448FCF784FC17
:10CBE000DCE700BFBC6C0024D31F0A08A62E0A088D
:10CBF0002DE9F04F9246002689B04FF019095546AD
:10CC0000B3464FF461780C461A4600210746FEF7FA
:10CC100039F80790BAF1000F27D02946062220469E
:10CC200046F07CF90028079A384613BF01210021FD
:10CC30004FF0010B4FF0000BFEF724F86A790790D4
:10CC4000334619FB02825946384605922A7919FB68
:10CC500002820492EA780392AA7802926A78019298
:10CC60002A780092104AFCF7BFFB627933460136FE
:10CC7000594619FB0282384606350592227919FB7E
:10CC800002820492E2780392A27802926278019280
:10CC900014F8062B0092044AFCF75EFB0A2EB9D169
:10CCA00009B0BDE8F08F00BFBA2E0A082DE9F04F99
:10CCB00080468BB008460F46FEF786F838B1002351
:10CCC000534901201A460BB0BDE8F04F90E707909A
:10CCD0000846504CFBF73EF90928054694F894B7EE
:10CCE00094F895A794F87E98079A00F38980062611
:10CCF0008DF827204643781CFAF7B7FA074648B163
:10CD0000FBF728F90D2805D8A31983F87C0A01231D
:10CD10008DF827303846FAF7A8FA074668B1FBF7CE
:10CD200019F9584509D8062303FB054383F87D0A02
:10CD30009DF8273001338DF827303846FAF795FAF9
:10CD4000074668B1FBF706F9504509D8062303FBEF
:10CD5000054383F87E0A9DF8273001338DF827308C
:10CD60003846FAF782FA074668B1FBF7F3F88145CF
:10CD700009D3062303FB054383F87F0A9DF8273078
:10CD800001338DF82730DFF88890311D0DF127022F
:10CD900038464944FBF7E2F89DF82730062B0BD0C4
:10CDA000002309EB0602404649F8063093800BB099
:10CDB000BDE8F04FFDF7A4B903FB05444FF46171E2
:10CDC000192394F8812A13FB0212059294F8802A01
:10CDD00013FB02130021104A0493084694F87F3A8B
:10CDE000039394F87E3A029394F87D3A019394F871
:10CDF0007C3A00932B46FCF7AFFA0BB0BDE8F08FFE
:10CE00000923064940460BB0BDE8F04FFDF750BA84
:10CE1000145E002498530024BA2E0A08022E0A0831
:10CE20002DE9F04F14468BB00F461A4600210646F6
:10CE3000FDF728FF0546002C00F0D78022783B78CC
:10CE40009A42024630460DBF4FF001084FF00008ED
:10CE500001210021FDF716FF237805469B4A414634
:10CE60003046FCF7C1FA3B784146984A3046FCF719
:10CE700073FA002C00F0BB80627830467B789A42CF
:10CE80002A460DBF4FF001084FF000080121002194
:10CE9000FDF7F8FE637805468D4A41463046FCF7BB
:10CEA000A3FA7B7841468A4A3046FCF755FA07F1E7
:10CEB000C90307F1020A04F1CA0B0593A31C4FF042
:10CEC00000090693822307933B784B4500F391803A
:10CED000002C00F0F58097F8EA30304694F8EA200C
:10CEE0009A422A460DBF4FF001084FF00008012179
:10CEF0000021FDF7C7FE94F8EA300546754A414621
:10CF00003046FCF771FA97F8EA304146714A3046EC
:10CF1000FCF722FA002C00F0D58004F1EA0307F1B7
:10CF2000EA0204F1FA014FF0010833F802CF32F8B7
:10CF3000020F844518BF4FF000089942F5D188F0E0
:10CF400001012A463046C9B2FDF79CFE082105467C
:10CF500004F1EC00FAF75EFE5F4A034641463046B4
:10CF6000FCF742FA97F8EA1007F1EC00FAF752FEE4
:10CF7000594A034641463046FCF7EEF9002C00F0D2
:10CF8000A3804FF0FC094FF0010807EB090104EB07
:10CF90000900F9F72DFE09F10409002818BF4FF028
:10CFA0000008B9F58E7FF0D188F001012A4630469D
:10CFB000C9B2FDF767FE082104F1FC00FAF767F932
:10CFC000464A034641463046FCF70EFA97F8EA1007
:10CFD00007F1FC00FAF75BF9404A03464146304648
:10CFE0000BB0BDE8F04FFCF7B7B9A0463BE7A04651
:10CFF00057E7079BFB180993002C5FD0079B099804
:10D00000E31819460893F9F7F3FD059B5A789BF846
:10D0100000309A424FD1B0FA80F84FEA5818069A79
:10D02000AAF102030AF10E01023A33F802CF32F8F4
:10D03000020F844518BF4FF000088B42F5D188F0ED
:10D0400001012A463046C9B2FDF71CFE62780699F6
:10D0500005469BF81800FAF7AFFD02909BF80030E8
:10D0600041461F4A30460193089B009309F1010392
:10D07000FCF7BAF9059B51467A7809F10109587E07
:10D080000AF1100AFAF798FD059A0290414612F843
:10D09000013F30460BF1010B0193099B0592009370
:10D0A0004B460F4AFCF758F9069B10330693079B33
:10D0B0000933079308E74FF00008B0E7A046D9E727
:10D0C000A04620E7A0464DE7A0467FE7D32E0A08FA
:10D0D000E52E0A08132F0A082B2F0A08422F0A08E8
:10D0E000FA2E0A082DE9F04F8FB004460846B249DF
:10D0F00002AA45F09CFD054640B903460246AF49E9
:10D100004120FFF78DFE0FB0BDE8F08FAC49F9F775
:10D110006FFD064628BB02AAA74945F088FDFAF72D
:10D1200019FF0828054606D908233246A549204696
:10D13000FDF7BEF8E7E7A44C94F8943783420CDC83
:10D1400084F89457DFE731460136384629F0CAFFA4
:10D1500094F89437B342F6DCF2E7064604F294778B
:10D16000F6E79A492846F9F743FD0646E0B902AAD0
:10D17000914945F05CFDFAF7EDFE0828054603D914
:10D18000082332469249D2E78F4C94F89537834270
:10D1900002DC84F89557B6E730460136294639F067
:10D1A000C9FE082EF8D1F4E78A492846F9F720FD90
:10D1B000064600BB02AA804945F039FD0028A2D0EE
:10D1C000FAF7C8FE0828054603D9082332468249E3
:10D1D000ADE77D4C94F87E38834209DD014604F2C8
:10D1E000947029F0C5FF294604F2947029F0CEFF0F
:10D1F00084F87E5887E779492846F9F7F9FC06460E
:10D2000018BB06AD704BDFF8B0910146A84610225E
:10D21000284693F87E7845F02DFDBE4202AA80F2A2
:10D220000A814946002045F002FD10B93A466C4992
:10D230000AE1FAF78FFE013628F8020BEDE7694C98
:10D2400095E80F0084E80F005DE767492846F9F785
:10D25000CFFC0646C0BB5C4B06ADDFF85C9193F893
:10D260007E78BE4202AA80F2F3804946002045F053
:10D27000DEFC014610B93A465C49E5E0AA464FF0AB
:10D2800000080322284645F0F7FD284643F0C0FC7D
:10D29000404502D801360435E3E79AF8000008F16A
:10D2A0000108FAF765FD0AF8010BEEE7B60004463F
:10D2B0004F4DB4423FF427AF06AB2819032219198A
:10D2C000043429F0F9FEF4E74A492846F9F790FCBE
:10D2D0000746002840F0AC80DFF8EC8002AA36490F
:10D2E00098F8946745F0A3FC00283FF40CAFFAF7D8
:10D2F00031FE451E01D4AE4203DC334601223E49D5
:10D3000015E72D4902AA002045F091FC01460028AE
:10D310003FF4F9AE00260DF10C09082203A88DF8A0
:10D32000146045F0A9FD03A843F072FCB0421BD87D
:10D3300002AA2149002045F07AFC00283FF4E3AE20
:10D340000026037898F895A7B1460193564502AA9E
:10D3500019494FF0000080F2858045F068FC834653
:10D3600050B9524625496FE099F800000136FAF7A6
:10D37000FFFC09F8010BD6E7A6B99BF80030303B5B
:10D38000092B0FD91E49F9F733FC38B11D4958460E
:10D39000F9F72EFC70B15A461B4955E04FF00109D0
:10D3A0004FF0FF365846FAF7D5FD002830DA5A46D6
:10D3B000164949E0B146F3E7D31F0A082C5B002465
:10D3C000592F0A085F2F0A08985300246A2F0A0869
:10D3D000732F0A08812F0A088D2F0A089F2F0A0829
:10D3E0008E300A08185C0024C92F0A08AE300A08DB
:10D3F000285C0024F32F0A08F82F0A08CE300A0808
:10D40000B51F0A0804300A080B300A0840300A0821
:10D410000EAB03EB4603013623F8200C96E7524689
:10D420001F4911E033F8022B013724F8022F30E0B6
:10D430002A461C4908E01C49002045F0F8FB00285A
:10D440003FF4FDAE3A4619492046FCF707FE5AE67E
:10D450001549002045F0EBFB00283FF427AF3A4682
:10D460001349F1E745F0E3FB0028D8D105EBC500EF
:10D47000104C082203A98230204404EB051429F043
:10D480001BFE0198FAF774FC08EB050383F85E08AD
:10D4900006ABBE42C6DC454485F8769833E600BF4D
:10D4A00055300A0878300A08D31F0A08AB2F0A083B
:10D4B000D52F0A082C5B00242DE9F04F0F4690462B
:10D4C00089B0002187EA08080646139A00250393CD
:10D4D000FDF7D8FBDFF884906FEA08030446069353
:10D4E00028460BF035FC129B184230D0069BDFF823
:10D4F00070B0034014BF4FF0010A4FF0000A0493CC
:10D5000010EA070328460CBF4A465A46059307927D
:10D510000BF030FC039B8046079A51460090304642
:10D52000FBF762FF049B22463046B3FA83F14909B8
:10D53000FDF7A8FB059A0446039B002A0CBF5A4638
:10D540004A4651463046CDF80080FBF705FF0135CD
:10D55000172DC5D109B0BDE8F08F00BFF3300A0820
:10D56000562E0A0870B504460E46084643F050FB96
:10D570003146054602462046FAF700FC68B9635D6D
:10D580001846FAF7DFFB00B933B901352C442046C1
:10D5900001340378202BFAD070BD0020FCE708B5D9
:10D5A00004460948FBF7CCFEFBF7AEFE074BD3F869
:10D5B00060060EF05DF903F0E5FA012C01D13BF0B5
:10D5C000A3FFF5F7A3FA00BFFA300A08906400241D
:10D5D00010B5044608460B46FDF7F6FB28B90322B2
:10D5E00008491846FAF7CAFB28B90748FBF7CEFEE8
:10D5F0000120FFF7D4FF20460449BDE81040FCF7A6
:10D600002DBD00BF06310A080A310A082F2A0A0870
:10D610002DE9F74F4FF0000B064601AA08462E49A8
:10D620005D4645F004FB01270446DFF8BC80DFF8C7
:10D63000BC90DFF8A4A01CBBBBF1000F28D1274C85
:10D64000002D44D029462648FBF74EFF94F834308D
:10D650000BB902F0E5FA34F0C5FB002384F85D3025
:10D66000FBF728FE15B12846FDF719FB9FB13046A0
:10D67000FDF7CCFA78B1FBF79BFC0020FFF78FFF9A
:10D68000BBF1000F0AD02046FAF764FC85B2C5B999
:10D690003046FCF7F9FC03B0BDE8F08F4146204668
:10D6A000FAF790FB80B949462046FAF78BFB002831
:10D6B000EED05F4601AA5146002045F0B8FA044674
:10D6C000B9E74FF0000BF5E74FF0010BF2E7054823
:10D6D000FBF75CFEBFE700BFD31F0A089853002486
:10D6E00035310A0858310A082C310A085D380A0811
:10D6F00010B50C46FDF78AFA78B1084B01229A74EE
:10D70000FBF756FC0648FBF741FE06492046F9F7B1
:10D710006FFA10B10020FFF742FF10BD98530024AC
:10D720006E310A08D51F0A080329F0B5054685B0F1
:10D730000C46164614D80B4F3970FBF709FE0A4900
:10D740002846FDF7F9FF2246084901A8FAF71EFA14
:10D7500001AB324608212846FDF7C4FAFF233B708F
:10D7600005B0F0BD8C040024B32B0A08522D0A0822
:10D770000329F0B5054685B00C46164614D80B4F64
:10D780007970FBF7E5FD0A492846FEF705F82246C1
:10D7900008496846FAF7FAF96B46324610212846DE
:10D7A000FDF7A0FAFF237B7005B0F0BD8C040024C8
:10D7B000B32B0A084E2D0A0810B5114B86B011493B
:10D7C00004460493104B11480393114B114A0293E2
:10D7D000114B0193114B0093114BFBF71DFEFBF70F
:10D7E000B7FD10491048FBF77FFE3CB10F4A1049C6
:10D7F000104806B0BDE81040FBF776BE06B010BD7D
:10D80000B5310A087F310A08BA310A088A310A0894
:10D81000C4310A0875310A08CD310A08D9310A081D
:10D82000A3530024E9310A08F1310A08D8260A086E
:10D8300029270A0802320A080120BDE72DE9F04F26
:10D840003B4C89B00A4600210546FDF71BFA0590BE
:10D8500094F9000003F040FA8146608834F088FAB9
:10D86000344BD0F808B093F8347017B15F46D0F855
:10D870000CB0A3790026012B38BF0123069322792F
:10D88000637906FB02331BF80380002F3AD0FB5C60
:10D890004345059A2846079313BF012100214FF005
:10D8A000010A4FF0000AFDF7EDF9079B01360590DC
:10D8B00053B303F00F021B0951462846403302922E
:10D8C0001D4ACDE900634B46FBF78EFDB8F1000F12
:10D8D00024D008F00F034FEA1818174A5146029354
:10D8E00008F140032846CDE900634B46FBF734FDC1
:10D8F000069BB342C3DC0834104BA342A8D109B045
:10D90000BDE8F08F3B46C3E7002FDFD04B460C4A03
:10D91000514628460096FBF767FDD7E76B06E7D42C
:10D920004B46074A514628460096FBF715FDDFE7B0
:10D93000A4480908985300242F320A087C49090892
:10D9400045320A082DE9F04F724C8DB0DFF8D091C6
:10D950000A4604F1B00A00218346FDF793F90390CB
:10D960000025A37A99F83460AB4200F3928010341A
:10D970005445F5D140F216200DF1180A34F0F8F9AB
:10D980000027002E4FF015024FF00001D0E90245AC
:10D99000504604BF2546344645F06CF92E78002EDB
:10D9A0003ED069783046059104F01CF995F9029053
:10D9B000049009F1010253425341002C00F0A6806B
:10D9C00000220599A05CB04240F09C80224492F96C
:10D9D0000280C14540F0948052788A4208BF0123FA
:10D9E000012203F001030AF8072083F00101039AE2
:10D9F00058460593FDF746F9059B039044B1464A06
:10DA000030460499CDE900B24246F9F7B3FC059BD4
:10DA1000424A30460499CDE900B24A46F9F7AAFCD9
:10DA200001370335152FB9D184B3564604F13F07AA
:10DA3000DFF8E480DFF8E49016F801ABBAF1000FEC
:10DA400021D12078F8B194F9023001331BD06178EC
:10DA500004F0C8F80546039A01215846FDF712F96B
:10DA600094F902205346294603902078CDE900B866
:10DA7000F9F780FC207853464FF0FF322946CDE974
:10DA800000B9F9F777FC0334BC42D5D10DB0BDE83D
:10DA9000F08FE08834F06CF9002E627AD0E9023120
:10DAA000207A04BF1946334605FB00228F5623B364
:10DAB0009E56B742039A5846049313BF0121002192
:10DAC0004FF001084FF00008FDF7DCF8049B0390CD
:10DAD00043B1114B324629462046CDE900B34346B7
:10DAE000F9F704FC0D4B29463A4620460135CDE9AD
:10DAF00000B34346F9F7FAFB33E74FF0FF36D8E7B8
:10DB000000236DE703323F2A7FF45CAF4FF0FF380C
:10DB10006BE700BF40050024E9930408599304080B
:10DB2000985300242DE9F04F80468BB008460D46EF
:10DB300043F06EF80246A8B3A6492846FAF71EF944
:10DB4000044678BBFBF704FCA34DA448A44EFBF7A6
:10DB500017FCA44F1420DFF8D08239F0FFF9E11050
:10DB6000304604F007020131FBF756FC95F81D9092
:10DB700095F91C00B9F1000F0DD003F0ADF84A463D
:10DB800001464046FBF7B0FC01342435102CE6D1A9
:10DB90000BB0BDE8F08F03F09FF801463846FBF765
:10DBA000A3FCF1E7284605AA8F4945F040F8054651
:10DBB00020B901464120FFF7C5FEE9E78B49F9F797
:10DBC00017F820B98A494046FCF748FAE0E7894E41
:10DBD0000B27002431682846F9F70AF8002808BF07
:10DBE0003446013F06F11006F4D154B98249284663
:10DBF000F8F7FEFF28B12A4680494046FCF72EFA86
:10DC0000C6E7002005AA78498DF8130045F00FF803
:10DC10000646002C4ED000284AD0FAF79BF9031E86
:10DC200043DB2279062A3BD10121E26801FA03F0A5
:10DC300010423AD0DBB2724840FA03F2D20734D530
:10DC400099400139084045F0C5F90546E0880027AC
:10DC500034F08EF86B49039791F83410D0E9022321
:10DC6000002918BF1A46217A637A05FB0133D118BF
:10DC700012F90390029105AA5B49002044F0D7FFF6
:10DC8000834600283FD101235F499CB3029A204676
:10DC900092F90020CDE900312946F9F727FB77E713
:10DCA0005D1E13B1A37A9D42D0DB32465749A4E7EB
:10DCB000574EFAE768B10DF11301FAF725F928B1CB
:10DCC0009DF813502846F4F79DFC20B9324651497F
:10DCD00093E74F4EFAE72846F3F7B4FC814628460F
:10DCE00003F06CFF03902846254603F09FFF029443
:10DCF0000746C0E7CDE900314A4639469DF8130092
:10DD0000F9F738FB44E73949F8F772FF064600286F
:10DD10002FD1ACB1EDB2404F72B229462079F3F762
:10DD200065FC00283FF434AF02883146037838465A
:10DD300001360093C2F30323120BFBF7D5FBEBE78D
:10DD400038687979344C72B2F3F798FC00283FF4C4
:10DD50001FAF028831460378013620460093C2F394
:10DD60000323120BFBF7C0FB102E38687979EAD138
:10DD70000EE72A495846F8F73BFF002877D0584667
:10DD8000FAF7E8F8824642B29CB1E9B22079F3F79B
:10DD90002DFC00284ED1266829462046F9F770F957
:10DDA000324603461E49CDF800B04046FCF756F90E
:10DDB000EEE65FFA8AF6386879790F2E36D99DF843
:10DDC000133018491A09CDF800B003F00F034032A0
:10DDD000EBE700BF59320A083C0100245E320A0812
:10DDE00074320A08E2220A08D31F0A086A240A08C1
:10DDF00085320A0840050024B5350A0899320A0818
:10DE0000FEF103009853002459930408A8320A082D
:10DE1000B32B0A08B8320A08CA320A0821280A08AD
:10DE2000EB320A080E330A08E3330A08F3F726FC3C
:10DE30000028C4D006AE50463146F9F71DFF08A9A8
:10DE40004846F9F719FFCA4520D04FFA8AF38CB13A
:10DE5000029A2946204613702768F9F711F908AB92
:10DE60000246394614480096FBF73EFB90E64FF019
:10DE7000FF3ADFE7039A1148937008AB9DF813202F
:10DE80000096110902F00F024031EDE75CB12668FF
:10DE900029462046F9F7F4F808AB0246314608480F
:10DEA000FBF722FB74E69DF8132008AB0548110927
:10DEB00002F00F024031F3E736330A0859330A08FB
:10DEC00081330A089C330A082DE9F04F0C460746B7
:10DED0008BB040F2162033F04BFF2246054600215E
:10DEE0003846FCF7CFFE404B0646152293F83430F7
:10DEF000002104A8002BD5E9024504BF25461C4695
:10DF000044F0B8FE05F13F03039395F80090B9F192
:10DF1000000F30D095F801A0002C63D022460023DA
:10DF20001178494557D1283392F8018001226B447A
:10DF300003F8182CD0453246384613BF0121002182
:10DF40004FF0010B4FF0000BFCF79CFE064654B15E
:10DF5000B8F1000F07D0254B5A464146484600937A
:10DF60003B46F9F74FFA224B5A4651464846009332
:10DF70003B46F9F747FA0335039B9D42C5D13CB3B5
:10DF8000651C0DF110084034DFF86090DFF860A0E8
:10DF900018F8013BCBB915F8013CB3B116B13046C6
:10DFA000FBF7F4F929783B4615F8010C0022CDF86F
:10DFB00000900026F9F726FA002215F8010C3B46DE
:10DFC0001146CDF800A0F9F71DFA0335A542DFD1BF
:10DFD0000BB0BDE8F08F01330332152BA0D14FF009
:10DFE0000008A7E7A046A5E798530024E993040892
:10DFF000599304082DE9F04F07468DB008460D46A9
:10E0000042F006FE044628B9014601200DB0BDE8E5
:10E01000F04F59E70246A6492846F9F7AFFE30B956
:10E02000A44938460DB0BDE8F04FFCF717B82246BA
:10E03000A1492846F9F7A2FE002854D1FBF788F938
:10E04000DFF8B8A29D480E27DFF8B4B2FBF798F9C5
:10E05000172038F083FF1AF9018BB8F1000F36D082
:10E060000025414658462E46FBF7D6F9B1004046FA
:10E07000013689B203F010FE814603F095FE90F957
:10E0800000300446CBB10DB9FBF762F999F80630C0
:10E09000657803F0020394F90000894A894C002B4B
:10E0A00018BF1446B5B102F017FE224603463146AA
:10E0B00085480095FBF718FA0125042ED6D115B92D
:10E0C0008248FBF75DF9013F17F0FF07C3D10DB0A0
:10E0D000BDE8F08F02F000FE2246034631467C4840
:10E0E000FBF702FAE8E7002407AA764928468DF8EC
:10E0F0001B4044F09CFD18B93846FBF7C5FFE6E726
:10E100000DF11B01F9F700FF81460028F4D09DF8BE
:10E110001B502846F4F776FA20B96E493846FBF7CB
:10E120009DFFD4E72346DFF8DC814FF0FF3403EB9B
:10E13000430218F8022095420BD0002C02DA002A84
:10E1400008BF1C460133152BF1D1002C16DA6249A9
:10E15000E4E71C4607AA5B49002044F068FD064638
:10E16000002800F097805249F8F742FD38BB04467A
:10E170005A4FDFF84C81DFF8909117E04FF000091B
:10E18000E8E73068F3F71CFBB1797379024611F0C8
:10E19000020F96F807A04FEA930348460CBF394692
:10E1A0004146013300915146FBF79EF90134284660
:10E1B000214603F017FD06460028E2D187E74FEA23
:10E1C000151A0222464930460AF1400A05F00F0BA3
:10E1D000F9F7D4FD002845D10390B01CF9F7BAFE39
:10E1E000039902460491013128460592039103F0F8
:10E1F000F9FC059ADDE9031338B95B465246394903
:10E2000000963846FBF72AFF61E7C0799042E9D1D2
:10E210001F466300B9F1000F31D01A1942445678F5
:10E22000013E7A1C23440AAC284614BF294600212B
:10E2300008EB030208F803107B1C39465370FF23D8
:10E2400093702246F9F728FD08AA31462846F9F7C7
:10E2500023FDB74216D108AB5A4651462248FBF778
:10E2600043F934E721493046F8F7C2FC20B15B4658
:10E2700052461F490096C4E74FF0FF37C9E74FF0F9
:10E28000FF36CEE708AB5A4651461A480094FBF7D2
:10E290002BF91CE704EB4404174B02462846A04424
:10E2A0000093012398F80110F9F7ACF80FE700BFCD
:10E2B0006A240A0885320A0859320A08B8330A085B
:10E2C000BD200A08D31F0A08D8330A08F9330A0800
:10E2D000EA330A08FF330A0816340A08B32B0A087F
:10E2E0003F340A0842340A0894340A0821280A08EC
:10E2F0006E340A08B2340A085993040810B10908A8
:10E30000D1330A08482000242A340A082DE9F04FA6
:10E3100089B0074608469C4905AA44F088FC054692
:10E3200030B901464120FFF789FA09B0BDE8F08F06
:10E330009649F8F75DFC044600283BD19448954D7A
:10E34000FBF71EF8944E1420DFF88C8238F006FE9E
:10E3500095F9060002F0C0FC2968AA88034601F17D
:10E3600027413046B2FA82F201F57E01C2F11F0266
:10E37000890A4131FBF750F8E97911B14046FBF7C2
:10E380004BF80134FAF7E4FF0835902CE0D17E49D0
:10E3900005AA002044F04BFC8049F8F729FC00282E
:10E3A000C3D138467949FFF725FE78493846FFF74B
:10E3B000B9FBBAE70024DFF8F89119F9340002F04C
:10E3C0008BFC804601462846F8F712FC40B1013428
:10E3D0001B2CF2D12A4672493846FBF73FFEA4E7D0
:10E3E00005AA694944F023FC064690B3F9F7B2FD4B
:10E3F00005466C4B4FEAC40A03EBC40393F8FE35A1
:10E400004BBB002D29DC09EB0A03588893F80490D4
:10E4100093F805A033F0ACFCEBB2D0F808B003FBE6
:10E4200009AA0093002E00F09A803378002B00F0A8
:10E43000968006A93046F9F767FD002800F08C8029
:10E440009DF818500DBB58480BF80A50FAF798FF82
:10E450006BE70546CDE7002D05DD012B1A4638BFD9
:10E460000122954209DD012B4FF001024F49384648
:10E4700038BF0123FBF71CFF57E705AA42490020DC
:10E48000013D44F0D4FB0646BDE72846F4F7BAF850
:10E49000814600285CD02B09454F4FF000080BF84F
:10E4A0000A504033029305F00F030393BB79002613
:10E4B000012B38BF0123019397F804B097F805A00A
:10E4C000788833F055FC06FB0BA38268D15CA94227
:10E4D00022D1444504D10099B1421DD00021D1542C
:10E4E0005FFA86FB33485FFA88FADDE90212FAF731
:10E4F00093FF59465046FAF7D9FF444509D12E48B3
:10E50000FAF78AFF50465946FAF7D0FF2B48FAF738
:10E5100083FF2B48FAF734FF0136019BB342CBDC73
:10E5200008F101080837B8F11B0FBFD1D9F8001066
:10E53000B9F8042001F127412248B2FA82F201F52C
:10E540007E01C2F11F02890A4131FAF7CDFFECE6E4
:10E550003846FBF799FDE8E632461B493CE71BF8D5
:10E560000A30013573B11A09184903F00F0306A8E0
:10E570004032F9F70BFB06AB2A4641461448FAF73E
:10E58000B3FFD2E6134BF7E7D31F0A0859320A0844
:10E59000D8340A08C820002416350A0821350A088C
:10E5A00025350A08AC42090841350A08022E0A0836
:10E5B000A448090853350A0838200A0877350A089C
:10E5C000F9390A0881350A089D350A083E320A08D9
:10E5D000B9350A08091F0A086A200A08224BB0F553
:10E5E000FA6F1A680346A8BF4FF4FA63B3F57A7F4F
:10E5F000B8BF4FF47A73D20416D540F2DC52904281
:10E6000015D040F2DB5207EE903A9042F8EE677A6E
:10E610001FD8DFED166A9FED167A77EEE67A9FED4A
:10E62000150AA7EE870A7047B0F57A7F02D89FEDEA
:10E63000120A704707EE903ADFED106A9FED107AEC
:10E64000F8EE677A9FED0F0A77EEE67AA7EE870A73
:10E650007047DFED0D6A9FED0D7A77EEE67A9FED5C
:10E660000C0AA7EE870A7047BC59002400007A44C0
:10E67000D62000C000E082440000000000407A4440
:10E68000661000400000404200A0BB44D62000407D
:10E690000000834409494FF4EB7200234FF0550CFE
:10E6A000C0F80210C2800649064A0370A0F808C0EC
:10E6B000C0F80A104382C0F80E2070474A01B40027
:10E6C000C2010E0196004400704700BF704700BFB2
:10E6D0000020704701207047704700BF704700BF9F
:10E6E000704700BF704700BF9FED010A704700BF31
:10E6F0000000000000207047064B1B78834206D9BB
:10E7000000EB4000044B03EBC00358697047002046
:10E71000704700BF000600203C05002000EB4000D1
:10E72000024B03EBC003587C704700BF3C05002040
:10E73000024B1878003818BF0120704700060020EF
:10E7400003681B6903B11847704700BF70B5094CD7
:10E75000236873B10546002606E099681A681E739F
:10E7600021609047236823B15A681846AA1A002AE4
:10E77000F3DA70BDA47A00240B4B1A79D20700D5C6
:10E7800070479A68002AFBD04FF47A7101FB02F2BD
:10E790009042F5D3054A12781AB9054A9168126970
:10E7A0000A6000229A607047A47A0024CC5D00249D
:10E7B000E05D002408B5294B1B68DB041ED5B5EECF
:10E7C000400AF1EE10FA26D0DFED257AB4EEE70A22
:10E7D000F1EE10FA1FD49FED237AB4EEC70AF1EEE2
:10E7E00010FA2AD870EE677A9FED1F7A9FED1F0A04
:10E7F000A7EE870A43F008FD80B208BDDFED187A66
:10E80000B4EEE70AF1EE10FA0BDA9FED190A43F0C5
:10E81000FBFC80B208BD9FED170A43F0F5FC80B207
:10E8200008BD70EE677A9FED147A9FED140AA7EE8B
:10E83000870A43F0E9FC80B208BDDFED117ADFED15
:10E84000116A70EE677A9FED107AA7EEA67AB0EEA5
:10E85000470A43F0D9FC80B208BD00BFBC59002470
:10E860000000404200E0824466BEFFBE0060BB4440
:10E8700000007A440080BB4438DFFF3E00407A4409
:10E880000000834466BEFF3E00A0BB44904B1B6863
:10E8900013F0200370B52DED048B00F094808D4CA7
:10E8A000237B13F0020300F0CC80D4ED077A238C95
:10E8B000F8EEE77AC4ED047A002B00F0DE8007EE74
:10E8C000903ADFED856A9FED857AF8EEE77A86EE7D
:10E8D000A79A89FE479A2279012394F84C1012F0E6
:10E8E000010279D0002900F0AF80D4ED169AF1EE44
:10E8F000699A002B40F0B480D4ED1A8A9FED789A83
:10E90000784B1E780D2E07D19FED770A28EE800AEE
:10E9100043F07AFC754B98800123D4ED1C7A94ED7A
:10E920001D7A78EEE78A94ED1B8AE7EE287A77EE77
:10E93000C86AC4ED1C7AA7EE268A84ED1B8A84ED92
:10E940001A8A0BB184ED158AD4ED207A94ED1E7AE3
:10E95000B0EE676ADFED605A38EE477AD4ED216A8F
:10E9600094ED1F0A84ED1E8A97EE256AE6EE867AFC
:10E9700037EEC07AC4ED207AA6EE870A84ED1F0A2E
:10E9800084ED220A43F040FC02B282EAE273A3EB78
:10E99000E2739BB2092B73D9002AACBF0A380A3044
:10E9A0000D2E05B2A4F88C506FD0242E00F082807A
:10E9B000382E05D1B0EE480A43F026FC4B4B988028
:10E9C000BDEC048B70BD9FED4A9A424C227994F8BD
:10E9D0004C1012F0010285D171BB94ED147ADFED79
:10E9E000456AD4ED167A27EE267AF1EE677A84ED41
:10E9F000147AC4ED157A4BB1012194F86020236993
:10EA00008A4284F84D10E36518BF6365354B1E7864
:10EA10000D2E0BD1D4ED047A9FED377A334B67EE90
:10EA2000877AFDEEE77A17EE902A9A80DFED2C8A3E
:10EA30000023F0EE689A70E784F84D2084F84C20AB
:10EA4000CBE79FED2B9AC1E7D4ED149A0122C4EDD8
:10EA5000169AF1EE699A84F84C20002B3FF44CAFE3
:10EA600094F84D3033B1D4ED048AD4ED177A78EEB2
:10EA7000E78A45E7D4ED1A8A42E79FED1D9A2AE717
:10EA800000250D2EA4F88C508FD1DFED137A9FED69
:10EA9000160A29EE279A154C29EE800ABDEEC99A6E
:10EAA00019EE103A238043F0AFFBE5806080BDECA7
:10EAB000048B70BDDFED0C7A94ED150A20EE270A69
:10EAC00043F0A2FB094BBDEC048B588070BD00BF26
:10EAD000EC620024A47A00240000C8426666663F07
:10EAE00000000000142B0024CDCCCC3D182B0024BA
:10EAF0009A99993ECDCC4C3F0AD7233C494B1B6891
:10EB00001B0600D470472DE9F041474CD4F89C30E7
:10EB10002DED048B84B013B104F1900098470023CD
:10EB2000D4F8A02069464148CDE90033CDE902334D
:10EB30009047009BD4F8B820BDF904609D1AA4F852
:10EB4000A46004D104B0BDEC048BBDE8F08194F85E
:10EB5000C0209DED020A9DED039A002A5ED0B1EE21
:10EB6000408AB4F8C220002A55D094ED327AD4ED10
:10EB7000357A38EE475A94ED336A79EE675AD4ED18
:10EB8000366A94ED318AA6EE057AD4ED348AE6EE43
:10EB9000A57A37EE485A84ED327A77EEE85AC4ED1A
:10EBA000357AA6EE058AE6EEA58A84ED318AC4EDB3
:10EBB000348A1F4A84ED2A0A127884ED2B9A1C2A83
:10EBC00084ED2C8AC4ED2D8AC4F8B830BAD1DFEDBB
:10EBD000199A194C20EE290A43F016FB29EE290A4E
:10EBE000074643F011FB28EE290A804643F00CFB50
:10EBF000002328EEA90A1A4666F30F0368F30F02F2
:10EC000067F31F4360F31F42C4E9003243F0FCFA8C
:10EC10006581208196E7F0EE498ACAE7B0EE408A26
:10EC20009FE700BFEC620024A47A0024347B002418
:10EC3000142B002400007A44182B00246B4B1B7803
:10EC40002DE9F04F87B0002B00F0CA80684D4FF0DF
:10EC500000086848A968FAF747FC69686648FAF747
:10EC600043FC664B6648D3E90031C91A654B1A6804
:10EC7000B1FBF2F2FAF738FCFAF76AFB6248FAF7EE
:10EC80007FFB6248FAF77CFB614B5FFA88F41B78E4
:10EC9000A34221D85F4D00245F4EFAF759FB01349F
:10ECA00055F8041F3046FAF7B7FB162CF7D15B4D29
:10ECB0000124594EFAF74CFB2B4669680134304663
:10ECC0001B680435C91AFAF7A7FB162CF4D107B054
:10ECD000BDE8F04FFAF73CBB514B14264FF03C0B0C
:10ECE000671C03EB840306FB045693ED000A43F014
:10ECF0008BFA96F81EA081B2B6F80E901AF0010FAA
:10ED000080B20CBF2D2252221AF0020F0490454807
:10ED10000CBF2D2354231AF0040FB1FBFBF10CBFE1
:10ED20004FF02D0C4FF0560C1AF0080F05914FF0D4
:10ED300064010CBF4FF02D0E4FF0430E1AF0800F00
:10ED400001FB09F10CBF4FF02D0A4FF0530ACDE93A
:10ED500000CECDE902A13946FAF75EFBB37FDB07AF
:10ED60003AD55C23304A6343D118D05891ED010A5B
:10ED700070B1B8EE400ADFED2D7A20EE270A07EEDB
:10ED8000900AF8EE677A80EE270A43F03DFA00B267
:10ED9000642290FBF2F102FB11022548FAF73CFBDA
:10EDA0001421244808F1010801FB075701FB045412
:10EDB000F988628A0491218B02F00303920803917F
:10EDC000E18A0291A18B0191A18A009119214B4303
:10EDD000218AFAF789FB57E71748FAF7B1FADFE714
:10EDE000164807B0BDE8F04FFAF7CABA0400002091
:10EDF000341B0020FB350A080B360A083C1C002097
:10EE000022360A08601E00244F360A08AB360A086C
:10EE10003C200020DC1B00205B370A08E01B0020A0
:10EE20007C34002007370A085418002000401C4694
:10EE300024370A0839370A0830370A085F370A08C2
:10EE40002DE9F84F002607460C461D4DB046DFF869
:10EE50007890DFF878A02046FBF7B6FFD5F800B031
:10EE600048B921465846F8F7ADFF20B921466868F1
:10EE7000F8F7A8FF80B15846FAF762FA696811B14D
:10EE80005046FAF7C9FAA96811B14846FAF7C4FA28
:10EE90004FF00108FAF75CFA01361035382EDAD156
:10EEA0002046FBF791FF48B9B8F1000F06D1224682
:10EEB00038460449BDE8F84FFBF7D0B8BDE8F88FF5
:10EEC0009878090887370A0881370A087B370A08C3
:10EED000F8B5384C2368002B57D00A2801D00D28EC
:10EEE00051D1354D95F8DC300BB1FAF731FA334E8C
:10EEF0002321304643F0D5FE08B1801B20602368F3
:10EF0000002273B902B12360FAF7EEF995F8DC300C
:10EF1000F3B12B48BDE8F840FAF712BA01220B46CC
:10EF2000EFE7591E705C2028F8D092B90022254CDA
:10EF3000224FF2543926013E0DD13146224B9C42DC
:10EF400012D2E3682068984795F8DD30002BDBD1BA
:10EF5000F8BD2360EAE721683846FEF703FB014667
:10EF60000028EBD11034E6E795F8DC3023B11749DF
:10EF70001748FAF761FFC7E71648FAF7E1F90F48B3
:10EF8000FAF7FEF9C0E7FF2BE2D8A0F120025E2AD3
:10EF9000DED80BB92028DBD05A1C2260074AD05497
:10EFA000054B93F8DC30002BD2D0BDE8F840FAF7DF
:10EFB00011BA00BFB4620024A47A0024B461002412
:10EFC000D01F0A0898780908187C09089B370A0896
:10EFD000B7370A08BD370A0870B5254C2378012BCE
:10EFE00000D070BD234B1B68002BFAD0224D2B683C
:10EFF00028465B6898470028F3D0204B204E1A68BB
:10F00000338892889A421FD31E49002228460968F5
:10F010004968EA622A6803FB01F1D36898472B68C4
:10F020009B6813B128469847F8B13388164A0133D4
:10F0300052683380002AD4D0116893884A691342F9
:10F0400018BF1B048B6170BD0F4A00210F4B526823
:10F050001B782170002AC4D0C3F340039188126842
:10F060001B0101FA03F3936170BD3AF055FADCE736
:10F07000562C0024801D0024841D0024502C0024C4
:10F08000542C0024482C0024C01D0024CC1D002436
:10F09000C04BDB79022B40F01D812DE9F047BE4CBF
:10F0A000B4F8DE30B4F8E0209A422DED028B82B045
:10F0B00000F00581A4F8E0300126B4F8E23013F442
:10F0C000006300F0038194F8E470002F00F00382E5
:10F0D000DFF8F48294ED1A8A98F80050B4F95CA134
:10F0E0004A2D00F04881492D11D10023B4F8F0C019
:10F0F000B4F8F2101A46E08F6CF30F036AF30F02B4
:10F1000060F31F4361F31F42A449C1E90032B4F91F
:10F110005E21DFF8B892AAEB0203DFEDA16ADFED12
:10F12000A17A07EE103A99F81C30B8EEC77AA3F12D
:10F130000503B3FA83F3B4EEE67A5B0967EE277A48
:10F14000F1EE10FA84F8F43000F208819FED967A1F
:10F1500077EE877AF0EEE78A4A2DA4F8F220C4ED24
:10F160003E7AC4ED438A00F0CC80002E61D0D4ED0D
:10F17000587A4C2D94ED590AF8EE677A8B4A9FED38
:10F180008C7A116830EE670AC4ED3A7A67EE876AC6
:10F19000C4ED597AD2ED017AA38F20EE270AC4F884
:10F1A000FC10C4ED3B6AB4F86E1184ED400AA4F87B
:10F1B000F03000F0418199B307EE903A94F8853130
:10F1C000F1EE005AD4ED6A6AF8EEE77AF5EEC06A1D
:10F1D00077EEC07AF1EE10FAF0EEE77A67EE877A12
:10F1E00007EE103AB8EEC77A87EE876A36EE257AD0
:10F1F000C5EE877AC4ED537A40F38D81DFED6D7AE9
:10F20000B0EE007A66EEA77AC7FEC77A042F05D162
:10F21000B0EE0C7A86FE476A76EE277AC4ED447A21
:10F22000482D00F053814A2D03D142F0EDFF5B4B96
:10F230001880F5F73DFB99F81C30052B40F0C8808D
:10F24000237B13F0010200F0DD80D4F888215A49B5
:10F25000821A8A4240F3E28203F0020394F84020CB
:10F26000C4F88801002B15BF0023012301210021D0
:10F27000032A84F88C3194F98E318CBF4FF0FF3221
:10F2800001221344022B1A46A8BF0222012B22EAB4
:10F29000E27284F88E2100F3C982002384F88D3154
:10F2A00084F85411082F3FD8DFE817F038017402B2
:10F2B000C10189010202E901300033007201B4F892
:10F2C000E230002613F400637FF4FDAE1F4684F89D
:10F2D000E430FDE6394B03F1780102E00633994250
:10F2E0000ED01A780A2AF9D19878DA789042FFF489
:10F2F000D4AE5A79002A7FF4D0AE06339942F0D1C9
:10F300007047264BA3F808A05A812EE7304618F024
:10F310001BF82B4BD4ED4F7A93ED187AB4EEE77AC5
:10F32000F1EE10FA00F3E28098F800304A2B29D071
:10F33000242B09D1DFED1B7A94ED450A20EE270A34
:10F3400042F062FF154B188017F0B8FE304602B04D
:10F35000BDEC028BBDE8F04717F0D0BBDFED196ABA
:10F36000B4EEE67AF1EE10FA7FF7F4AE9FED0E7A86
:10F3700077EEC77AEEE6B0EE480A42F045FF074B5B
:10F380009880C4E694ED470A42F03EFF034BD880D4
:10F39000DAE700BFFC590024A47A0024182B0024CB
:10F3A0000000E1C4CDCCCC3D0000B443F005002406
:10F3B0000AD7233C3EC3AE393F420F00085A00240F
:10F3C000D42100200000E144142B0024F06200242A
:10F3D000002384F85431082FA6D801A353F827F04E
:10F3E0001DF504080FF804082FF60408BFF50408FB
:10F3F000B1F604087FF604080DF3040813F30408BB
:10F4000091F5040884F85421082F8DD801A353F8EE
:10F4100027F000BF1DF5040815F804082FF60408AE
:10F42000BFF50408B1F604087FF604080DF30408DC
:10F4300013F3040891F50408FDEEC07ACC4D17EEE5
:10F44000900A288100293FF4F4AE07EE903A94F830
:10F450008531B1EE005ADFEDC76AF8EEE77A94ED38
:10F460006A6AB5EEC06A77EEC07AF1EE10FAF0EE95
:10F47000E77A67EE877A07EE103AB8EEC77AC7EEFA
:10F48000875A75EE854A65EEA67A85EE247AFDEEFA
:10F49000E77A17EE903A6B8184ED537A40F3DF817F
:10F4A0009FEDB57AF0EE007A26EE077A87FE677A4E
:10F4B00067EE267AFDEEE77A17EE903A1BB2042F3C
:10F4C000AB8100F0D08184ED447AB2E642F09CFE3C
:10F4D000A74B9880ADE60123384684F8E43017F056
:10F4E0000DFB17F0EBFD94F8E470F1E5A34A136807
:10F4F00043F0805313602379D90708D594F8A221EB
:10F5000012B943F002032371072011F039FB0023E5
:10F5100084F8E43008E7DFED9A7A77E62379DD07AF
:10F5200004D4984B1B7A002B00F0B581D4ED457ABA
:10F53000C8FE277AC4ED457A002E3FF4F5AEB4F844
:10F540006C31F6EE005AD4ED3B6A06EE103A94F8B0
:10F550007B3166EEA56AB4F88021B8EE466A012BCD
:10F5600007EE102A84ED478AC6FEC66AC4ED4C6ACF
:10F5700000F0D881B8EEC77ADFED7E6A022B27EE65
:10F58000267A00F0C88177EE877AC4ED467ACBE61A
:10F590007A4A136843F0805313602379DA0708D559
:10F5A00094F8A22112B943F002032371012011F053
:10F5B000E7FA002384F8343184F8E430B4E6B7EE97
:10F5C000007AD4ED4E7AF4EEC77AF1EE10FA05D552
:10F5D0009FED6D7A77EE877AC4ED4E7AF3EE0E7A70
:10F5E000F4EEE78AF1EE10FA0DD5B4F8683107EEC3
:10F5F000903A0423F8EE677A84F8E4300023C4EDEF
:10F600004A7A84F83431B4F86E3194ED407A07EEDA
:10F61000903A5E4B84ED497AF8EEE77AB4EEE77AF9
:10F62000F1EE10FA4CBF012200225A727CE694EDF2
:10F63000467A564BB4EEC87A1A7AF1EE10FACCBF7D
:10F6400001230023934200F0F680B4F87631D4ED24
:10F650003B6A07EE903A002384ED477AF8EEE77AAA
:10F66000C4F82031F4EEE76AF1EE10FA02DD03236C
:10F6700084F8E430D4F80031C4F8243154E694F826
:10F6800090319FED3C7A07EE903AF8EEE77A67EE1C
:10F69000877AB4EEE78AF1EE10FA05D50622002348
:10F6A00084F8E42084F83431304617F04DFE3BE610
:10F6B000364AB7EE007AD4ED4E7AF4EEC77AF1EE20
:10F6C00010FA05D59FED307A77EE877AC4ED4E7A41
:10F6D000B4F86E3194ED497A07EE903A537AF8EE29
:10F6E000E77AF4EEC77AF1EE10FACCBF01220022DD
:10F6F0009A4207D177EEC77ADFED236AA7EEA67AA2
:10F7000084ED497AF7EE006AD4ED547A9FED206AD1
:10F71000B0EE007A76EEE76AE6EE867A37EE677A42
:10F72000C4ED547A84ED527A002E3FF4FDADB4F866
:10F730006831B6EE007AD4ED3B5A06EE903A94ED7D
:10F740004C6AF8EE666AF4EEC65A26EE877AC4ED85
:10F750004A6AF1EE10FA67EE277AC4ED4B7A3FF66B
:10F76000E3AD0522002384F8E42084F83431DBE59E
:10F77000182B00240000C8423EC3AE39805C002430
:10F78000000000006C5900240AD7233CF005002437
:10F790000AD7A33BF1EE047A94ED3B7AB4EEE77A14
:10F7A000F1EE10FA00F18680B4F8763107EE903A67
:10F7B000F8EEE77AB4EEE77AF1EE10FA00F18E8017
:10F7C000D4ED467AB4EEE78A00230022D4F8001183
:10F7D000C4F83831F1EE10FAC4F82C31C4F82831ED
:10F7E000C4F85031C4F820314FF07E5384F83421EE
:10F7F000C4F84831C4F84C314CBF01230023504AAF
:10F80000C4F824111372022384F8E4308CE5237BBE
:10F81000D807BFD4072384F8E53085E594F88C3108
:10F820003BB994F88D1181F0010139E5012384F889
:10F830008D31002134E593B3B4F87C319FED417AEA
:10F8400007EE903AF8EEE77A67EE877A94ED477A1A
:10F85000C4ED487A77EE277AC4ED477A0AE79FED40
:10F860003A7A00232BE6F0EE0C7A0192C5FEE77A95
:10F8700077EE877AC4ED447AF5F71AF899F81C30D8
:10F88000019A052B43D1237B13F001017FF4DDACFA
:10F8900084F854110DE70023C4F8143144E5B4F89A
:10F8A0007E319FED2A7A07EE903AF8EEE77A67EE1E
:10F8B000877ACBE794F89031DFED256A07EE903A2E
:10F8C000F8EEE77A67EEA67AB4EEE78AF1EE10FA80
:10F8D0007FF56AAF082384F8E43025E5B4F8803179
:10F8E000B6EE007ADFED1A5A06EE903A9FED196AED
:10F8F00067EE877AF8EEE66AB0EE487AC4ED4C7AA5
:10F90000A6EEA57AC7FE067AC4ED467A5AE700232A
:10F9100084F85431CDE678EE077AC7FE877AC4EDD5
:10F92000467A01E5B4F86A319FED097A07EE903A1C
:10F93000F8EEE77A67EE877AC4ED467AF4E400BF22
:10F94000F00500240AD7233C000000000AD723BC9E
:10F950000000C84200007A44F8B5994B1B68D906EC
:10F960002DED028B02D4BDEC028BF8BD954CD4F882
:10F97000BC3113B104F5D6709847D4F8C03194ED7A
:10F98000808A002B00F0A2808F489847C21C054651
:10F99000E9D0002875DA431C00F0FB806FF001000D
:10F9A0008A4E4FF60922C4F8C801F368EB1A03FB2C
:10F9B00003F3934200F39C80854AA2FB032343F3A5
:10F9C000CF0394F81D124A1C04EB4101A1F8203228
:10F9D000D3B2052B84F81D3200F0A88094F82A32A7
:10F9E000F56094F8D451002B00F0B780B4F82022D1
:10F9F000B4F822321344B4F824221344B4F8262273
:10FA00001344B4F8282213441BB2B3F5FA4F1A4634
:10FA1000A8BF4FF4FA4222EAE272A4F8DC21002DDA
:10FA200069D001256B4B1B781A2B6DD01B2B41D154
:10FA3000D4F8CC716849D4F8D861002F08804D8083
:10FA40008E8035DDB2F5167F32DA002830DD002DEC
:10FA500000F0AB80D4ED717A8642B4EEE78AD4BF71
:10FA600000260126F1EE10FACE802AD407EE900A85
:10FA7000F8EEE77A67EE887AFDEEE77AC4ED737AFE
:10FA800071E7D4F80432554904EB83020133096865
:10FA9000052BC2F80802C4F8D011C4F804327DD096
:10FAA00094F81C32002B3FF47BAF37F0B7FC77E7BC
:10FAB0000022CA80D4ED717AF4EEC87AF1EE10FA21
:10FAC0003EDD4FF0FF33C4F8CC314CE74FF0FF324E
:10FAD000404B10461B78C4F8C8211A2BC4F8CC211F
:10FAE0007FF441AF3C4948808A80BDEC028BF8BD71
:10FAF0004FF4C85365E7002894DDB3F5167F38DB73
:10FB0000012384F8D4318CE7D4ED717A3249B4EE14
:10FB1000E78ACA80F1EE10FA01D4002812DA4FF019
:10FB2000FF334FF0FF32C4F8CC31DCE70023F5603F
:10FB300094F8D45184F81D32012384F82A3255E711
:10FB40000028BEDB07EE900AF8EEE77A67EE887AC7
:10FB5000FDEEE77A17EE902ABFE74FF6FF734FF0FE
:10FB6000FF32A4F8DC31002D7FF45CAF00287FF772
:10FB700059AFD4F8D831834209DA00EB8003184931
:10FB8000C3EB0313A1FB03135B09C4F8D8310025B1
:10FB900048E7124B1B68C4F8D03101E7002201236B
:10FBA000C4F8042284F81C327FE7D4ED717A012373
:10FBB000B4EEE78ACB80F1EE10FA82D456E700BFAC
:10FBC000EC620024A47A0024507C0024F005002478
:10FBD000CDCCCCCC142B0024182B0024B81D002431
:10FBE0001F85EB5138B50546F9F78EFB0A4B00240B
:10FBF00018680BF03DFEF9F777FB084B83F8DD4002
:10FC000083F8DC401AF000FC25B12046BDE83840FE
:10FC1000FDF7C5BC38BD00BFF06A0024A47A0024FB
:10FC200038B5074C074DAC4203D3074B01221A707D
:10FC300038BDA288D4E9021042F0BEFF1C34F2E7BE
:10FC4000FC820A08148B0A08CC5300242DE9F04FDB
:10FC50000E4693B082469F4930461746FDF782FC18
:10FC60000546002840F01F819B493046FDF77AFC8D
:10FC70000546002840F0198198493046FDF772FC8E
:10FC80000546002840F0138195493046FDF76AFC8F
:10FC90000546002840F00D8192493046FDF762FC90
:10FCA000002805460ABF0124082435467F428E49B4
:10FCB000284607F010073C43FDF754FC002800F0ED
:10FCC000FA8044F02004894B1B780BB9FFF7A8FF9A
:10FCD00032F088F814F0090F00F02C838448F9F70B
:10FCE00055FB0020FDF768FD14F48073059340F088
:10FCF000EC808048F9F74AFB7F48F9F741FB04F0B4
:10FD00001803182B05D17D48F9F740FB7C48F9F71B
:10FD100037FB01230493F9F71BFB7A497A48F9F77B
:10FD2000E3FB7A497A48F9F7DFFB04F48473082B84
:10FD300007D178495046F9F7ABFC76495046FAF7B7
:10FD400057FB14F0800307930ED1734B204693F8B2
:10FD50002C2203F50B73002A704A06BF01211346BB
:10FD600000216F4AF9F7F8FA6E492046FDF766FD63
:10FD70006D492046FEF7A8F86C492046FDF7E2FDE4
:10FD80006B4B1D686B4B1E6814F01003039340F01F
:10FD90009E806948F9F7FAFA039B02934FF0000836
:10FDA000664B9946069365EA0603099359F804BB26
:10FDB000BBF1000F21D00127099B029A204607FAC8
:10FDC00008F73B400CBF012100210893FAF75AFFC6
:10FDD00066EA05035A4A029020463B425B4614BF3E
:10FDE00001210021F9F700FB08995B46544A0039CC
:10FDF000204618BF0121F9F7AFFA08F10108B8F160
:10FE00001D0FD3D166EA05034FF00008DFF84C91CF
:10FE10000893069B53F804BB0693BBF1000F23D055
:10FE2000012707FA08F73E420AD065EA06034A4668
:10FE300020463B425B4614BF01210021F9F7D4FA6A
:10FE40003D4211D0089B2046029A1F400CBF012161
:10FE50000021FAF717FF391E02905B464A4618BF89
:10FE600001212046F9F778FA08F10108B8F11D0FD1
:10FE7000CFD1344B2046344A3449FCF70BF8079B6A
:10FE8000002B6DD0134B224618215046FAF72AFF5B
:10FE9000049B002B00F0AE812D48F9F777FA2D482E
:10FEA000F9F76EFAA6E1012400E70224FEE6042435
:10FEB000FCE68124FAE628492846FDF753FB002892
:10FEC0003FF401AF44F48074FDE6002322E71A4BAF
:10FED00063E700BFDD370A08E4370A08EC370A0891
:10FEE000F2370A0821350A084F310A08CC5300249A
:10FEF00000380A0808380A0820380A082C380A0886
:10FF000054380A08D8260A081B270A0829270A088D
:10FF10003E270A08B32B0A08A47A0024253B0A08C6
:10FF200064380A0871380A087B380A085B220A0814
:10FF3000D879002468590024CA370A08A44C090853
:10FF400081380A0898380A08E85800248C77002479
:10FF500055390A086B390A08FB370A088D380A0830
:10FF6000DFF8AC832046DFF8AC9398F8002099F8CE
:10FF70000030B34F9A42B34A13BF0121002101263A
:10FF80000026FAF77FFE99F8003005463146013B1E
:10FF9000AD4A204657F82330F9F726FA98F8003092
:10FFA0003146AA4E013BA84A204657F82330F9F7BC
:10FFB000D3F9D6ED007AA64A2046F5EE407AF1EE66
:10FFC00010FA0CBF01210021F9F7C6F92B46324681
:10FFD000A0492046A04EFCF7DDF9A04DA04B2046DD
:10FFE000A04A0193009232682968FDF765FA9E4B9A
:10FFF00040F20222204601930092B268A968FDF700
:020000040805ED
:100000005BFA039B002B40F0FB809848F9F7BEF9A0
:10001000039A974E012597480021974F16F8013B08
:1000200010F801EB03F1480CEC440CF820EC17F845
:1000300001CB0CF14808E84408F810EC002D00F062
:10004000E180A3EB0C056B426B4101311D46082991
:10005000E4D1002683F0010120468DF83060FAF7E4
:1000600011FE0EAB854A294620468DF84060F9F70F
:10007000BBF90AAB814A29462046F9F76DF9804B56
:10008000804A20468049FCF7B3FB804B804A2046DB
:100090008049FCF739FC804B7A4A20467A49FCF7C4
:1000A000C5FC7E4B7E4A20467E49FBF7B1FD7E4B68
:1000B0007E4A20467E49FCF739F87E4B7E4A204630
:1000C0007E49FCF7D5FA7E4B7E4A20467E49FCF7F6
:1000D000A7FE7E4B7E4A20467E49FCF789FD039BA6
:1000E000002B40F091807C48F9F750F9DDF80CB016
:1000F0007A4E00257A4FDFF82082394602223046B8
:1001000042F00CFF002833785A4614BF0121002129
:1001100020460CBF4FF001094FF000090293FAF797
:10012000B1FD029B8346022B71D17B78192240F2EC
:10013000EE21204612FB03136A4A494601933B789D
:1001400018F8033000932B46F9F74EF9737819220B
:1001500040F2EE21204612FB0313624A4946019306
:10016000337818F8033000932B46F9F7F5F801358A
:1001700002360237122DC0D100215B4B2246504679
:10018000FAF7B0FD210740F1C9800025E9B2013539
:1001900022465046FDF7C8FA042DF7D1534E544D70
:1001A00033782B70059B33B95248F9F7EFF8524971
:1001B0005046FBF7C1FAFF232B700025E9B2013549
:1001C00022465046FDF7D4FA042DF7D173784B4CF4
:1001D0002370059B83BB4A48F9F7D8F84649504637
:1001E000FBF7DAFA4748F9F7D1F84748F9F7A8F8E2
:1001F000FF232370002013B0BDE8F04FFAF74FBD86
:100200001A4A06E72B4620E7DFF8CCB070E73B78C8
:1002100049463E4A204618F8033000932B46F9F72A
:10022000E3F83378394A494618F8033020460093FA
:100230002B46F9F791F89AE7FF23237028E600BFD1
:10024000184D09089F380A08A5380A080C5D0024D3
:10025000AE380A080C780024A05A0024647A0024DE
:10026000BD380A08FFFF7F00C4380A08D2370A08E1
:1002700020730024A0C00908B458002466260A0888
:10028000DC270A08BC6C0024346E0024D0380A082D
:100290003C6D0024B46E0024CB380A08D6380A0816
:1002A000085A002494720024DA380A08806B00246B
:1002B0003C6F0024E3380A08AC6C0024286F00244B
:1002C000EB380A082C5B002420710024F4380A085B
:1002D000145E0024E4780024D6370A086C700024E9
:1002E000386B0024672A0A08DD370A08D078002412
:1002F0008C040024F8380A08B32B0A088D04002463
:100300001B390A0842390A085F380A08772A0A089E
:10031000E0790024AC580024B0C209080F4D2246F1
:1003200050462978FDF700FA224669785046FDF7D5
:100330001FFAADE5A20706D5084B224650461978AC
:10034000FDF7F2F956E763077FF554AF034B2246FA
:1003500050465978FDF70CFA4CE700BFD0780024DE
:10036000002273E4012271E4294B30B583B09A79FD
:100370000190AAB393F82420DFED266A07EE902AB5
:10038000DB79254AF8EEE77AA3F10203234CB3FAAE
:1003900083F3157886EEA77A5B0984F8243084ED20
:1003A000087ADDB11E4BDDED017AB3F89E32F8EE2E
:1003B000677ADFED1C0A00EE103A67EEA00AB8EE8D
:1003C000400AF7F797F804F12803002103EBC50270
:1003D0001960083303ED010A9A42F9D103B030BD28
:1003E000114A12681001F9D593F82420DFED096A4B
:1003F00007EE902ADB79094AF8EEE77A991E4B421C
:1004000086EEA77A4B4182F8243082ED087AE5E740
:100410001C2A002455555540FC0500207C34002042
:10042000A47A0024BD378635BC5900248C4B1B7838
:10043000002B00F0E9808B4B2DE9F04F93F804A1DD
:1004400085B0BAF1010F40F09980874B18780828E1
:100450008646A8BF4FF0080E002800F0FE80834BB0
:100460000021DFED837A40F6FF76D3ED086A9C46E3
:1004700093F824508B4666EEA76A7A4A7D4C019128
:10048000CDE902A3938925B992F81E80B8F1010F36
:1004900009D913F4706F4FEA2329C3F3032802D05C
:1004A00019F0010F6DD0B34200F08D80C3F308083E
:1004B0005B0A08FA03F31FFA83F8B8F1000F00F0A3
:1004C00096806D4F9BB207EB5808B8FBF3F35FFAC9
:1004D00081F8404507D9DFF8B08198F80080B8F17D
:1004E0002D0F08BF23804FF6FF77BB4240F08D8071
:1004F000013114320CF1040C02347145C2D1DDF823
:100500000C80BBF1000F0DD0DDED017AB8EE677AFB
:1005100007EE90BAF8EE677A27EE267AC7EE276ADA
:10052000C8ED1A6ADFED556AC8ED1B6A10B3544A6C
:1005300098ED085A4B4902EB8000A2F14403CC89A4
:10054000083353ED037A143107EE104A53ED025A83
:10055000B0EE676AB8EEC77A97EE056AE5EE867A7E
:10056000E2EC017A904243ED037AC6FEE76AE6D1F7
:10057000C8ED1B6A02233B4A82F8043105B0BDE88E
:10058000F08F404F01EB81095FFA83FA07EB5808BF
:10059000344F98F8808308EB4909B8F1010F07EB55
:1005A0004909029FA9F80EA007FA08F792F81E90D1
:1005B00049EA070982F81E9041D192F81F80C2458E
:1005C00096D9D37794E7CBB298422DD92E4B1B788E
:1005D0002D2B31D00023DFED2D7AD381937F43F093
:1005E000010393770BF1010BCCED007A80E7CBB2DE
:1005F00098427FF67DAF244B1B782D2B7FF478AF8C
:100600004FF6FF73238073E77047019F07EE903A20
:100610001F449BB2F8EEE77AD381937F67EEA67A08
:10062000019743F00103DCE70023DFED187AD38163
:10063000937F43F00103D4E700232380CAE7B8F196
:10064000000F7FF455AF07EE90AA019BF8EEE77A12
:100650005344019367EEA67AC4E7DFF8108061E7A0
:1006600004000020341B0020FC0500207C34002006
:1006700000007042182B0024C0270900FFFF7F7F75
:10068000EC34002098780908142B002400000000A6
:1006900038B5094D2B7963B100242B6820465B6B7C
:1006A00013B10134984708B9002038BD2B799C421A
:1006B000F3D3012038BD00BFC82100200B4B1A7CAA
:1006C00012B90B4B98797047094A906800B9704786
:1006D000084940F6B83C0968091A614503DD002164
:1006E0009079197470470020F1E700BFF0050024ED
:1006F000C8210020B81D00242DE9F04FDFF8349206
:100700001F46531E83B016460546D9F80040142BE9
:1007100000F2CD80DFE803F05D5D5D5D5DCB0B0B2E
:100720000B0BCB0B0B0BCBCBCBCBCB0B0B004FF477
:100730007A734FF00A0A0193012F50D0002F45D150
:10074000764A774B14781878631C03F003038342CE
:100750003CD0137004EB4403DFF8D4814FF47A7279
:100760004FEA440908EBC30383F80CA09A60C1B1B7
:100770001822A5F1FF0002FB0482B0FA80F00C32CF
:10078000400905E038B9013702F8013F8F4208D02F
:10079000AF420346F6D1013733468F4202F8013F9C
:1007A000F6D1FFF775FF002800F0A78009EB0403DE
:1007B0005C4A0120DB00526908EB030108F80300E2
:1007C00042F20F731344B3FBF2F34B6003B0BDE886
:1007D000F08F554B012F4FF0010A0193AED1534AD0
:1007E000537C012B03D0022B00F09280002799F854
:1007F000040008B34A4B1821A5F1FF0E1A780C2308
:10080000BEFA8EFE11FB0231494B4FEA5E1E1944BF
:10081000002307E0BEF1000F08D1013301F801CF3A
:10082000984209D0DAB2F446AA42F3D10133B44671
:10083000984201F801CFF5D142F22830F4F7FAFCE2
:1008400038F0C6FA87B3236A03B1984799F80430A1
:10085000EBB1A5F1FF084FF0000BB8FA88F8584645
:100860004FEA5818E26B90475D45A26A314603D0C3
:10087000B8F1000F00D14146584690470BF10103F3
:1008800099F804205FFA83FB93455846EAD3A3699D
:1008900003B19847E36A98477FB90AF1FF3A1AF023
:1008A000FF0A14D038F094FAE3699847CBE74FF485
:1008B0007A734FF0010A01933EE70AF1FF3AE369C8
:1008C00098471AF0FF0A02D038F082FABBE7019885
:1008D000F4F7B0FC99F80420002A3FF477AF104CED
:1008E0000D2118231248247813FB04130021184407
:1008F00003B0BDE8F04F42F0BDB909EB0403DB00E3
:1009000008EB030208F80300506003B0BDE8F08F65
:100910009778083F18BF012769E700BF801A0024B5
:10092000811A0024F0050024A08601001C2A00245E
:10093000841A0024C82100202DE9F041134C2478AA
:100940000CB9BDE8F08180460F4616461D46BBB186
:10095000012BF6D10E4B98792F2EF2D80028F0D12A
:100960000C4B0D4A1B781278013303F003039342BA
:10097000E7D02B46324639464046BDE8F041BBE65B
:10098000FFF79CFE80F00100C0B2E5E75C6B00243D
:10099000C8210020801A0024811A002410B5437B4E
:1009A00004468268581C6073D154627B237B934257
:1009B00000D802B910BD2368D4E90101984700238B
:1009C000637310BD427B42B1036810B50446D0E9A1
:1009D000010198470023637310BD7047F8B5224E9C
:1009E0003378012B10D1042894BF002301235BB975
:1009F0001E4C0D461E4F04EB4000E188C7F8A032A4
:100A000042892078638800B1F8BD07EE903A6423EC
:100A10009FED187AF8EEE77A03FB02F29FED166A73
:100A200003FB012167EE877A07EE102A06EE901A83
:100A3000B8EEC77AF8EEE66A67EE877A96ED047A42
:100A4000B8EE477A87EEA60A27EE067A20EE070A66
:100A500041F0DAFBB268A3881060084A12681344B8
:100A60002B44BB60F8BD00BFE05D0024CC5D0024DA
:100A7000A47A00240AD7233CCA269B3EB81D002432
:100A8000036810B59B68044698470122FF236273F0
:100A9000A37310BD036810B504461B689847012175
:100AA000236820469B689847E37B0133E37310BDBE
:100AB0002DE9F041069F0D460446164638469846F5
:100AC00040F0A6F82844E672A072387850B1069734
:100AD00029462568204643463246AC69A446BDE80F
:100AE000F0416047BDE8F08103689B6A184700BF8A
:100AF00003685B6D03B11847704700BF0368DB6C88
:100B000003B11847704700BF0B46002110B5C173F1
:100B1000044642749A6C0360017302B190472368E3
:100B2000012120469B689847FF2123680122A17379
:100B3000DB6C62731BB12046BDE81040184710BD46
:100B40000E4B012210B482400D4C1B7854F820004B
:100B5000134071B1003B18BF012338B183F001038A
:100B6000828801681B0102FA03F38B615DF8044B74
:100B70007047B3FA83F35B09EFE700BFCC1D002495
:100B8000C01D002410B50A4C23681B6B9847094B05
:100B9000094A40F2DC5099780023032998BF104697
:100BA000A360A4F80530BDE81040F4F743BB00BFD4
:100BB000C82100201C2A0024FCA607001B4B70B58E
:100BC0005B7906460D46012B18D1194B1B68ABB15A
:100BD000184B0846B3F9A442FAF7F6F898B9284634
:100BE000F7F7B8F900F543730446B3F5C36F0AD9B4
:100BF00030461149BDE87040F9F730BA0F48BDE8FA
:100C00007040F8F7C3BB0E48F8F7C0FB0D48F8F783
:100C100097FBF8F779FB0C4B18680AF029FEFFF7F1
:100C2000B1FF2046BDE87040F5F76ABC582C00249F
:100C3000801D0024A47A0024A2390A0875390A0804
:100C4000BA390A08FA300A08F06A002410B5044CD0
:100C500023681B6998470023A371A36010BD00BFE0
:100C6000C821002010B5074C63791BB12368DB68ED
:100C7000984700B910BD044B01221B68A271A36004
:100C800010BD00BFC8210020B81D0024F8B5114DCB
:100C9000002452272E1D013415F8010BF1F7B2FC88
:100CA00000222021E4B218B18771C471F0F754FE1C
:100CB00016F8010BF1F7A6FC4FF0530C002240216F
:100CC00020B180F806C0C471F0F746FE042CE2D1D2
:100CD000F8BD00BF4C7D0024C3B25E2B05D8044B89
:100CE00003EB8003D3F8880370470248704700BFC6
:100CF00098780908DCF0090838B50C4614F8011B8F
:100D000041B105462B6828461B68984714F8011B1B
:100D10000029F7D138BD00BF03681B68184700BF22
:100D200003682DE9F0415F6A1FB13B46BDE8F04121
:100D3000184704460D46164600E023689B68204687
:100D400098478642F9D8002E08DD2E4423682046B5
:100D500015F8011B1B689847B542F7D1BDE8F08133
:100D600003685B68184700BF03689B68184700BFAB
:100D70000368DB68184700BF03685B69184700BF5A
:100D800003689B6A03B11847704700BF0368DB6ABA
:100D900003B11847704700BF03682DE9F0411646BC
:100DA0009A6A04460D460AB1904723685F6A5FB1AC
:100DB000324629462046B8472368DB6AC3B120463D
:100DC000BDE8F041184723689B6820469847B04229
:100DD000F9D3002EF0DD2E442368204615F8011BC0
:100DE0001B689847B542F7D12368DB6A002BE6D130
:100DF000BDE8F08170B504460E46154623682046CE
:100E00009B689847A842F9D32A4631462046BDE858
:100E10007040C1E72DE9F04F804D8FB095F8DD604F
:100E200016B10FB0BDE8F08F7D4F3B685C05F8D57B
:100E3000D5F8DC3404467B4AC31A93425FDC95F84C
:100E4000E034002BEDD095F8E4349807E9D195F81B
:100E5000EC2442B1D5F8F00410B17349FFF79CFFC0
:100E6000002385F8EC3495F8ED34002B40F0C48075
:100E700095F8C437002B47D195F89324002A40F009
:100E80007E816A4BD5F8C807196895F8CC373BB115
:100E9000674BD5F8D0679E4202D18842C0F083816B
:100EA00095F8F827634BB3FBF2F3D5F8C02713444A
:100EB0009C42B6D395F80338C5F8C0472B4493F845
:100EC000FC47E10700F17883620700F11B832307E9
:100ED00000F1F782E10600F1A882A20600F18D82FE
:100EE000630600F17B8295F8033895F8F827013303
:100EF000B3FBF2F102FB113385F8033891E71CF0E4
:100F0000A7FFC5F8DC449AE74B4BC8274B4A06A815
:100F10004B4900260092A3F13F0285F89C74CDE96D
:100F20000423484B484AF6F731FEDDF810802921AA
:100F3000EA2208F1010306A8049388F80060049BE4
:100F400003F1010CCDF810C01970049B591C0491D9
:100F50001A70049B5A1C04921F703FF059FE471CE4
:100F600006A904983A4641F027FE0499012204A8F4
:100F7000CB1913440493CE55049B991804911E7009
:100F8000049B991804911E70049B991804911E707B
:100F9000049B991804911E70049B991804911E706B
:100FA000049B991804911E70049B991804911E705B
:100FB000049B991804911E70049B991804911E704B
:100FC000049B991804911E70049B991804911E703B
:100FD000049B991804911E70049B991804911A702F
:100FE000049BA3EB080388F800302BF01DF985F86B
:100FF000C467C5F8C04714E795F8EE34002B40F0FD
:101000008081D5F89435002B00F0B480DFF83C8067
:101010000027A8F5217908F1680A7DE0A47A002468
:10102000BC590024BFC62D00987F0024B81D0024A1
:1010300078820024A0860100807F0024A35300242E
:1010400040F1090824F1090834F10908D87F002487
:10105000012A00F02981052E50D9437800F1060EAF
:10106000811985F8B8374388A5F8B4378388C02B31
:1010700000F28F8100224B44CF48A5F8B627012209
:10108000C5F8AC97C5F8B03785F8BC27A3EB000BC3
:10109000A1EB0E0285F8BDC75A45C0F26381BBF1D2
:1010A000000F40F03481C54BC54AC5F8B0079869B8
:1010B000002302F11001C5F8AC9785F8BC37C5F8DC
:1010C000A437069306ABC5F89CA7C5F8A0270AF07D
:1010D00083FC013000F05581069B0BB1002098473E
:1010E000D5F89C37C5F89CA7C5F8A03795F8EC341F
:1010F000002B00F0EB80012385F8EE3401363744F5
:10110000EFF31183502282F31288D5F89425974289
:1011100028DADBB283F31188EB1993F83465012EDA
:10112000ECD9791C6B1893F83435C3F3411203F0F2
:101130000F0C032A85F8982500F0CD8013F01003DA
:1011400008EB010084D195F8BC27002AD6D095F889
:10115000BD27013202F00F02624500F0CA8085F817
:10116000BC37CBE7002295F8EE64DBB2C5F89425D6
:1011700083F3118885F8ED64C5F8C04751E6914ABC
:101180004FF4327185F8933406A8A2F13A03A5F81A
:10119000A014CDE906328C4BC5F89C342BF044F8F2
:1011A000C5F8C0473DE695F89014002940F0B78097
:1011B000D5F8E80700283FF473AED0E900218A4251
:1011C0003FF46EAED5F8F037D5F8F427E31A934222
:1011D0007FF766AE95F8EC277A4B85F8A2247B4A18
:1011E000A3F1380795F8EDE7C5F89C244FF4E472B5
:1011F00085F8A3E4A5F8A024CDE90673D0E900A9F9
:10120000D14500F05F83A3F1060C4FF00008CA45FA
:10121000ACEB070B9AF8006000F0FF825346002207
:1012200003E0994502F1010203D013F8011B8E423D
:10123000F7D093B25FFA8BFB012B00F2B1829B4592
:1012400080F0EC82CA4500F03D836745DFD3BEF1F4
:10125000000F07D195F8A23463F07F0385F8A2341C
:10126000D0E900A9CA4500F03183069B06A8584E74
:101270009B1B85F89D342AF0D7FF95F8EC244AB1E2
:10128000D5F8F00418B106F15701FFF785FD0023EA
:1012900085F8EC3495F8ED37C5F8F0470133C5F81B
:1012A000C04785F8ED37BCE5022E3FF427AF8378C1
:1012B000A5F8B4374378FF2B5FD1042E7FF61EAF1D
:1012C000B0F8033000F1050E8119D0E635F0AEFC20
:1012D00085F8EE0412E73F4BC5F89C370133C5F89B
:1012E000A037002385F89C35A3F52023C5F8A43743
:1012F000FCE600F1010E8119D5F8B037D5F8AC073E
:10130000C4E635F093FC064685F8EE0432E77146F4
:101310005A4641F051FCD5F8AC075844C3E695F85D
:10132000EC1785F89024013185F8ED272A4A82FBD5
:1013300001020A445211C2EB8212891AA3F26442DA
:10134000A3F5507385F8EC17184695F89214C5F874
:10135000E83795F89134C5F8942403FB0121C5F8CA
:1013600098142CE77146039241F026FCD5F8AC376F
:10137000039A1344C5F8AC37C0E600F1030E811997
:1013800075E6D5F89C370222591CC5F89C171A70CF
:10139000A2E6104BC5F89C370133C5F8A037B5F865
:1013A000B437A5F8A437032385F89C354FF6F673B8
:1013B000A5F8A6379AE600BF547D0024F005002466
:1013C00040820024807F0024C8057DEAC8007DEAB1
:1013D000417F002440800024832008826E4BC82473
:1013E0006E4A06A8A3F13B0185F8A044C5F89C24E9
:1013F000CDE906132AF018FF75E5674B4FF49961A4
:10140000B5F88C2006A807933B3B120AA5F89C145C
:1014100006930721B5F98C3085F89F2485F89E1432
:1014200085F8A0342AF000FF5AE5AA8F242064260C
:10143000AB6900FB02F269691BBA574F323209BA35
:10144000C5F8A334EB8FC5F89F14002103EB830389
:1014500095ED150A07972E3F5B00B2FBF6F2C2F33B
:10146000072060F3070162F30F21C3F307229BB249
:1014700062F3174163F31F6141F2C813A5F89C346E
:101480000223C5F8A71485F89E3440F0BDFE444AF7
:10149000034606A806979342A8BF134623EAE373C0
:1014A000B3FBF6F303F57A73C3F3072285F8AC3484
:1014B00095F8403085F8AB2485F8AD342AF0B4FEB9
:1014C0000BE5C823344AA5F89C342123079285F8FC
:1014D0009E34B5F8E2305E0540F1C881314B393AAF
:1014E00018680692C5F89F04069B00212E4A581CD6
:1014F000069006A81970069B9B1A85F89D342AF061
:1015000093FEE7E4244A40F6C82307920822A5F890
:101510009C3495F80F3885F89E24002B00F08A81C2
:10152000224B1B781BB1224A1288B2FBF3F305331E
:101530000A22B3FBF2F3C3F30720DBB2D5F830186D
:101540000A22D5F838881B4E91FBF2F1002206964C
:10155000043660F3070263F30F22C1F3072363F33A
:10156000174261F31F62C5F89F240FF007FA4FEA94
:1015700018420023069662F307034FEA182262F32B
:101580000F2368F3174360F31F6306A8C5F8A3345D
:101590002AF04AFE9BE400BF807F0024C8040B00B1
:1015A00020A107001CF10908417F0024B46A00242F
:1015B000A46A0024477F002440F6C803A24AA5F885
:1015C0009C34B5F95A3107921E22B3F5E16F85F8C4
:1015D0009E2440F382819AB2A2F561631BB2B3F5F7
:1015E000E16F2CDDA2F5E1531BB2B3F5E16F26DD0F
:1015F000964B13441BB2B3F5E16F20DDA2F56153A6
:101600001BB2B3F5E16F1ADD914B13441BB2B3F576
:10161000E16F14DD8F4B13441BB2B3F5E16F0EDDA8
:101620008D4B13441BB2B3F5E16F08DDA2F5E14326
:101630001BB2B3F5E16F02DD884B13441BB207EE1A
:10164000903A9FED877AF8EEE77A67EE877AFDEEBB
:10165000E77A17EE903AC3F3072285F8A034B5F97C
:10166000583185F89F24B3F5E16F40F3C6819AB2F3
:10167000A2F561631BB2B3F5E16F2CDDA2F5E15376
:101680001BB2B3F5E16F26DD704B13441BB2B3F50B
:10169000E16F20DDA2F561531BB2B3F5E16F1ADDF6
:1016A0006B4B13441BB2B3F5E16F14DD694B13446C
:1016B0001BB2B3F5E16F0EDD674B13441BB2B3F5FC
:1016C000E16F08DDA2F5E1431BB2B3F5E16F02DD86
:1016D000624B13441BB207EE903A9FED617AF8EE2D
:1016E000E77A67EE877AFDEEE77A17EE903AC3F372
:1016F000072285F8A234B5F95C3185F8A124B3F549
:10170000E16F40F334819AB2A2F561631BB2B3F585
:10171000E16F2CDDA2F5E1531BB2B3F5E16F26DDDD
:101720004A4B13441BB2B3F5E16F20DDA2F56153C0
:101730001BB2B3F5E16F1ADD454B13441BB2B3F591
:10174000E16F14DD434B13441BB2B3F5E16F0EDDC3
:10175000414B13441BB2B3F5E16F08DDA2F5E14341
:101760001BB2B3F5E16F02DD3C4B13441BB207EE35
:10177000903A9FED3B7A06A8F8EEE77A67EE877A13
:10178000FDEEE77A17EE903AC3F3072285F8A4340A
:10179000344B85F8A32406932AF046FDFFF794BB4B
:1017A00012F0FF0146F0800614BF0127002707EB67
:1017B0001327FBB2BBEB430F1F46FFF648AD0123D7
:1017C000AFB19F4203F1010918D8DDF818A00AF162
:1017D000010306938AF80060069B03F1010ACDF825
:1017E00018A0197001D04B46EBE7D0F804900368BD
:1017F00013FA82F303609A46069F23E5069B03F1E2
:10180000010ACDF818A01E70069B03F1010ACDF85D
:1018100018A083F800804B46D3E700227B1C069378
:101820003E700368D0F8049013FA82F20260924688
:10183000069F07E50C4B0A221B880533B3FBF2F326
:10184000C3F30720DBB279E6807F0024D0D5FFFF09
:10185000B0B9FFFFA0ABFFFF909DFFFF7081FFFFBE
:1018600058A08B41497F0024A46A0024D5F83C2865
:10187000D0057AD4190540F12881A64E30463FF0B4
:10188000C7F93146A44E02468046304641F094F9ED
:101890002B7906EB080113F0010206917FF424AEC8
:1018A0003B6813F0800340F0EE809C4A1268002AE7
:1018B00059D1002B0CBF2A233F23013106F80830F1
:1018C000069111E6BEF1000F3FF4C4AC95F8A234C6
:1018D00043F0400385F8A234C7E413F5E16FBFF687
:1018E000AEAE9AB202F561631BB213F5E16FBFF6BB
:1018F000A6AE02F5E1531BB213F5E16FBFF69FAE42
:1019000042F6302313441BB213F5E16FBFF697AED6
:1019100002F561531BB213F5E16FBFF690AE44F2CE
:10192000506313441BB213F5E16FBFF688AE45F266
:10193000604313441BB213F5E16FBFF680AE46F26D
:10194000702313441BB213F5E16FBFF678AE02F5B6
:10195000E1431BB213F5E16FBFF671AE47F690633A
